:020000040002F8
:10700000608F0020C5730200CD730200CF730200B1
:10701000D1730200D3730200D57302000000000098
:10702000000000000000000000000000D773020014
:10703000D973020000000000DB730200DD73020060
:10704000717F0200DF730200018902002D850200BA
:1070500041850200DF730200B17E0200D58202008A
:10706000D1880200E9880200DF730200DF730200AA
:10707000DF730200DF730200DF730200DF730200C0
:1070800011890200CD7F0200DF730200DF7302006E
:10709000DF730200DF73020069850200DF73020004
:1070A000DF730200DF730200DF730200DF73020090
:1070B000B97F0200DF730200000000000000000042
:1070C000DF730200DF730200DF73020055850200E8
:1070D000E57F0200DF730200DF730200DF7302004E
:1070E000DF7302000000000000000000000000004C
:1070F00000000000DF73020000000000DF730200E8
:10710000000000000000000000000000000000007F
:10711000000000000000000000000000000000006F
:10712000000000000000000000000000000000005F
:10713000000000000000000000000000000000004F
:10714000000000000000000000000000000000003F
:10715000000000000000000000000000000000002F
:10716000000000000000000000000000000000001F
:10717000000000000000000000000000000000000F
:1071800000000000000000000000000000000000FF
:1071900000000000000000000000000000000000EF
:1071A00000000000000000000000000000000000DF
:1071B00000000000000000000000000000000000CF
:1071C00000000000000000000000000000000000BF
:1071D00000000000000000000000000000000000AF
:1071E000000000000000000000000000000000009F
:1071F000000000000000000000000000000000008F
:10720000DFF810D000F042FA0048004705CF020036
:10721000AFF30080608F002030B450E8012F93B2AC
:10722000C48923448489A34228BF1B1B0489A34229
:1072300002BFBFF32F8F002007E0C3EA020340E83C
:107240000134002CE9D14FF001000A6030BC7047D6
:1072500050E8012FC2EA024240E801210029F7D19B
:10726000704730B450E8022F1FFAA2F3C488A3423B
:1072700002BFBFF32F8F00200DE0C489234484890F
:10728000A34228BF1B1BC2EA034340E80234002C80
:10729000E8D14FF001000A6030BC704750E8022F7F
:1072A000C2EA224240E802210029F7D17047034692
:1072B00053E8022FD988B2EB324F4FF0000017BFCE
:1072C00092B241EA014142EA014104E05A68B2EB5C
:1072D000324F08BF012043E80212002AE8D170476C
:1072E00030B4044654E8000F0D4644E80053002B28
:1072F000F8D1156030BC704730B4044654E8000F34
:1073000040EA010544E80053002BF7D1156030BC7A
:10731000704730B4044654E8000F00EA010544E821
:107320000053002BF7D1156030BC704730B40446D1
:1073300054E8000F80EA010544E80053002BF7D120
:10734000156030BC704730B4044654E8000F00EBC1
:10735000010544E80053002BF7D1156030BC70479D
:1073600030B4044654E8000FA0EB010544E8005394
:10737000002BF7D1156030BC704770B404464FF055
:10738000000054E8006F0D68AE4207BF44E80023D8
:10739000012044E800630E60002B1CBF0020F0E7D2
:1073A00070BC704730B4044654E8000F88422CBFCC
:1073B000451A054644E80053002BF5D1156030BC52
:1073C000704700000648804706480047FEE7FEE792
:1073D000FEE7FEE7FEE7FEE7FEE7FEE7FEE7FEE785
:1073E000158702000172020000487047E443030061
:1073F00010B50446FFF7F8FF0068005D00F00100DB
:1074000010BD40EA01039B0703D009E008C9121F21
:1074100008C0042AFAD203E011F8013B00F8013B4E
:10742000521EF9D27047D2B201E000F8012B491E7A
:10743000FBD270470022F6E710B513460A46044611
:107440001946FFF7F0FF204610BD421C10F8011B43
:107450000029FBD1801A704730B50446002003464E
:1074600000E05B1C934203D2E05CCD5C401BF8D093
:1074700030BD034611F8012B00F8012B002AF9D189
:10748000184670470FB400B58DB010A909900B9045
:1074900000914FF0FF300A9000200C9005480690B4
:1074A000054807906A4609A80F9900F0C1F80DB089
:1074B0005DF814FB4D7602006B7602002DE9FF5F4C
:1074C0001D464FF0FF3BD5E9014691465F464FF020
:1074D0000008A9697F1C01988847296A8246884765
:1074E0000028F6D1BAF1FF3F0CD024F4C064002E7E
:1074F00019DD600614D5BAF12B0F09D0BAF12D0FA2
:107500000ED103E0584604B0BDE8F09F44F4806417
:10751000A9697F1C01988847761E8246002E02DDED
:10752000BAF1300F03D0B9F1000F26D032E0A969CB
:10753000761E44F400747F1C019888478246002E12
:1075400005DDBAF1780F06D0BAF1580F03D0B9F1C2
:10755000000F10D01EE0B9F1000F02D0B9F1100FEA
:1075600018D1A969761E24F400747F1C01988847FD
:107570008246102002E0082000E00A20814609E04F
:1075800008FB0908A969761E44F400747F1C019861
:1075900088478246002E05DD4946504600F034F803
:1075A0000028EDDAE96901988847A00502D46FF058
:1075B0000100A8E7E00725D1600613D5600502D5D4
:1075C000C8F1000000E0404629680A1D2A600968E9
:1075D000220501D5087015E0220701D5088011E0C9
:1075E00008600FE02868011D29600068210502D5A8
:1075F00080F8008006E0210702D5A0F8008001E0B5
:10760000C0F8008038467EE73A2800D2303820F0B3
:107610002002412A01D3A2F13700884201D34FF062
:10762000FF307047026811441378016018467047B4
:10763000D160044951610449116200211161114670
:1076400000F036B825760200F1730200426842B1BC
:10765000016811F8013B23B1521EC0E9001218461F
:1076600070470121C160881E704742685AB1C368E3
:10767000016843B983688B4205D0491E521CC0E99A
:107680000012002070474FF0FF307047064C074D46
:1076900006E0E06840F0010394E8070098471034E2
:1076A000AC42F6D3FFF7B0FD9C4E0300BC4E030086
:1076B0002DE9F34F8BB04FF0000801F10C000C46A0
:1076C0004FF0010B46460DF1080A01906269012155
:1076D00001989047051E2DD0252D2CD0216A884772
:1076E000C0B16269012101989047216A884700284A
:1076F000F7D1411E62690198904700E0761CA169AC
:107700000B988847216A88470028F7D1E1690B98D0
:107710008847DBE7A1690B9888470746A84201D153
:10772000761CD3E7E1690B9888477F1C02D1B8F13A
:10773000000F6FD047E1002762693D463946019846
:1077400090472A2804D162690121019890470125B8
:10775000DFF888926269012101989047A0F1300119
:107760000A290AD24F45E5DC07EB870100EB410708
:10777000303FDFD445F01005ECE7E90601D46FF0A7
:1077800000476C280AD04C2814D0682815D06A28E5
:107790000DD074281CD07A281AD01DE0626901210E
:1077A000019890476C2802D045F0040514E045F09C
:1077B00002050DE045F020050AE06269012101980B
:1077C0009047682802D045F0080505E045F40065BB
:1077D0006269012101989047C4E9015765283DD0AD
:1077E00019DC58287AD00CDC452837D004DC252851
:1077F00026D0412831D131E046282FD047282CD13E
:107800002CE05B2877D0612828D063287CD06428BE
:1078100023D15AE0D1E06F2848D008DC66281DD07B
:1078200067281BD0692821D06E2816D127E0702840
:1078300045D0732868D0752847D078280DD14DE001
:10784000A1690B988847054625283FF469AFE1698F
:107850000B9888476D1C3FF46AAFB4E023466A4634
:107860006FF001000B99AFF300809FE045F04000FE
:107870006060A80723464FF0000236D43EE0E807D8
:107880007FF447AF2068011D21600068290501D5FC
:1078900006701BE7290701D5068017E7A90703D55E
:1078A000F117C0E9006111E706600FE745F04000FD
:1078B0006060A80723464FF0080216D41EE040F689
:1078C0000E0125EA0100606016E045F040006060AE
:1078D000A80723464FF00A0207D40FE045F0400006
:1078E0006060A80708D5234610226FF001000B99AD
:1078F000AFF300805AE007E0234610226FF001004A
:107900000B99FFF7DBFD51E04FF000094F464B4666
:10791000632802D05B2807D041E02079C00601D45B
:107920000120A06001273AE0626901210198904797
:107930005E2805D14FF001096269494601989047D8
:10794000216939B900210A46534643F82120491CD0
:107950000829FADBB0B3216969B9C11700EBD1621C
:1079600053110AEB830122F01F02821A01200B68D7
:10797000904003430B6062690121019890475D28A4
:10798000E8D1B9F1000F09D00020514651F820206C
:10799000D24341F82020401C0828F7DB02AB2246E6
:1079A00000976FF001000B99AFF3008000280CDA0C
:1079B000401C08D1BBF1000F05D04FF0FF300DB0D7
:1079C000BDE8F08FFFE74046F9E7E90701D108F18C
:1079D000010806444FF0000B78E60000CCCCCC0C3C
:1079E00070B58C1810F8015B15F0070301D110F881
:1079F000013B2A1106D110F8012B03E010F8016BAE
:107A000001F8016B5B1EF9D12B0705D40023521E30
:107A10000DD401F8013BFAE710F8013BCB1A921C98
:107A200003E013F8015B01F8015B521EF9D5A14296
:107A3000D8D3002070BD00002CB5294800F080F894
:107A400028480078002847D100BF274A012127484D
:107A500001F046FE0546D5B125482649264A891A31
:107A6000C9080322CDE9000542EA014040F215238E
:107A700022A228A106F0F4FD06F02CFC00BF00BFF6
:107A800024B100BF204601F05DFB00BF00BF00BF76
:107A900000BF284A0021284801F022FE0546D5B142
:107AA00026481449144A891AC9080322CDE9000559
:107AB00042EA014040F2162310A216A106F0D0FDC2
:107AC00006F008FC00BF00BF24B100BF204601F053
:107AD00039FB00BF00BF00BF0120024908702CBD68
:107AE00061910200D52C002051800200783F0300F4
:107AF00034440300644F0300CC4E03007372635C94
:107B00006170705F626C655F736572766963652E24
:107B10006300000025733A2564205A4552524F52A3
:107B20005F434845434B28257329206661696C3AB9
:107B300025640000158002007C3F03008C44030094
:107B400004490A680968491C024B1960024941F856
:107B500022007047402D00202455002010B52048F9
:107B60000078022800D110BD01221EA1002004F0DF
:107B70005BF9002003F042FE00221146052006F0CA
:107B80006FF9002211460B2006F06AF90022114617
:107B9000112006F065F900221146042006F060F974
:107BA00001211E2006F066FA642005F02DFE00215A
:107BB0001E2006F05FFA0021012006F05BFA00218A
:107BC0001C2006F057FA1E2005F01EFE01211C2085
:107BD00006F050FA02200249087000BFC3E7000017
:107BE000442D0020000000002DE9F843574800789C
:107BF000012801D1BDE8F88301211E2006F03AFAE0
:107C00000121084606F036FA1E2005F0FDFD002190
:107C10001E2006F02FFA01244FF00A0805E000208C
:107C200003F088FC0446A8F10108B8F1000F01D068
:107C3000002CF4D1002C25D04549464A891AC908A0
:107C4000032242EA0140224643A106F0D9FC00BFCC
:107C500049A03F493F4A891AC9080322009042EAD5
:107C600001409A2345A24DA106F0E6FC06F032FB46
:107C700000BF4FF0000800BF002001F063FA00BF12
:107C800000BF00BF3249334A891AC908032242EAB9
:107C9000014048A106F0AAFC01224EA14E4804F082
:107CA000C3F80546002D24D029492A4A891AC90853
:107CB000032242EA014049A106F098FC00BF2EA031
:107CC0002349244A891AC9080322009042EA014044
:107CD000A1232AA231A106F0AFFC06F0FBFA00BFF7
:107CE0004FF0000800BF002001F02CFA00BF00BFD9
:107CF00000BF3E48006841693C48884740684FF4EF
:107D00008011B1FBF0F6394800684169374888476F
:107D10000068B0FBF6F70E490E4A891AC90803221B
:107D200042EA014032A106F061FC0949094A891A78
:107D3000C908032242EA01403A4631A106F060FC3C
:107D400001200249087000BF54E70000442D0020C4
:107D5000644F0300CC4E03004469736B20696E6965
:107D60007469616C697A6174696F6E206661696CAF
:107D700065642E2025640000300000007372635C8F
:107D8000626F6172645C626F6172645F736463618D
:107D900072645F6472697665722E630025733A259A
:107DA00064205A4153534552542825732920666153
:107DB000696C00004469736B20696E697469616C59
:107DC000697A6174696F6E20737563636565646554
:107DD000642E0000000000004C5500204D6F756EB1
:107DE00074206661696C65642E000000803F0300AA
:107DF0004D6F756E74207375636365737300000057
:107E000043617061636974793A202564204D4200B2
:107E10000148007870470000442D002010B51E482E
:107E2000007800B110BD00221146052006F018F8B8
:107E3000002211460B2006F013F8002211461120F3
:107E400006F00EF800221146042006F009F803217E
:107E50001C200CF061F801211C2006F00BF9032115
:107E600001200CF059F80021012006F003F903214C
:107E70001E200CF051F800211E2006F0FBF8002017
:107E8000064908700121064803F0A2FD01200249BD
:107E9000087000BFC6E70000452D0020442D0020DB
:107EA000482D00200148007870470000282D002050
:107EB0002DE9FC4700260020009001904FF48077C8
:107EC0000125002410E0384606F00AF940B100BF51
:107ED00025480068284018B1384606F0F3F82E43CC
:107EE0006D00381D87B2641C082CECD34FF4BE70B3
:107EF00006F0F6F850B14FF4BE7006F0E3F846F025
:107F000000466A460221002005F0E4FFF0B210B3FB
:107F1000012500241DE005EA0600C0B100BF13489A
:107F200050F82400C0F30520814600BF0F4850F8E8
:107F30002400C0F301408246204602F05BFD8046EB
:107F4000B8F1000F02D051464846C04700BF6D004F
:107F5000641C082CDFD306F0004010B1684608F01E
:107F60005DFBBDE8FC870000046300401065004035
:107F700010B54FF4807005F02BFC50B14FF48070B9
:107F800005F02FFC012005F035FC0A4801680020AF
:107F900088474FF4827005F01BFC50B14FF482709B
:107FA00005F01FFC022005F025FC024801680120B5
:107FB000884710BD642D002010B50249024804F026
:107FC000CFFD10BD742D002000C0014010B5034A44
:107FD0001068034A1168884710BD0000C82D0020B2
:107FE000C42D002010B504220021024804F00AFE2E
:107FF00010BD00000040024010B500200349087089
:108000000348006801F0E5FB002010BDD42C0020DF
:10801000783F030010B504460248006800F004F8F9
:1080200010BD0000D02C002070B50546074C072677
:108030006A20A0700020607003202070C4F80350F4
:10804000314620460BF097FD70BD00001C4F00200C
:108050002DE9FC4E81466548007808B9BDE8FC8EE4
:108060006348006800284AD14FF480716148FFF7E7
:10807000E1F94FF480725F495F48006800F0C2FA8E
:108080008246BAF1000F36DC5C495D4A891AC9089C
:10809000032242EA01405BA106F0A8FA00BF604853
:1080A0004FF4F67102685F48006801F063FB834695
:1080B000BBF1000F1BD05C485049514A891AC908CE
:1080C0000322CDE9000B42EA0140C42357A25DA17F
:1080D00006F0C6FA06F0FEF800BF00BFB8F1000FC8
:1080E00004D000BF404601F02DF800BF00BF00BF24
:1080F000FFF782FFB2E73E48C0F800A000BF3C484F
:10810000006800B9AAE70BF013FB0546802D01DAE1
:10811000284600E08020054635480068C0F580709C
:108120003449461832480068A84201DD284601E07B
:108130002F48006807463149314A891AC908032285
:1081400042EA01402A4900953A460B6845A106F0EB
:1081500073FA0BF0DBFD60B92849294A891AC9086E
:10816000032242EA014043A106F040FAFFF744FF30
:1081700074E7B8B2019001A930460BF0A3FC0446A5
:1081800000BF0CB3082C0CD11C491D4A891AC90820
:10819000032242EA01403FA106F028FAFFF72CFF34
:1081A0005CE7112C01D0132C00D157E71349144A76
:1081B000891AC908032242EA014022463DA106F07D
:1081C0001FFAFFF719FF49E7002006E0315C144A67
:1081D00012681144124A1160401CB842F6D3044898
:1081E0000068C01B0249086000BF37E7D42C00209C
:1081F000CC2C002040510020C82C0020644F0300EC
:10820000CC4E0300726561642066696C6520656E02
:10821000642C73746F702075706C6F616400000063
:10822000D02C00207C3F0300104503007372635C78
:108230006170705F626C655F736572766963652EED
:108240006300000025733A2564205A4552524F526C
:108250005F434845434B28257329206661696C3A82
:108260002564000075706C6F6164202564202564AE
:1082700020256400626C6520697320646973636FF4
:108280006E6E65637465642C73746F702075706CAA
:108290006F616400626C6520756E656E61626C650D
:1082A000206E6F746966792C73746F702075706CB2
:1082B0006F616400626C652073656E642065727224
:1082C0006F722C73746F702075706C6F61642025F1
:1082D00078000000FEB54FF4827006F057FC0028CD
:1082E00037D04FF4827006F05BFC6C4890F82E009B
:1082F00018B16A4890F82F0058B300208DF800009C
:1083000066484068019065480189ADF80810C0686A
:1083100018B900206149087412E06048008B5F4979
:1083200048830846C06848600846008B08810020E2
:10833000C860084690F82E0010B9002006F03CFCFA
:1083400056480168684688470020544981F82F0044
:1083500000BF524890F82E00002852D04FF4807091
:1083600006F014FC00284CD04FF4807006F018FC86
:108370004A48408B494991F82D10884216DD4748FC
:10838000408B464991F82D10401A444948830A46CB
:1083900012890B465B8BD21A0B465B6803EB4200DB
:1083A0000A4692F82D1006F0E9FB23E03B48408B8B
:1083B0003A4991F82D1088420FD13848C06860B111
:1083C0000120364981F82F00002048830A4692F8A0
:1083D0002D10D06806F0D2FB0CE03048408B2F49BE
:1083E00091F82D10884205D101202C4981F82F00E9
:1083F000002048834FF4827006F0D2FB042006F080
:10840000DBFB4FF4887006F0C1FB70B14FF488704D
:1084100006F0C6FB00202149087402208DF80000F8
:10842000084601686846884700BF4FF48A7006F026
:10843000ADFB38B14FF48A7006F0B2FB002017494B
:1084400008742AE01548456924E0B5FA85F64FF02E
:108450000040F0408543B00000F58C74204606F0E3
:1084600095FBB8B1204606F09BFB01208DF800007B
:10847000A4F58C70C0F3C7008DF80400A4F58C70CF
:10848000012121EA90018DF8051004480168684631
:10849000884700BF002DD8D100BFFEBDF058002096
:1084A00010B500F055FA10BD2DE9F0470746884693
:1084B0001646C24607EB47011B4800EBC109D9F835
:1084C000140020B1012811D0022826D11EE0484610
:1084D00000F076FA0546B54201D2002405E03446A4
:1084E00032465146484600F0B2FA18E0484600F0DD
:1084F00067FA0546B54201D2284600E030460446F8
:1085000022465146484600F0A2FA08E0324651465B
:10851000484600F063FA044601E0002400BF00BFB3
:108520002046BDE8F08700006078002010B50249C1
:10853000024804F003FB10BD205900200030004029
:1085400010B503494FF040200AF008FD10BD0000AF
:108550008859002010B50249024804F0EFFA10BD16
:10856000445900200030024010B506F029FD10BD2E
:1085700010B50949094A891AC908032242EA01408B
:1085800007A106F033F8FFF743FC012801D108F0FA
:1085900085FAFFF7E3FA10BD644F0300CC4E0300E9
:1085A0006368616E676520746F20657874206D6FF5
:1085B0006465000010B50749074A891AC9080322F3
:1085C00042EA014005A106F011F8FFF70DFB08F0A3
:1085D00065FA10BD644F0300CC4E03006368616E02
:1085E000676520746F206C6F63616C206D6F6465CC
:1085F0000000000010B5FFF711FCFFF7DBFFFFF7ED
:10860000B7FF10BD2DE9FC4180460D46164600BF60
:1086100021480078002817D120A02349234A891A2D
:10862000C9080322009042EA01408F2320A229A119
:1086300006F002F805F04EFE00BF002700BF002044
:1086400000F080FD00BF00BF00BF01AB32462946ED
:10865000264803F00EFD044600BF002C17D024A0CE
:108660001149124A891AC9080322009042EA0140BE
:1086700092230FA217A105F0DFFF05F02BFE00BF2C
:10868000002700BF002000F05DFD00BF00BF00BF5D
:108690000198BDE8FC810000F82C00206D5F697333
:1086A0005F6F70656E000000644F0300CC4E0300E6
:1086B0007372635C73616D706C655F646174615F3C
:1086C0006D616E616765725F736572766963652E51
:1086D0006300000025733A2564205A4153534552E4
:1086E0005428257329206661696C0000EC52002033
:1086F00066665F726573756C74203D3D2046525FFF
:108700004F4B000001480249086070470090D003B9
:10871000702E002010B504F015FE40B10020644911
:1087200008604FF08041C1F810016249086004F010
:1087300023FE002855D060480068604908605E4804
:10874000001D0068091D08605B4808300068091DAD
:10875000086059480C300068091D08605648103000
:108760000068091D0860544814300068091D08603D
:108770005148183000685149203108604E481C307B
:108780000068091D08604C4820300068091D086019
:10879000494824300068091D0860474828300068AF
:1087A000091D086044482C300068091D08604248D3
:1087B000303000684149403108603F48343000683B
:1087C000091D08603C4838300068091D08603A48B7
:1087D0003C300068091D0860374840300068091DBA
:1087E000086004F07BFD40B13548006800F00100EE
:1087F00018B16FF00100324908603248006840F457
:1088000070003049086000BF00BF00BFBFF34F8F4A
:1088100000BF00BF00BF00BF00BF00BFBFF36F8F2E
:1088200000BF00BF00BF00BF04F072FD20B12648AA
:10883000006820492031086000BF2348001D0068FF
:1088400000F0010080B3012007F024F91E48001D4C
:10885000006820F001004FF01021C1F80C0207F071
:1088600023F9002007F016F900BF00BF00BF00BFCA
:1088700000BFBFF34F8F00BF00BF00BF11487C385F
:10888000006800F4E06011490843001D0D497C397F
:10889000086000BF00BF00BFBFF34F8F00BF00BF25
:1088A00000BF00BF00BFFDE7FFE7FFF72BFF10BDD4
:1088B0000C010040380500400404001020C50040B1
:1088C0000004004088ED00E0081200100000FA05E6
:1088D00010B504220249034804F0F0F910BD00006D
:1088E000C45900200080004010B50422024903480A
:1088F00004F0E4F910BD0000D059002000900040C1
:1089000010B502490868804710BD00006C2D00209A
:1089100008B500BF4FF480700B49405808B10120E2
:1089200000E0002078B109480068804700BF0020BF
:108930004FF48071044A8850084611464058009010
:1089400000BF00BF00BF08BD00000140802D002017
:1089500010B5124C02202061606111A0A061134982
:10896000E1614FF4007121620021A1626162E16264
:108970000BA0A0640E49E164102121650021A165CE
:108980006165E1650BA1E01DFEF773FD0AA12046BC
:10899000FEF76FFD2020A07110BD00004878002078
:1089A0005465726D696E616C00000000C078002033
:1089B000C07A0020525454005345474745520000A6
:1089C00010B501460A69CB689A4204D88C68641EC7
:1089D000E41AA01801E0D41A601E10BD2DE9F0477A
:1089E0000446894617464FF0000AE56800BFD4F8F0
:1089F0001080A84503D9A8EB0500461E04E0A5EBAE
:108A00000800401CA1680E1AA068401BB04201D9A2
:108A1000304601E0A068401B0646BE4201D2304607
:108A200000E0384606466168481932464946FEF776
:108A3000E8FCB244B144BF1B3544A068A84200D151
:108A40000025E560002FD2D15046BDE8F0872DE922
:108A5000F047044689461546E668A068871BAF4282
:108A600008D9616888192A464946FEF7CAFC701978
:108A7000E06010E0B8466168881942464946FEF752
:108A8000C0FCA5EB070809EB070142466068FEF74A
:108A9000B8FCC4F80C80BDE8F08702E008C8121FDB
:108AA00008C1002AFAD170477047002001E001C1D7
:108AB000121F002AFBD170470146202908DA012045
:108AC00088400A4A104008B1012070470020FCE7A6
:108AD000402909DAA1F12000012202FA00F008B1D0
:108AE0000120F2E70020F0E70120EEE7FC06FFBDE1
:108AF00000BFEFF31081084672B6704702460021AE
:108B000004E0505C08B101207047491C0629F8D3E5
:108B10000020F9E7FEB5FF205849C870142088707E
:108B20000F20487029200870C00788600320087350
:108B300000BF00231A46524804F08AFF0546002D64
:108B400019D050A05B495C4A891AC9080322CDE9B3
:108B5000000542EA0140842358A25FA105F080FD90
:108B600005F0B8FB00BF00BF24B100BF204600F0F5
:108B7000E9FA00BF00BF00BF002103200BF0CCF9D1
:108B800000211D200BF0C8F9032005F04CFA1D2030
:108B900005F049FA5848594908600020486056498C
:108BA000564800F067F94021544800F065F9064640
:108BB0004049414A891AC908032242EA0140324623
:108BC0004FA105F01DFD002211464C4800F07AF936
:108BD0000020029002AB41224F4950A00AF04CF90C
:108BE000BDF80800002837DD3249334A891AC90820
:108BF000032242EA01404BA105F0F8FC82224F49D2
:108C00004548FEF729FC50B12A492B4A891AC90860
:108C1000032242EA01404AA105F0E8FC09E02549A7
:108C2000254A891AC908032242EA01404DA105F0EC
:108C3000DDFC00240BE0384800EB44004278364865
:108C400010F814102D4800F04DF9601C84B2BDF8E6
:108C500008008442EFDB0FE000240BE0374800EB14
:108C600044004278354810F81410244800F03AF9CE
:108C7000601C84B2412CF1D3FEBD00005C2C0020AE
:108C8000643F03006E72665F6472765F7370695F43
:108C9000696E697428267370692C20267370695F69
:108CA000636F6E6669672C204E554C4C2C204E55D8
:108CB0004C4C2900644F0300CC4E03007372635C7C
:108CC000616473313239335F73696D706C655F74E1
:108CD00065737465722E630025733A2564205A45C6
:108CE00052524F525F434845434B28257329206613
:108CF00061696C3A256400009D8E0200B82B00204B
:108D0000616473313239335F302072657669643A59
:108D10002025640A0000000098300020302E636691
:108D2000670000006C6F616420302E636667206608
:108D3000726F6D2066617466730A0000C02B00209C
:108D4000302E6366672069732064696666657265A4
:108D50006E742066726F6D2064656661756C740A4E
:108D600000000000302E6366672069732073616D18
:108D7000652061732064656661756C740A0000008B
:108D8000FEB505460C4600263726002000900190CF
:108D9000029009236A463146284600F043F89DF8C0
:108DA000000000049DF8011000EB01209DF8021066
:108DB000084420609DF8030000049DF8041000EBB7
:108DC00001209DF80510084460609DF8060000042D
:108DD0009DF8071000EB01209DF808100844A060E2
:108DE000FEBD70B505460C46002020706070A07076
:108DF000E07020716071A071072322461821284677
:108E000000F010F870BD000070B504460D4604482F
:108E10000068401C0249086009F0D8FF70BD0000DE
:108E2000542C00202DE9F04105460E4617461C46FD
:108E3000FF2C01DDFF2000E02046044646F08008BC
:108E40000A4880F800802146401CFEF7F3FA601CB7
:108E5000C2B2074905482B68984722460449491C75
:108E60003846FEF7CEFABDE8F0810000742E0020EF
:108E7000742F0020016070477CB504460D4645F014
:108E800080008DF8040000208DF80500022269465C
:108E900001A8236898479DF801007CBDF8B50446F9
:108EA0000D461646032005F02FF82B463246214684
:108EB0000348009604F010FE032005F0B4F8F8BD56
:108EC000643F0300F8B504460D46164605F07F00E2
:108ED0008DF800008DF801600222002168462368A9
:108EE0009847F8BDFEB506460C4615460020029090
:108EF0000295182C02DB1E2C00DCFEBD302C02DBA0
:108F00003F2C00DCF9E7402C00D1F6E7502C00D1D3
:108F1000F3E702AB2A462146304600F02FF89DF8D1
:108F20000800A8420FD09DF80800CDE9005007497D
:108F3000074BC91AC908012343EA0140234605A18A
:108F4000726805F08DFB00BFD7E70000644F030097
:108F5000CC4E03006164735F256420777269746589
:108F6000202578206661696C65642C773A25782025
:108F70007265616462616B3A25780A002DE9F041FF
:108F800005460E4617461C463A4631462846FFF728
:108F900099FF31462846FFF76FFF2070BDE8F0814A
:108FA00070B50446002501252A4600212046FFF71A
:108FB00089FF70BD70B504460D4604F22740FFF7E7
:108FC0009DFD0646012D06D0022D0DD0032D11D09A
:108FD000042D19D113E0A07928B194F8240010B918
:108FE0000EB1012070BD00BFE07910B10EB10220BA
:108FF000F8E700BF207A08B10320F3E700BF607AEA
:1090000008B10420EEE700BF0020EBE70146481C52
:10901000052290FBF2F302FB1300C0B27047014639
:1090200091F82420012A01D1EE2000E01F20704792
:1090300010B501220221002001F0E8FB044600BF28
:109040001CB1072C01D0204610BD00BF0722022111
:10905000012001F0DBFB044600BF1CB1072C01D04E
:109060002046F1E700BF0A220021084601F0CEFBAE
:10907000044600BF1CB1072C01D02046E4E700BF26
:109080000020E1E710B572B600BF05F09DFB00BF00
:1090900000BF05F01FF90028FBD100BF00BF1E492B
:1090A0001E4A891AC908012242EA01401CA105F0A2
:1090B0009DFA00BF1D48006800F0010000B100BE2D
:1090C00000BF1549154A891AC908022242EA01401F
:1090D00017A105F08BFA00BF00BF00BF00BF00BFA3
:1090E000BFF34F8F00BF00BF00BF1048E4380068D7
:1090F00000F4E06012490843001D0C49E43908609F
:1091000000BF00BF00BFBFF34F8F00BF00BF00BF55
:1091100000BF00BFFDE70000644F0300CC4E03001A
:10912000466174616C206572726F7200F0ED00E050
:1091300053797374656D2072657365740000000067
:109140000000FA053EB50446002000900190029010
:1091500002946A46002144F20100FFF793FF3EBDEE
:1091600070B505460E462C46207820B961792079E5
:1091700007F0DAFB1CE02078012807D10D480068D1
:10918000401C0C490860FEF78DFE11E0207809288C
:1091900002D107F0B9FB0BE02078032808D106487C
:1091A000007828B1042204F10801606807F02AFB66
:1091B00070BD0000EC2C0020812C00202DE9F8432C
:1091C00007460C46904626480088844244DC4FF609
:1091D000FF7500200090684600F01EFB00BF21488C
:1091E00090F800902048007804F050F8484501D1EC
:1091F000012000E0002030B91B480578007804F019
:1092000045F8194908709DF8000000F00BFB4FF677
:10921000FF7085421ED01548006840F835808FB138
:10922000002C0FDD124909680D4A128805FB021057
:1092300022463946FEF7E5F80C48006800EBC50009
:10924000848005E000200949096801EBC501888098
:10925000002600E0042600E009263046BDE8F88339
:10926000962D0020942D0020952D00208C2D00207F
:10927000902D00202DE9F0411AE016480478164898
:1092800000681649098804FB01051548006800EBD1
:10929000C40086881248006850F834703146284669
:1092A000B8470C48007803F0F1FF0A49087000BF86
:1092B00000BF002058B900BF06490878094909785D
:1092C000814201D1012100E000210029D5D0BDE873
:1092D000F0810000942D0020902D0020962D00207C
:1092E0008C2D0020952D002030B50346481C4FF6EC
:1092F000FF7505EAC004104600F003050DB901250D
:1093000000E000250DB9072030BD084802601019A3
:10931000074D28600020074D2870074D287007482A
:109320000380074801800020EEE700008C2D00201C
:10933000902D0020952D0020942D0020962D0020AA
:10934000982D00202DE9F04707460E4614461F4889
:1093500090F8220010B90820BDE8F0871B4890F86B
:109360002200032801D01120F6E70CB90720F3E70B
:109370000421164880F82210807AC0F3C00018B982
:1093800071021248016101E0104806610F48C76090
:109390008482C48200218183012C01DD522000E0FF
:1093A00051208146094801220169484607F070FEB4
:1093B000054600BFA846B8F1000F04D000BF4046E4
:1093C000FFF7C0FE00BF00BF0020C5E7AC5A002079
:1093D0002DE9F04107460E4615462D4890F822002B
:1093E00010B90820BDE8F081294890F82200032830
:1093F00001D01120F6E70DB90720F3E70521244835
:1094000080F82210807AC0F3C00018B97102204899
:10941000016101E01E4806611D48C7608582C58262
:1094200000218183012D12D101220169582007F00A
:109430002FFE044600BFA046B8F1000F04D000BFC5
:109440004046FFF77FFE00BF00BF0020CAE710487C
:10945000807A00F00700012807D10D480122016938
:10946000592007F015FE044605E001222946D720C1
:1094700007F00EFE044600BFA046B8F1000F04D06E
:1094800000BF4046FFF75EFE00BF00BF0020A9E717
:10949000AC5A0020064890F82200032805D0044862
:1094A00090F8220008B1012070470020FCE700007E
:1094B000AC5A0020044890F82200032802DB02483E
:1094C000001D70470020FCE7AC5A0020F0B587B0C3
:1094D00004460E463A4890F8220010B1082007B022
:1094E000F0BD5EB1E078FF2808D06078FF2805D095
:1094F0002078FF2802D0A078FF2801D10720EEE7CE
:10950000E0782F4981F85800084690F858700020FC
:1095100000900346012211460190384604F05DFC9C
:1095200000BF00BF264991F8580004F096FD00BF27
:10953000244B0FCB03AD0FC5A0788DF80C0020781D
:109540008DF80D0060788DF80E0000231E4A03A9E7
:109550001E4804F07DFA054600BF2F4627B100BF24
:109560003846FFF7EFFD00BF00BF15480660012138
:1095700080F82210807A20F0070111488172807AE9
:1095800020F008010E488172002180F82310FF208E
:109590000B4981F828000A2001F138030122283103
:1095A00000900A4804F0B1FA054600BF2F4627B1E3
:1095B00000BF3846FFF7C6FD00BF00BF00208EE7A2
:1095C000AC5A002048420300B9250300384203008A
:1095D0007CB5144890F8220008B908207CBD1148D9
:1095E00090F82200032801D01120F7E70E4C201D2F
:1095F00006F0B2F900BF0B4890F858400025002053
:1096000000902B46024601460190204604F0E5FBFF
:1096100000BF0021034880F8231080F822100020AA
:10962000DCE70000AC5A00203842030010B50446C5
:10963000022C0AD10C490D4A891AC908032242EAB0
:1096400001400BA104F0D2FF01E0012010BD00BFDA
:109650000549064A891AC908032242EA014010A1B5
:1096600004F0C4FF0120F1E7644F0300CC4E030077
:10967000506F776572206D616E6167656D656E74A0
:109680002077616E747320746F2072657365742027
:10969000746F20444655206D6F64652E00000000F5
:1096A000506F776572206D616E6167656D656E7470
:1096B00020616C6C6F77656420746F2072657365D0
:1096C0007420746F20444655206D6F64652E000031
:1096D00010B5024802F0D8F910BD0000A02D0020FE
:1096E00030B503460C460AB9072030BD19684FF063
:1096F000FF358D60CD604A61012C01D1012000E071
:10970000002008610020F0E738B513480068009099
:109710000823A82211491248006803F047FE0446B6
:109720000CB1204638BD0F4A69460F4802F0B2F925
:1097300004460CB12046F5E701210B4802F050FA2F
:1097400001230A4A1946084802F070F90120084925
:1097500008702046E6E7000058400300DC5900206E
:1097600048400300F90C0300A02D0020FFFF7F00FC
:10977000AC2D00202DE9F84306460D4690463446B0
:1097800000200090684600F047F84FF0FF33D4E91E
:10979000021059405840014308D103F009F940191B
:1097A00041F10001C4E90201012700E000279DF812
:1097B000000000F037F817B90020BDE8F883C4F8BE
:1097C0001880206900B125612146002009F0DCFAEB
:1097D000F3E7F8B50446254600200090684600F0FF
:1097E0001BF84FF0FF33D5E90210594058400143B0
:1097F00001D1002604E04FF0FF31A960E9600126A5
:109800009DF8000000F00EF80EB90020F8BD2946C2
:10981000012009F0B9FAF9E710B50446204607F02F
:1098200087FB10BD70B5044625460E488068B0B170
:10983000ADB9FFF75DF906460A4800680A490860B5
:10984000084840684FF0E021C1F8040100200549B4
:1098500088601EB900BF62B600BF00BF00BF00BF76
:1098600070BD0000945A002000E100E0F8B5054604
:109870000C4617462088001DB84201D90C20F8BDBF
:10988000684679DF064600BF304600B1F7E700BF03
:109890000320218868542088401C208019202188BA
:1098A00068542088401C208020884119BDF80000A1
:1098B00009F0CBFD2188084420800020DFE700006C
:1098C000002113E00C480269012308E000BFD068C2
:1098D0000079884201D1002303E0D0680268002AA1
:1098E000F4D100BF0BB108467047491C0A29E9DBD7
:1098F0004FF0FF30F8E70000287800202DE9FC4108
:10990000054688461646002437880020308095F8A2
:109910002D0058B13A463146404600F095FA0446CB
:1099200000BF204608B1BDE8FC8100BFA87850B157
:109930003A4631464046FFF799FF044600BF2046AD
:1099400000B1F0E700BFE87860B1E97848B23B4683
:109950003246414602F06CFE044600BF204600B18C
:10996000E1E700BF686868B1696891F900003B46AB
:109970003246414609F048FD044600BF204600B18A
:10998000D1E700BF288900280EDD434606220221C8
:1099900005F10800CDE9006709F003FE044600BFA9
:1099A000204600B1BFE700BF288A00280EDD4346ED
:1099B0000722032105F11000CDE9006709F0F1FD50
:1099C000044600BF204600B1ADE700BF288B002849
:1099D0000EDD43461522142105F11800CDE900677C
:1099E00009F0DFFD044600BF204600B19BE700BF41
:1099F000286A58B13B4632464146286A01F017FAB8
:109A0000044600BF204600B18DE700BF686A58B128
:109A10003B4632464146686A03F0D6FA044600BF28
:109A2000204600B17FE700BF95F82C0000280BDD31
:109A30003B4632464146284608F0E8FA044600BF55
:109A4000204600B16FE700BF287858B13B46324648
:109A50004146284603F0B6FB044600BF204600B14D
:109A600061E700BF20465EE7F8B504460E4615469E
:109A7000002000902B466A463146204600F008F848
:109A800007460FB90020F8BDBDF800002044FAE7F2
:109A9000F0B504460D461E4604B10AB90020F0BDDB
:109AA000002103E0605C401C084481B2481CA842CD
:109AB00006DA10888842F5DC481C205CB042F1D1FF
:109AC000A94201DB0020EAE7881C87B2605C10B184
:109AD000605C401E00E0002083B213B1F818A84279
:109AE00001DD0020DBE717801846D8E780F830104A
:109AF000704770B504460D4605B10CB90E2070BD17
:109B000005F1780001F03CF908B90720F7E70020DB
:109B1000A0702C2205F17801201DFDF772FC0020B9
:109B200084F83000D5F8A4006063D5F8A800A063DD
:109B30004FF6FF70A4F8240404F58260C4F82004F2
:109B4000002140F22C40C4F82614A4F82A14015530
:109B5000207810B9FF2084F8540004F15500C4F8AF
:109B600010042046FFF75BFA40F21441085304F258
:109B7000144204F155012846FFF7C0FE064600BF17
:109B8000304600B1BBE700BF04F231204FF48361DF
:109B900008512046FFF743FAA4F81C044FF48360F1
:109BA000015904F21C4205F13C00FFF7A7FE0646EE
:109BB00000BF304600B1A2E700BF0121512001558E
:109BC000208B81B248200153012084F83C00002101
:109BD0002164502001556169616404F13C02002157
:109BE00004F1540072DF064600BF304600B186E73C
:109BF00000BF01202070304681E770B504460D4655
:109C00002E462088102804D0112807D026280FD1EE
:109C100009E02146304606F09FF80AE0214630462A
:109C200006F096FA05E02146304606F019FC00E001
:109C300000BF00BF70BD70B504460E46207808B95D
:109C4000082070BDA670002140F22C40C4F82614F4
:109C5000A4F82A140155A07910B1A078012809D0E0
:109C6000E07910B1A078012804D0E07970B1A07833
:109C700002280BD1606B30B1012084F82D0408203C
:109C8000616B884702E0002084F82D0431462046AD
:109C9000FFF790F9A070606BA0B1A078032802D004
:109CA000A07804280ED1607960B194F82E0448B9E8
:109CB000002084F83004012084F82F040720616B11
:109CC000884702E0002084F82F04182104F13C00AA
:109CD000FDF7B0FB012084F83C0004F12C0006F0F5
:109CE0004EFC20B194F82C105120015502E00121C6
:109CF0005120015594F8240060B104F1280006F0C9
:109D00003EFC20B194F828105220015502E00121B8
:109D100052200155002150200155A078052824D259
:109D2000DFE800F01F030A11180004F13C0120468F
:109D300008F0CFF9054619E004F13C01204608F08F
:109D4000B0F9054612E004F13C01204608F0D3F9D1
:109D500005460BE004F13C01204608F0FAF90546FF
:109D600004E0002084F8310000E000BF00BFA078CC
:109D700098B104F13C0204F15400D4F8201472DFCD
:109D800005460DB128465CE794F8301094F854006D
:109D900073DF05460DB1284653E7606B18B194F8A0
:109DA0003100616B884700204BE700002DE9F0414E
:109DB000044600BF14B90E20BDE8F08100BF1C228C
:109DC00021461C48FDF71DFB1B481A490860206806
:109DD00060B120687ADF05460DB12846ECE71648E9
:109DE00021680A6802604968416005E012487BDF2B
:109DF00005460DB12846DFE7002617E006EB860092
:109E00000E4901EB800700BF4FF6FF70388000BF9E
:109E10000B4800EB461078600A4A0021381DFFF716
:109E20005FFC05460DB10320C6E7761C002EE5D089
:109E30000020C1E7DC5700205C2D0020C85700201F
:109E4000A8570020113503002DE9FC4105460C46BA
:109E5000174620880930B84202D90C20BDE8FC81A1
:109E600068466DDF064600BF304600B1F6E700BF2A
:109E70000820218868542088401C20801B202188CD
:109E800068542088401C208020882844DDF8011078
:109E90000160BDF8051081802088801D20809DF81C
:109EA0000000400818B900202188685402E0012011
:109EB000218868542088401C20800020CEE70000C4
:109EC00070B503F0B9FC044600BF204600B170BD78
:109ED00000BF00BF084D28464FF0030C00DF00BF55
:109EE000044600BF204600B1F1E700BF03F01EFDAD
:109EF00004462046EBE70000347F002010B51349EC
:109F0000134A891AC908042242EA014011A104F047
:109F10006DFB4FF0FF3100203DDF044600BF2046BF
:109F200000B110BD00BFB12100203CDF044600BFDE
:109F3000204600B1F5E700BF13484169012088477A
:109F4000022004F097FD0020EBE70000644F0300BF
:109F5000CC4E0300496E20626C655F6466755F627B
:109F60007574746F6E6C6573735F626F6F746C6F12
:109F7000616465725F73746172745F66696E616C4F
:109F8000697A650D0A000000187F002010B50548A9
:109F90000068416900208847FFF7B0FF044620466B
:109FA00010BD00006C2E002070B504460D4600BFA9
:109FB00004B970BD00BF2088102806D0112808D031
:109FC00051280AD0532810D10BE0204605F0BEFEE0
:109FD0000CE0204606F0AEF808E0204606F01EFA37
:109FE00004E0204606F0F6F900E000BF00BF00BF25
:109FF000DFE7000070B504460426207B012802D06C
:10A00000022822D109E001F089FE05460DB901269A
:10A0100002E0112D00D1062619E0607B142801DC36
:10A02000607B08B905260FE0627B04F10E0112483F
:10A03000FDF7E7F9607B1049091F8861084608F0C1
:10A04000B7F8054605B9012601E0022600BF00BFAA
:10A05000012E0FD0207B314600F058F8054625B17F
:10A060000648006841690320884704480068416940
:10A070000220884770BD0000447F00206C2E002025
:10A0800070B505460E4600BF1E48006820B11D4849
:10A09000406808B1012000E0002000B970BD00BF99
:10A0A000184800F10801426828469047044600BF5E
:10A0B000082C24D07CB90020134909684876012176
:10A0C000022000F023F80446CCB10F480068416933
:10A0D0000320884713E000200B49096848760621D1
:10A0E000022000F013F8044624B1074800684169D3
:10A0F000032088470448006841690220884700BF60
:10A10000CCE70000347F00206C2E0020F0B587B033
:10A1100004460D460327002001900290039004900E
:10A120000320069020208DF814008DF815408DF83E
:10A1300016500E48C088ADF8040002208DF80600C5
:10A140000020ADF8080006A8039005A80490074970
:10A15000888801A9AEDF064626B9BDF81800032895
:10A1600000D00C26304607B0F0BD0000187F00205C
:10A1700070B505460E462888102802D011282CD12B
:10A1800015E01748006860B900F0B8FE044600BF4B
:10A1900034B11448006818B120461249096888474C
:10A1A00000BF0F480068401C0D49086016E00C48CD
:10A1B0000068401E0A4908600846006860B9FEF75A
:10A1C00037FF044600BF34B10648006818B1204686
:10A1D00004490968884700BF00E000BF00BF70BDA8
:10A1E000582D0020542D002070B504460D462088BF
:10A1F000102806D0112808D012280ED0502810D1CF
:10A2000007E0204605F06AFD0CE0204605F078FFE7
:10A2100008E0204606F044F904E0204605F046FD3B
:10A2200000E000BF00BF70BD2DE9F04104460F46BD
:10A23000A6882088102806D0112817D019283DD0CC
:10A240001A2848D116E006F0D1FC304606F0AAFCE8
:10A2500020B900BF0420FEF775FF06E0E07B02286E
:10A2600003D131461D4803F00BF934E0304606F0C7
:10A27000E1FC30E0207A0509042D01DB012000E03B
:10A2800000200246314615480C3002F0C2F9032D79
:10A2900001DB012000E00020024631460F48083073
:10A2A00002F0B7F9022D01DB012000E00020024698
:10A2B00031460A48001D02F0ACF90CE0207A48B99A
:10A2C000607AC0F3C0052A46314604480C3002F0DB
:10A2D000A0F900BF00BF00BFBDE8F0810458002016
:10A2E0002DE9BE4105460F46288821282BD006DCE3
:10A2F00010280BD0112817D013287DD154E03B280B
:10A300007BD052287BD05628F7D1C5E0A888774962
:10A3100008800120764908707648006818B1084620
:10A32000744909688847DDE04FF6FF706F4908807F
:10A3300002206F4908706F48006818B108466D49DF
:10A3400009688847CEE06C496C4A891AC90804221A
:10A3500042EA01406AA104F049F900200290A8886D
:10A3600002A98FDF044600BFA046B8F1000F19D044
:10A3700068A06149614A891AC9080322CDE9000829
:10A3800042EA0140462366A26DA104F069F903F098
:10A39000A1FF00BF00BF26B100BF3046FEF7D2FECE
:10A3A00000BF00BF00BF9DE000231A4685214F4833
:10A3B00000887FDF044600BFA046B8F1000F19D027
:10A3C00054A04D494D4A891AC9080322CDE9000815
:10A3D00042EA01404C2352A259A104F041F903F092
:10A3E00079FF00BF00BF26B100BF3046FEF7AAFECE
:10A3F00000BF00BF00BF75E073E028E0FFE7002367
:10A400001A46194639480088B1DF044600BFA04605
:10A41000B8F1000F19D03FA03749384A891AC90846
:10A420000322CDE9000842EA014052233CA244A1A4
:10A4300004F016F903F04EFF00BF00BF26B100BFC5
:10A440003046FEF77FFE00BF00BF00BF4AE0A8888D
:10A45000132176DF044600BFA046B8F1000F19D0E3
:10A460002CA02549254A891AC9080322CDE90008EC
:10A4700042EA014058232AA231A104F0F1F803F086
:10A4800029FF00BF00BF26B100BF3046FEF75AFECD
:10A4900000BF00BF00BF25E0A888132176DF044677
:10A4A00000BFA046B8F1000F19D01AA01249134AF4
:10A4B000891AC9080322CDE9000842EA01405E2357
:10A4C00017A21FA104F0CCF803F004FF00BF00BFE7
:10A4D00026B100BF3046FEF735FE00BF00BF00BF0B
:10A4E00000E000BF00BFBDE8BE8100004C2E002090
:10A4F000542E0020502E0020644F0300CC4E030049
:10A500005048592075706461746520726571756575
:10A5100073742E006572725F636F646500000000E3
:10A520002E2E5C6C69627A6E6F726469635C737202
:10A53000635C7A626C655F6D6F64756C652E630039
:10A5400025733A2564205A4552524F525F4348457D
:10A55000434B28257329206661696C3A2564000005
:10A5600070B50446204608F06AFF0546C5F3400072
:10A5700070BD70B50446204608F061FF054605F041
:10A58000010070BD30B50246087A0B7833B1012B5B
:10A5900005D0022B05D0032B14D101E000BF00BF72
:10A5A00000BF4B7800EB4004084D2D6805EB840498
:10A5B0002372002300EB4004044D2D6805EB840456
:10A5C000A37200E000BF00BF30BD00005C2E002081
:10A5D00001460A46906970472DE9FE4380460C46C5
:10A5E00091464546AE692869B0F5007F02D0062045
:10A5F000BDE8FE831648006808B11120F8E7C6F8E8
:10A600001890B460124805600027124905F1140043
:10A61000FEF75CFF07464FB944B907F037FC0E4818
:10A62000007808B9002000E00D20074677B100202F
:10A630000749086054B1094A07CA8DE80700B069A4
:10A64000029069464046B268904700BF3846CFE75F
:10A65000E02D002089110300DC2D002008420300BA
:10A6600030B503461D4611B101290ED105E014464F
:10A670000CB100202070002030BD0AB90720FBE794
:10A680001446281D20600020F6E700BF00BF06200A
:10A69000F2E700002DE9FE4307460D46B846D8F81C
:10A6A000184000261B480068404502D01120BDE834
:10A6B000FE83FEF7EFFE08B11120F8E795E80700EA
:10A6C000C4E90412E060AB889AB22968A868FEF772
:10A6D00039FE064656B9A06840B907F0D7FB0E48C8
:10A6E000007808B9002000E00D200646A06870B18F
:10A6F0006EB10A4A07CA8DE8070004F10C00019008
:10A70000A069029069463846A268904700BF30466B
:10A71000CDE70000E02D0020DC2D002020420300CA
:10A72000FEB506463746BD6913480068B84201D0F9
:10A730001120FEBDFEF7AEFE08B11120F9E7FEF7CD
:10A7400047FF044614B900200B490860A86880B18F
:10A750000A4A07CA8DE807000CB1012000E000207A
:10A760008DF80100A869029069463046AA689047B2
:10A7700000BF2046DDE70000E02D0020144203006A
:10A780002DE9FE4307460D46B846D8F81840002686
:10A790001B480068404502D01120BDE8FE83FEF74B
:10A7A00079FE08B11120F8E795E80700C4E9041222
:10A7B000E060AB889AB22968A868FEF709FE0646F1
:10A7C00056B9A06840B907F061FB0E48007808B997
:10A7D000002000E00D200646A06870B16EB10A4A64
:10A7E00007CA8DE8070004F10C000190A0690290EF
:10A7F00069463846A268904700BF3046CDE7000062
:10A80000E02D0020DC2D00202C42030030B5034653
:10A810000020042B23D2012A07D1012903D103F1FF
:10A820000E04E4B200E00024224679B1012902D0EE
:10A83000022911D104E003EB43040A4D2A550DE02F
:10A8400003EB4304074D2C44627007E003EB430421
:10A85000044D2C44A27001E0072000BF00E0072057
:10A8600030BD0000985700202DE9FC4704460D46F6
:10A870001646A71C4FF001080020019001A8FEF722
:10A88000CBFF3048406828602E4840682D498968D1
:10A89000411A2D480068401CA0EB010915E0012178
:10A8A0002A4802F00AFE02F0C7FA824651462748BB
:10A8B00002F003FE2348406822498968411A224871
:10A8C0000068401CA0EB010900BF4F45E7D8B8F174
:10A8D000000F30D00021009176B1009921F00301E2
:10A8E000491C0091009921F00401091D0091009973
:10A8F00064F3891100910DE0009921F00301891C96
:10A900000091009921F00401091D0091009964F360
:10A910009F5100910B4949680B4A12681140094A3E
:10A920000C3202EB81000099016006494968394404
:10A930000C3A516000BF9DF80400FEF773FF4046DB
:10A94000BDE8FC8728680020F82D0020447800200E
:10A9500070B504460D460A2D03D10D212046FFF7A0
:10A96000F7FFA168481CA06020684554D4E9011095
:10A97000884202D3204603F0F6F870BD0448806890
:10A9800003494968884201D1012070470020FCE753
:10A990002868002070B504460D46032C06D1A92076
:10A9A0000349086000BF002004F064F870BD000097
:10A9B0002005004010B504490448FEF712FA044986
:10A9C000014807F0A5FA10BD422C0020B82B00204A
:10A9D000492C00204FF0FF31054A42F8201008288A
:10A9E00004DBFF23A0F108015A32535470470000E2
:10A9F000885800200146024850F8210070470000A6
:10AA0000885800202DE9F04F03460C464FF0FF39DF
:10AA10000AB1002000E0082084460AB1082000E0C6
:10AA20000C208046614624E0154850F82100401C67
:10AA3000F0B91D460846274616464FFA80FBDFF858
:10AA400040A00AF1300A0AF805B0DFF834A04AF84D
:10AA500020704EB94FFA85FBA0F1080ADFF820E01C
:10AA60000EF15A0E0EF80AB000BF4FFA81F902E05B
:10AA7000491C4145D8D300BF4846BDE8F08F0000CF
:10AA8000885800200146014840567047B8580020B9
:10AA900070B590B006460C461546A07818B901204E
:10AAA0008DF80E0002E0A0788DF80E002088ADF839
:10AAB0000C0000200290607C02A907F0A9FBA07C9A
:10AAC0000DF1090107F0A4FBE07B08B1012000E0D3
:10AAD00000209DF80A1060F3C3018DF80A10207C55
:10AAE00008B1012000E000209DF80A1060F3041175
:10AAF0008DF80A10207B08B1012000E000209DF8AD
:10AB00000A1060F300018DF80A10207D08B10220C0
:10AB100000E001209DF80A1060F342018DF80A1050
:10AB20001C2109A8FCF786FC607BC0F3001018B953
:10AB3000607BC0F34010F8B100200090E07C0DF184
:10AB4000010107F065FB00BF9DF8000020F00F0039
:10AB5000401C8DF800009DF8000020F0F00010303F
:10AB60008DF8000000BF9DF8020020F00600801C58
:10AB70008DF80200CDF838D0607B8DF82400A07BE2
:10AB80008DF82500142104A8FCF754FC03A80490B8
:10AB900002A80590A088ADF81C00A06820B1E0884C
:10ABA000ADF81800A0680890A069002849D00020DE
:10ABB0000190A0690088ADF82C00A0694088ADF82C
:10ABC0002E00A06940680A9001A80D90A169087B39
:10ABD00001A907F01DFBA169487B0DF1050107F0F4
:10ABE00017FBA069807A08B1012000E000209DF8E1
:10ABF000061060F3C3018DF80610A069C07A08B191
:10AC0000012000E000209DF8061060F304118DF88B
:10AC10000610A069007A08B1012000E000209DF82C
:10AC2000061060F300018DF80610A069807B08B162
:10AC3000022000E001209DF8061060F342018DF82B
:10AC40000610E06908B1E0690C902B4604AA09A936
:10AC50003046AADF10B070BD70B504460D46002026
:10AC6000E070401EE0622946204602F091FA08B1E9
:10AC7000042070BD04F22E2002F0BFF84AF65521E0
:10AC8000884201D00320F4E794F83000E92807D087
:10AC900094F83000EB2817D13220005D902813D1B2
:10ACA00004F1660002F09DF820F07F4007498842D9
:10ACB00001D10020DDE704F1820002F092F804499E
:10ACC000884201D10020D4E70220D2E74641540057
:10ACD00046415433024600E0521C107810B11078FF
:10ACE0008842F9D11078704770B505460DB9094C06
:10ACF00001E0084C083409E0204602F046F8064618
:10AD000006B904E028467168884700BFF4E700BF31
:10AD100070BD00007C58002010B504462CB90120FD
:10AD2000064948700020FFF7DFFF012C04D1012005
:10AD300002498870FFF7D8FF10BD0000745800204A
:10AD40000246891E5069801E884201D80020704743
:10AD50005389906A01FB0300F9E72DE9F0470246A9
:10AD600013468C46D3E90245DCE90267B6EB0408DA
:10AD700077EB050002D30120BDE8F0870020FBE758
:10AD800001468878012805D191F82000012801D1D9
:10AD9000002070470120FCE733B58BB0054600204A
:10ADA00000900C9878B100240BE021460CA802F02A
:10ADB00058FB28B1009A501C009001A820F81240BE
:10ADC000641C142CF1D32C2269462846FCF719FB8D
:10ADD0000DB030BD01460888062808DB0888B0F5AC
:10ADE000486F06DD08884FF6FF72904201D00720B9
:10ADF00070474888062808DB4888B0F5486F06DDAC
:10AE000048884FF6FF72904201D00720F0E708888B
:10AE10004FF6FF72904208D04888904205D00888CB
:10AE20004A88904201DD0720E2E70020E0E72DE9B3
:10AE3000F04107460D46144698462088801D40453F
:10AE400002D90C20BDE8F0813846FFF7C3FF064663
:10AE500000BF304600B1F5E700BF052021886854E7
:10AE60002088401C20801220218868542088401CA3
:10AE7000208022885119388808F0E7FA2188084490
:10AE8000208022885119788808F0DFFA2188084448
:10AE900020800020D6E710B5044600BF2046FEF70C
:10AEA00051F900BF10BD0000F8B505460C46607AA8
:10AEB00088B9207A10B91048476801E00E488768C1
:10AEC0002A4639466068FEF755FC064616B13046FC
:10AED00007F03CF80EE0002020720748406948B1B6
:10AEE00001208DF80000ADF8025003484169684622
:10AEF000884700BFF8BD0000DC57002010B50122D4
:10AF000000210846FFF782FC044600BF1CB1072C55
:10AF100001D0204610BD00BF072202210120FFF70B
:10AF200075FC044600BF1CB1072C01D02046F1E798
:10AF300000BF042202210020FFF768FC044600BF86
:10AF40001CB1072C01D02046E4E700BF0020E1E758
:10AF50002DE9F04782468946DAF80040B9F1000F42
:10AF600006D1E76817B16069B84215D8012713E028
:10AF70004946504601F020FC0646022E02D201202E
:10AF8000BDE8F087701C08B93046F9E76069B04247
:10AF900001D93046F4E74F463D4600BF6D1C60695D
:10AFA000A84204D80225BD4201D90020E8E729467D
:10AFB000504601F001FC064606B909E0012E01D019
:10AFC000701C08B93046DBE7BD42E7D10020D7E767
:10AFD00000BF00BF4FF0FF322946204605F0BAFC03
:10AFE0008046B8F1000F08D1B9F1000F05D02A460C
:10AFF0004946204605F0AEFC8046B8F1000F0DD161
:10B00000E560D4E90410801E814202D22069401E0E
:10B010002061207940F00100207107E0B8F1010FB4
:10B0200002D14FF0FF3000E0012005462846A7E797
:10B030002DE9F35F8A46DAF80090009800F12005C8
:10B040000B222021284602F019F8002080460746EE
:10B050004FF0080B00BF38467F1C19F80040202C29
:10B0600000DC55E02F2C01D05C2C0AD100E07F1CC5
:10B0700019F807002F28FAD019F807005C28F6D035
:10B0800046E02E2C01D0D8450CD3BBF10B0F01D0DC
:10B090002E2C02D00620BDE8FC9F4FF008084FF090
:10B0A0000B0BD8E7812C01DB9F2C03DDE02C1CDB94
:10B0B000FC2C1ADC38467F1C19F80060402E01DB9E
:10B0C0007E2E03DD802E05DBFC2E03DCABF10100C0
:10B0D000404501D80620DEE7404608F101082C541F
:10B0E000404608F101082E5411E0214614A0FFF754
:10B0F000F1FD08B10620CEE7612C04DB7A2C02DCDE
:10B10000A4F12000C4B2404608F101082C54A2E783
:10B1100000BF09EB0700CAF80000B8F1000F01D129
:10B120000620B8E72878E52801D105202870202CD2
:10B1300001DC042000E00020E8720020ABE7000002
:10B14000222A2B2C3A3B3C3D3E3F5B5D7C7F00003E
:10B150002DE9FF4105460C4629492A4A891AC908A2
:10B16000042242EA01402B46224627A103F054FA6A
:10B17000002002900390ADF80840ADF80A4000901E
:10B1800001906A4602A9284690DF0646002E32D07A
:10B19000304604F003F8074619491A4A891AC908C3
:10B1A000012242EA01403B462A46234903F034FA91
:10B1B000BDF8000010B9BDF8020068B1BDF802305A
:10B1C000BDF800200E490F4FC91BC908012747EAE7
:10B1D00001401AA103F020FABDF8040058B1BDF8EF
:10B1E00004200749074BC91AC908012343EA014053
:10B1F000224903F005FA304604B0BDE8F0810000B2
:10B20000CC4E0300CC4E03005570646174696E67C8
:10B210002064617461206C656E67746820746F20AF
:10B220002575206F6E20636F6E6E656374696F6E37
:10B2300020307825782E0000E04503005468652012
:10B240007265717565737465642054582F52582067
:10B250007061636B6574206C656E677468206973D8
:10B2600020746F6F206C6F6E672062792025752FB8
:10B270002575206F63746574732E00002C460300DF
:10B2800020BF70472DE9F04104460E46D4F80080F7
:10B290000021204600F000F90546EDB9002700BF67
:10B2A0004046A16901F074FF054605B113E0E0696D
:10B2B0000078E52802D0E069007820B9781C0746BC
:10B2C000B04201D107E000270121204600F040F8FC
:10B2D0000546002DE4D000BF042D00D107252846E7
:10B2E000BDE8F0812DE9F0410446276800212046A1
:10B2F00000F0D2F8054615B12846BDE8F08100BF40
:10B300003846A16901F044FF054605B11DE0E0693A
:10B3100006780EB9042518E0E069C07A00F03F0015
:10B32000A071E069C07A00F0080038B90B2204F17E
:10B330002001E06901F083FE00B906E0002120460B
:10B3400000F006F80546002DDAD000BF2846D4E705
:10B350002DE9F047044689462568206900F1200759
:10B36000A06910B1B7F5001F02D30420BDE8F08733
:10B37000C7F30800002868D1A069401CA06160697B
:10B3800038B92889B0EB571F5FD80020A06104208E
:10B39000ECE76889401E00EA5720002855D1204676
:10B3A000616901F009FA0646012E01D80220DDE7A5
:10B3B000701C08B90120D9E76869B0423FD8B9F1DB
:10B3C000000F03D10020A0610420CFE7204661696F
:10B3D000FFF7BEFD06460EB90720C7E7012E01D1D3
:10B3E0000220C3E7701C08B90120BFE7284607F018
:10B3F000DFFB08B10120B9E74FF40072002105F12D
:10B40000300001F03BFE4FF0000831462846FFF7C0
:10B4100097FCE8620CE00120E870284607F0C8FBC2
:10B4200008B10120A2E708F10108E86A401CE862BF
:10B4300068894045EFD8E86AA0EB0800E8626661D9
:10B4400031462846FFF77CFCA0612761C7F308015D
:10B4500005F130000844E061002087E770B504463C
:10B46000266801212046FFF70DFF054695B93046B5
:10B47000A16901F08DFE054665B920220021E06931
:10B4800001F0FCFD0B2204F12001E06901F0E9FD6F
:10B490000120F070284670BD2DE9F04104460D46AC
:10B4A0002668B5F5001F02D205F01F0010B102207A
:10B4B000BDE8F0812561A7681FB93078032800DB5B
:10B4C000776A47B93089B0EB551F01D80220EFE702
:10B4D000706AA0611CE070894FEA402811E039468B
:10B4E000204601F069F90746781C08B90120DFE71A
:10B4F000022F02D37069B84201D80220D8E7A5EB29
:10B5000008054545EBD239463046FFF719FCA061E6
:10B510006761A06908B90220CAE7A06900EB55205D
:10B52000A061C5F3080106F130000844E061002085
:10B53000BEE700002DE9F04104463E480078844211
:10B5400002DB0320BDE8F08104EB44003A490968BE
:10B5500051F8200008B90320F4E704EB4400364911
:10B56000096801EB8000407A00F0010038B904EB73
:10B5700044003149096801EB8000407AE2E704EBBE
:10B5800044002D49096801EB8000406838B92B4818
:10B5900004EB4401284A126802EB81014860012053
:10B5A00004EB4401244A126802EB8101887204EB27
:10B5B00044002149096851F82060214F3068224633
:10B5C0003946036830469847054600BF4DBB07E043
:10B5D00004EB4401184A126802EB81014868804775
:10B5E00004EB44001449096801EB8000807A0028CC
:10B5F000EED104EB44001049096801EB8000007AA9
:10B6000078B904EB44000C49096801EB8000407AEA
:10B6100020F0010004EB4401074A126802EB8101AB
:10B62000487204EB44000449096801EB8000407A49
:10B6300088E70000602E00205C2E002081B202000E
:10B6400085A50200F8B504460E4615462A4800783E
:10B65000844201DB0420F8BD26B1012E1BD0022E4E
:10B6600045D12EE00120009000BF04EB4401234AA5
:10B67000126852F821006A46002102F09EF807463F
:10B6800017B1112F00D003E09DF800000028ECD185
:10B6900000BF0020DFE704EB44001849096851F8B7
:10B6A000200008B90320D6E72F4604EB4401134AD3
:10B6B000126852F8210002F079F800683860002022
:10B6C000C9E704EB44000D49096851F8200008B9A6
:10B6D0000320C0E72F4604EB4401084A126852F8E1
:10B6E000210002F063F8808838800020B3E700BFB3
:10B6F00000BF0120AFE70000602E00205C2E00207C
:10B700002DE9FE4F0446884691461E462F48007894
:10B71000844200DA16B90420BDE8FE8F04EB440031
:10B720002B49096851F8200048B104EB440028492E
:10B73000096801EB8000407A00F0010008B10320A5
:10B74000EAE7CDF800900196CDF80880012004EBDF
:10B7500044011F4A126802EB8101887204EB440025
:10B760001B49096851F820506F46286841692846EE
:10B77000884700683968884201D8072004E02868B3
:10B7800039468268284690478246BAF1000F1BD19D
:10B7900007E004EB44010E4A126802EB810148689D
:10B7A000804704EB44000A49096801EB8000807A75
:10B7B0000028EED104EB44000549096801EB800044
:10B7C000007A08B90020A7E70120A5E7602E002035
:10B7D0005C2E0020014607480078814201DB0120F1
:10B7E000704701EB4100044A126802EB8000407A86
:10B7F000F6E70000602E00205C2E002070B50446A5
:10B8000036480078844201DB032070BD04EB44001D
:10B810003349096851F8200008B90320F5E704EB23
:10B8200044002F49096801EB8000407A00F00100D4
:10B8300038B104EB44002A49096801EB8000407AE2
:10B84000E3E704EB4401264A126852F82100002283
:10B85000114601F0B2FF00BF04EB44002049096823
:10B8600051F820603068416830468847054600BF7F
:10B87000112DF1D08DB907E004EB4401184A12688C
:10B8800002EB81014868804704EB440014490968D1
:10B8900001EB8000807A0028EED104EB44001049CF
:10B8A000096801EB8000007A78B904EB44000C4988
:10B8B000096801EB8000407A40F0010004EB44018C
:10B8C000074A126802EB8101487204EB4400044904
:10B8D000096801EB8000407A97E70000602E0020A5
:10B8E0005C2E00202DE9FE4F0446884691461E46F8
:10B8F00035480078844200DA16B90420BDE8FE8F8E
:10B9000004EB44003149096851F8200048B104EBC8
:10B9100044002E49096801EB8000407A00F00100E4
:10B9200008B10320EAE704EB44002849096801EB69
:10B930008000407A00F0040008B10220DEE7CDF874
:10B9400000900196CDF80880012104EB44001F4AC5
:10B95000126802EB8000817204EB44001B49096805
:10B9600051F820506F46286841692846884700688A
:10B970003968884201D8072004E028683946C2683F
:10B98000284690478246BAF1000F1BD107E004EB2E
:10B9900044010E4A126802EB81014868804704EBBB
:10B9A00044000A49096801EB8000807A0028EED142
:10B9B00004EB44000549096801EB8000007A08B9EE
:10B9C00000209BE7012099E7602E00205C2E0020DC
:10B9D000024A1060024B1970704700005C2E002074
:10B9E000602E002010B50021034801F087FD0446B9
:10B9F00084F3100010BD00004478002070B50546A7
:10BA00000C464FF4803000FA04F1284600F0AAF901
:10BA100070BD70B505460C464FF4A07000EB840075
:10BA200086B23146284600F0B7F970BD2DE9F047DF
:10BA300004460D4616461F464FF4803000FA05F8BE
:10BA40004FF4A07000EB85001FFA80F926F07F46C6
:10BA50004146206803F07DF84146206803F06AF80B
:10BA60004946206803F05CF832462946206803F016
:10BA700047F84146206803F063F81FB1414620684B
:10BA800003F06DF8BDE8F08710B50446206803F0B8
:10BA90003CF810BD2DE9F04704460D461746607985
:10BAA000324941F820706079314901EBC0000079DA
:10BAB00068B108262F49304A891AC908022242EA89
:10BAC00001402EA102F092FD3046BDE8F0872988A2
:10BAD0002068C0F8081500BF94F90420AB78104620
:10BAE0001946002808DB4FEA417C4FEA1C68DFF862
:10BAF000B0C00CF800800BE04FEA417C4FEA1C69B3
:10BB0000DFF8A0C000F00F08A8F104080CF80890B6
:10BB100000BF00BF94F90410084600280DDB00BFE9
:10BB200000BF00F01F0301229A4043099B0003F16C
:10BB3000E023C3F8002100BF00BF00BF00BF012009
:10BB400061790B4A02EBC10108716079114641F835
:10BB5000304000260749084A891AC908032242EAE8
:10BB6000014011A102F042FD3046AEE7C42D002095
:10BB7000C82D00204C4F0300CC4E030052544320EC
:10BB8000696E7374616E636520616C72656164795E
:10BB900020696E697469616C697A65642E000000C1
:10BBA00000E400E018ED00E05254433A20696E6969
:10BBB0007469616C697A65642E00000010B50146F5
:10BBC00091F90400002807DB00F01F0301229A40CE
:10BBD000024B440943F8242000BF10BD00E200E0FE
:10BBE00070B505460C4622460221284600F0C6F8EC
:10BBF00070BD10B504464FF48271204600F0CCF8B9
:10BC000010BD10B504460021206802F0B3FF10BD3E
:10BC100010B504460421206802F0ACFF10BD2DE9E8
:10BC2000F84F04468846154699464FF4803000FA8E
:10BC300008FA4FF4A07000EB88001FFA80FB25F093
:10BC40007F455146204600F08DF8206802F05DFFE8
:10BC500006464146206802F04DFF009032464146BC
:10BC6000206802F04DFF5946206802F059FF314626
:10BC7000009806F0C6FF012806D1102003F00EFB45
:10BC80005946206802F04CFF206802F03EFF06464D
:10BC90003146284606F0B5FF07465146206802F0B7
:10BCA0004FFF012F0FD16A1C4146206802F028FF88
:10BCB000102003F0F3FA206802F027FFB04225D0ED
:10BCC0000D20BDE8F88F2A464146206802F018FF93
:10BCD000206802F01AFF0646681E314606F091FF02
:10BCE00007466FF07F40A0EB0900B84201D20D205B
:10BCF000E7E75FB96A1C4146206802F001FF20684F
:10BD000002F003FFB04201D00D20DAE701225146D4
:10BD1000204600F033F80020D3E7000010B51048AB
:10BD20000068407E60B106210120FEF7EFF904466D
:10BD300024B10B480068416903208847002010BDEA
:10BD4000012007490968087601210846FEF7DEF957
:10BD500004461CB100200249096808762046EEE737
:10BD60006C2E002070B504460D462946206802F06E
:10BD7000E1FE2946206802F0ECFE70BD70B5044675
:10BD80000E4615463146206802F0DAFE1DB13146F6
:10BD9000206802F0E4FE70BD70B505460C462868C8
:10BDA000015929B12146286802F0BAFE012070BD70
:10BDB0000020FCE738B50546284600F047FA04465F
:10BDC0003CB96946284607F07EFC04460CB90020C1
:10BDD0002860204638BD2DE9FC4707468846914635
:10BDE00000243E4613E06B46012201A9484600F0BC
:10BDF00040F90098012800D00DE09DF8045000BFE4
:10BE000006F8015B641C0A2D00D104E000BFA8F114
:10BE10000100A042E7DC00BF0020307014B13846BA
:10BE2000BDE8FC870020FBE7F7B582B01646039813
:10BE3000019001A800F098FD0546002D02DA0B20C4
:10BE400005B0F0BD0E4850F825400CB10020207020
:10BE5000029810B10020029908700949029841F82F
:10BE60002500029808B1012E01D00020E8E7002249
:10BE700002A903A800F03AFA07463846E0E70000B6
:10BE8000642E00202DE9F74F8EB0044616461CB9EB
:10BE9000092011B0BDE8F08F06F03F06324602A936
:10BEA0000FA800F023FA0546002D70D102980390E8
:10BEB00003A80F9900F0EDFB05462DB99DF837005A
:10BEC00000F0800000B1062506F01C00002856D0C6
:10BED00045B1042D03D103A8FFF7C0FA054646F08B
:10BEE00008060AE09DF8120000F0110008B10725CD
:10BEF00003E006F0040000B10825002D51D106F042
:10BF0000080000284DD000F0C7FC01900A9901F10B
:10BF10000E00019906F042FD0A9901F116000199FF
:10BF200006F03CFD20200A99C8720A99029800F098
:10BF300045FF814600220A99029806F01DFD0A99E4
:10BF400001F11C00002106F029FD01200299C870B2
:10BF5000B9F1000F25D00298C06A0190002249462D
:10BF600003A804F071FE0546DDB9DDE9011001F01A
:10BF70000FF90546A9F101000299C86011E085B9E1
:10BF80009DF8120000F0100010B1042509E05DE0FA
:10BF900006F0020028B19DF8120000F0010000B187
:10BFA00007254DB906F0080008B146F04006029892
:10BFB000C06A20620A986062002D55D10A990298E1
:10BFC00000F0FCFEA0600A9901F11C0000F009FFDE
:10BFD000E060029820600298C088A080267400204B
:10BFE0006074E06160614FF40072002104F1280088
:10BFF00001F044F806F0200040B3E06830B3E06898
:10C000006061029840894FEA402AA768D4F80C8002
:10C010000CE03946204600F0CFFB0746012F00D840
:10C020000225781C00B90125A8EB0A080DB9D045F6
:10C03000EFD8A76155B9C8F3080038B1394602985E
:10C04000FEF77EFEB0F1000B01D102250CE00BEBF8
:10C050005820E061E26902994878012304F128013F
:10C06000FFF74EFB00B101250DB1002020602846EE
:10C070000FE72DE9FF4F85B0044615469A46DDF8D7
:10C0800018B00020CAF8000003A9204607F01BFBE7
:10C090000490049810B9607C049018B1049809B019
:10C0A000BDE8F08F207C00F0010008B90720F6E71A
:10C0B0006169E068401A01900198854200D9019DAC
:10C0C000A0E0A08AC0F3080000287ED10398408930
:10C0D000401E616900EA5129B9F1000F17D160696A
:10C0E00010B9A068029004E02046A16900F064FB4A
:10C0F00002900298022802D202206074CFE70298D0
:10C10000401C10B901206074C9E70298A061A169C0
:10C110000398FEF715FE064616B902206074BEE7C6
:10C120004E444FEA5528B8F1000F29D009EB08001A
:10C1300003994989884203D903984089A0EB0908EB
:10C1400003994878434632465946FFF7D9FA10B169
:10C1500001206074A3E7207C00F0800068B1E069F2
:10C16000801B404509D2E169891B0BEB41204FF44C
:10C17000007204F1280100F074FF4FEA482737E00D
:10C18000E069B04220D0207C00F0800078B1E26904
:10C1900003994878012304F12801FFF7A3FB10B1AC
:10C1A000012060747BE7207C00F07F0020740399FD
:10C1B00048780123324604F12801FFF7A1FA18B1AB
:10C1C000012060746BE700E0E661A08AC0F308001C
:10C1D000C0F50077AF4200D92F46A08AC0F308020D
:10C1E00004F1280011183A46584600F03AFF00BF03
:10C1F000BB44606938446061DAF800003844CAF82A
:10C200000000ED1B002D7FF45CAF002047E733B545
:10C210008BB00D46002269460BA800F067F8044673
:10C220008CB968460B9900F034FA04465CB99DF865
:10C230002B0000F0800008B1062404E01DB129465F
:10C24000684600F04BFB20460DB030BDF8B5044603
:10C250006946204607F037FA0646002E44D1207C76
:10C2600000F0400000283FD0207C00F0800070B13A
:10C27000E26900994878012304F12801FFF732FBB5
:10C2800008B10120F8BD207C00F07F00207400F090
:10C2900003FB0746216A009800F07AFF06461EBBA2
:10C2A000656AE87A40F02000E8722946A2682068B2
:10C2B00006F062FB05F11C00E16806F06FFB3946F1
:10C2C00005F1160006F06AFB002105F1120006F0E8
:10C2D00071FB01200099C870009806F021FC064609
:10C2E000207C00F0BF0020743046CBE72DE9F74FEB
:10C2F0008AB000210B9801600A9800F035FB089085
:10C300000898002803DA0B200DB0BDE8F08FB14982
:10C31000089851F820400CB90C20F5E70B98046000
:10C320000C9800F0FE000C90207878B16078FFF750
:10C3300051FA814609F0010040B90C9820B109F08A
:10C34000040008B10A20DFE70020DDE700202070AC
:10C35000089860706078FFF7EDF8814609F00100F9
:10C3600008B10320D0E70C9820B109F0040008B10F
:10C370000A20C9E7002739462046FEF76DFC05462E
:10C38000022D01D02EDA2DE0002614E04FF4DF70EC
:10C3900000EB061104F13000084409900998007977
:10C3A00020B10998083000F01CFD00E0002002A92F
:10C3B00041F82600761C042EE8D3002606B1761E2E
:10C3C00000BF02A850F8267027B139462046FEF774
:10C3D00043FC00E003200546022D03DB701C0646EB
:10C3E0000428EED3042D01D101208DE7022D01DBBD
:10C3F0000D2089E704F13B0000F0FFFCB0F5007F61
:10C4000001D00D2080E704F1460000F0F6FC8046E4
:10C41000B8F1000F04D104F1540000F0E2FC8046B2
:10C42000C4F818804020005DA070A078012804D0D6
:10C43000A078022801D00D2066E7A07808FB00F85C
:10C440003D20005D6081608918B16089411E08400F
:10C4500008B10D2058E704F1410000F0CEFC208126
:10C46000207A00F00F0008B10D204DE704F14300E1
:10C4700000F0C3FC8246BAF1000F04D104F1500071
:10C4800000F0AFFC824604F13E0000F0B6FC0190E3
:10C49000019808B90D2037E701984044218900EB45
:10C4A000111007900798824501D20D202CE70798BC
:10C4B000AAEB00006189B0FBF1FBBBF1000F01D1D9
:10C4C0000D2021E703254FF6F570834500D802259E
:10C4D00040F6F570834500D801250BF1020060613C
:10C4E000E76101983844206207983844A062032D20
:10C4F00013D104F15A0000F080FC08B10D2003E7CD
:10C50000208908B10D20FFE604F15C0000F069FC11
:10C51000606260698000069014E0208908B90D20EF
:10C52000F2E6206A40446062022D02D16069400058
:10C5300007E0207D00F00100616901EB410100EBA3
:10C5400051000690A169069800F2FF10B1EB502F40
:10C5500001D20D20D8E64FF0FF302061E06080204E
:10C560002071032D2CD104F1600000F046FC01285D
:10C5700026D1791C204600F00BFE08BB002020715C
:10C5800004F22E2000F039FC4AF65521884217D1DA
:10C5900004F1300000F025FC0F49884210D104F569
:10C5A000057000F01EFC0D49884209D104F50670A3
:10C5B00000F017FC206104F5077000F012FCE06049
:10C5C000257007480088401C80B205490880E0803B
:10C5D000002099E6642E002052526141727241613E
:10C5E000682E002010B50446E07FFF2808D0A07F09
:10C5F00018B1E07F01F095FC02E0E07F01F020FD42
:10C6000000206077207204F10800D4E900219047EF
:10C6100010BD70B505460E46144624B13146284675
:10C6200000F02EFF03E03146284600F00BFF70BDFE
:10C6300030B504461088C01C984201D90C2030BD8A
:10C640000220158848551088401C1080012015884C
:10C6500048551088401C108015884C551088401C87
:10C6600010800020EBE770B504460D4640F21442FE
:10C67000115B0122D4F81004FDF7F6F9064606B165
:10C68000357004F13C0204F5826104F1540072DF5C
:10C6900070BD2DE9F34104462646D6F8008002E03D
:10C6A0000198401C0190019800782F28F8D001983B
:10C6B00000785C28F4D00020B06001980078202831
:10C6C00008D280212B20015500212046FEF7E4FEF0
:10C6D00005462CE000BF01A92046FEF7A9FC05464F
:10C6E00005B123E02046FEF7FDFD05462B20075D42
:10C6F0003DB1042D04D100BF07F0040000B90525A9
:10C7000014E007F0040000B110E0B07900F0100070
:10C7100008B905250AE0208AC0F3080208F13000B4
:10C720001118404600F04AFBB060D4E700BF28462D
:10C73000BDE8FC8170B505460C4660880C49098847
:10C74000884214D1208840F6772188420FD1A088F2
:10C75000C01E084908802B886A880749074E891B34
:10C76000C908042646EA014005A101F055FF70BD45
:10C770004C2E00204E2E0020644F0300CC4E0300B0
:10C78000415454204D54552065786368616E676547
:10C7900020636F6D706C657465642E2063656E74C4
:10C7A00072616C20256420706572697068657261C1
:10C7B0006C202564000000002DE9F04781460C46FE
:10C7C000D9F80050022C02D36869A04202D84FF079
:10C7D00001085EE04FF0FF382878012804D00228D5
:10C7E0002CD0032851D13CE0264606EB5606286A99
:10C7F00000EB5621284600F0CBFC00B148E0304663
:10C80000761CC0F3080105F13000475C286A00EB94
:10C810005621284600F0BCFC00B139E0C6F30801FF
:10C8200005F13000405C47EA002704F0010008B140
:10C83000380901E0C7F30B00804629E0286A00EBC5
:10C840001421284600F0A4FC00B121E040F2FF11C1
:10C8500001EA440205F13001501800F0CEFA80469A
:10C8600016E0286A00EBD411284600F091FC00B1D4
:10C870000EE040F2FF1101EA840205F13001501888
:10C8800000F0AFFA20F0704802E04FF0010800BF5E
:10C8900000BF4046BDE8F0871CB51F201D211723AF
:10C8A0001A46CDE9001001214FF4FD6000F001F8B7
:10C8B0001CBDF0B50446DDE905560020A4F2BC77A6
:10C8C00040EA47604F1C40EA475040EA024040EAD5
:10C8D000C32040EA451040EA5600F0BD2DE9F0477C
:10C8E00005460C4600206072A86908B9BDE8F087CB
:10C8F000002637461CE03046761CEA6912F80090A4
:10C90000B9F1200F00D113E0B9F1050F01D14FF0BB
:10C91000E509092E05D12E2238467F1C04F10901B4
:10C920000A5438467F1C04F1090101F8009000BF49
:10C930000B2EE0D3002104F10900C155E869C07A4B
:10C940002072E96901F11C0000F04BFA2060E969EE
:10C9500001F1160000F045FA8046A4F806804FEA7F
:10C960001840A08000BFC1E770B502464FF0FF300D
:10C970001568DDB1116800E0491C0D78212D02D346
:10C980000D783A2DF8D10D783A2D0ED1146814F89F
:10C99000015BA5F130030A2B06D28C4204D11BB9EE
:10C9A00018464D1C2946156070BD002000BFFBE7EE
:10C9B00070B50B48FFF768F80A4B0CCB841843F1AD
:10C9C0000005094903C9201A75EB010004D24FF094
:10C9D0008073E41845F100052046294670BD00002B
:10C9E000A02D0020B02D0020B82D002038B51F202C
:10C9F0000090684601F0A2FA044600BFD4F8100582
:10CA00000099C84000F0010038BD00000246002136
:10CA10000CE001EB8100074B33F82000904204D179
:10CA200001EB810003EB80007047491C0029F0D026
:10CA30000020F9E7C85700202DE9FC5F83460E4629
:10CA400091461F46DDE90C45002E01DA704200E0F8
:10CA5000304682464FF0010803E09AFBF9FA08F1EC
:10CA60000108CA45F9DA474500D9B84634B1002E65
:10CA700003DB05F00400042800D1641E05F0020069
:10CA800000B167B105F0010048B944B104E0641E8B
:10CA900020215846FDF75CFF0CB1A045F7D3002ECE
:10CAA00005DA76422D215846FDF752FF07E005F0E2
:10CAB0000400042803D12B215846FDF749FF05F057
:10CAC000020002280DD105F0010050B94FB944B160
:10CAD00004E0641E30215846FDF73AFF0CB1A04532
:10CAE000F7D33B464A4631465846CDE9004506F065
:10CAF000B3FCBDE8FC9F30B5024600201378C3F3B9
:10CB00008003D3B1137803F00303012B02D0022B6F
:10CB100010D107E01388C3F383139B1C0C682344D4
:10CB20000B6008E00B680225146805EB945423445D
:10CB30000B6000E000BF00BF012030BD70B50546AE
:10CB40000C464FF48C71284602F0F4FA38B14FF4D9
:10CB50008C71284602F0F5FA2046FFF743FD70BDC0
:10CB600070B505460C464FF48871284601F053FF16
:10CB700068B14FF48871284601F054FF607900F0E5
:10CB8000040020B1206810B10120216888474FF4CB
:10CB90008A71284601F03FFF68B14FF48A71284638
:10CBA00001F040FF607900F0080020B1206810B16A
:10CBB0000220216888474FF48E71284601F02BFF30
:10CBC00068B14FF48E71284601F02CFF607900F0B7
:10CBD000100020B9206810B10020216888474FF468
:10CBE0008271284601F017FF58B14FF48271284630
:10CBF00001F018FF01202071206810B10320216886
:10CC0000884770BD2DE9F04781460C4616464FF423
:10CC100080374FF4A078002520E03946484601F0DF
:10CC2000A1FFA8B14146484601F08DFF80B13946C9
:10CC3000484601F07CFF3946484601F087FF4146EF
:10CC4000484601F066FFE8B21B4A52F824108847B4
:10CC50007F0008F104001FFA80F86D1CB542DCD398
:10CC60004FF480780121484601F07CFF68B14146CD
:10CC7000484601F068FF40B14146484601F049FF8F
:10CC80000D4850F82410042088474FF48278022180
:10CC9000484601F067FF68B14146484601F053FF3E
:10CCA00040B14146484601F034FF034850F8241093
:10CCB00005208847BDE8F087842D00202DE9F04746
:10CCC00004460E469046002722E0384602F074FAE9
:10CCD0000546384602F077FA8146204629464258F2
:10CCE0000AB1012200E0002282B14846D4F80413C0
:10CCF000014009B1012100E0002139B12946204657
:10CD000002F066FA2846D6E900219047781CC7B29F
:10CD10004745DADBBDE8F0872DE9F0410446A088FD
:10CD200000EB020CB4F80480904501DD104600E0F1
:10CD3000A088A8EB0005E088C618B4F806809845DE
:10CD400001DD184600E0E088A8EB00074888B4F849
:10CD50000080404504DB4888B4F80280404502DD8D
:10CD60000020BDE8F0818888A84202D38888604509
:10CD700001D90020F5E7C888B84202D3C888B0427C
:10CD800001D90020EDE70120EBE70146086808B172
:10CD900002680A60704710B504462246022100204E
:10CDA00001F098F8002105E054F8210008B10120B5
:10CDB00010BD491C0229F7D30020F9E770B50546DC
:10CDC0000C4604F11A0000F018F8064628780328EB
:10CDD00005D104F1140000F010F846EA0046304690
:10CDE00070BD0146C8788A7842EA00204A7842EA53
:10CDF00000200A7842EA00207047014648780A7805
:10CE000042EA00207047000010B502F00DFA20B988
:10CE100002F02EFA00200149887010BD74580020DD
:10CE2000F7210180172141800021017141711B21EF
:10CE30008171C171704770472DE9FF4100272E486D
:10CE400000F034FB2C48001F00F030FB2B488068BA
:10CE500003902B4805680398284028490C3101EBC2
:10CE6000800800BF03A94046FFF745FE30B1039894
:10CE7000284022490C3101EB800800E000E0F1E796
:10CE800000BF00240AE00398411C284003911B497D
:10CE90000C3151F820004DF82400641C022CF2D310
:10CEA000009800F0030001280DD0022814D1BDF82D
:10CEB00006700421009801EB9050401E039901EB8D
:10CEC0009000039009E0BDF806700098C0F383104D
:10CED00003990844039000E000BF00BF0648001F0C
:10CEE00000F0DDFA064616B104490398886038461A
:10CEF00004B0BDE8F08100004078002028680020E0
:10CF0000F82D002000BF1A4A64213820FCF7ECF904
:10CF1000044600BF254625B100BF2846FCF712F99C
:10CF200000BF00BF00BF06F073FF1249124A891A02
:10CF3000C908032242EA014010A213A101F060FBDC
:10CF400016490A680B490C4BC91AC908032343EA5E
:10CF5000014013A101F054FB15A0194908601948BC
:10CF60004860084606F0EAFBFAF766FD05F0B0F9FE
:10CF7000C4340020644F0300CC4E030030303A31FB
:10CF8000353A343000000000636F6D70696C6520C5
:10CF900074696D65203A2573000000008010001050
:10CFA000435553544F4D4552203A2564000000002C
:10CFB000414453313239335F544553544552000094
:10CFC000702C0020B9FA02002DE9F04105460E460A
:10CFD00014469846A888871C2088801C3844404501
:10CFE00002D90C20BDE8F081FE2F01D90C20F9E711
:10CFF000781C218870542088401C2080FF202188C4
:10D0000070542088401C208022889119288806F0BE
:10D010001CFA218808442080A88800280DDDA86813
:10D0200008B90720DEE7AA8823889819A968FAF7C3
:10D03000E8F92088A988084420800020D2E7F0B5CC
:10D0400003461D460C46002000BF15F8017B14F86E
:10D0500001CBA7EB0C00561E321E01D00028F4D0E5
:10D06000F0BD30B503460C463AB100BF14F8015B81
:10D0700003F8015B551E2A1EF8D130BD10B50346DA
:10D0800000BF03F8011B541E221EFAD110BD2DE96A
:10D09000FF4F87B0044691461E46A2462546BAF881
:10D0A00006009AF805104843001F0690BAF806B02B
:10D0B000301DB0FBFBF00590301DB0FBFBF10BFB0E
:10D0C00011000490D9F8000081190698814202D914
:10D0D0000698801B01E0D9F800000746C9F80070E7
:10D0E00003E02D680598401E059005980028F8D1AA
:10D0F00003900498ABEB0008B84501D9384600E02E
:10D100004046804623E00399089808440290281D71
:10D11000049908440190149828B14246DDE90110B1
:10D12000FAF76FF904E04246DDE90101FAF769F91F
:10D13000002004902D68A7EB080703984044039053
:10D14000BB4501D9384600E05846804600BF002F55
:10D15000D9D10BB0BDE8F08F70B503460C469CB139
:10D1600001F016FB054600220AE0084800EB8201A8
:10D1700008881E68B04202D11A60002070BD521C9F
:10D18000AA42F2D30520F9E70020F7E700000000EB
:10D1900070B504460D460026E06AA84210D020462D
:10D1A00005F006FD06465EB9607801232A4604F1C3
:10D1B0003001FEF7A5FA10B14FF0FF350126E56208
:10D1C000304670BD2DE9F84F05460F461446984687
:10D1D0002878012804D1687810B90720BDE8F88FB5
:10D1E0002088801C404508D82878012807D120884D
:10D1F000801C69780844404501D90C20EEE720885E
:10D20000A8EB0000801E86B200962188891CC819F0
:10D2100069467DDF814600BF484600B1DEE700BFBA
:10D220002878022804D06878BDF80010884206DB10
:10D23000BDF80000B04202DC4FF0090A0BE04FF0ED
:10D24000080A2878012805D16878B04202DC68789D
:10D25000009000E00096BDF80000FE2801D90C20E7
:10D26000BCE7BDF80000401C218878542088401C91
:10D270002080208807F800A02088401C208020887B
:10D28000BDF80010084420800020A7E701460448AC
:10D290000088814201DA481C00E00020C0B27047DB
:10D2A000982D0020FEB504460D4600200190029006
:10D2B000CDF808D00220ADF804000020ADF806003B
:10D2C00001AA29462046ADDF06462EB90298FDF791
:10D2D00050F908B10120FEBD0020FCE70B480268B0
:10D2E0004FF08050D0F834110D2A0DD121B1012911
:10D2F00004D0022906D103E0012070470120FCE799
:10D300000120FAE70120F8E70020F6E730010010DD
:10D310000B4802684FF08050D0F834110D2A0DD11F
:10D3200021B1012904D0022906D103E00020704771
:10D330000020FCE70120FAE70120F8E70020F6E7EB
:10D34000300100100B4802684FF08050D0F83411C3
:10D350000D2A0DD121B1012904D0022906D103E003
:10D36000012070470120FCE70120FAE70120F8E7DF
:10D370000020F6E7300100100B4802684FF08050A3
:10D38000D0F834110D2A0DD121B1012904D0022980
:10D3900006D103E0012070470120FCE70120FAE7F5
:10D3A0000120F8E70020F6E73001001010B5044630
:10D3B00009B90E2010BD92FBF3F003FB102008B159
:10D3C0000920F7E7216000206060A060A281E3816E
:10D3D00000BFEFE770B504460D4629462046F9F731
:10D3E0001BFF18B12A882168881870BD0020FCE74F
:10D3F00070B505460C4620886188884204D12846CD
:10D40000F9F74CFF012070BD0020FCE770B5044621
:10D410000D4629462046F9F724FF18B16A8821688D
:10D42000881870BD0020FCE770B505460C462088C2
:10D430006188884204D12846F9F70AFF012070BDAF
:10D440000020FCE770B505460C4604F01F030122DE
:10D450009A40D143620905EB820000F039F8064694
:10D4600070BD10B50246480952F8200001F01F04B3
:10D470000123A340184008B1012010BD0020FCE7A3
:10D4800070B505460C4604F01F03012202FA03F1B1
:10D49000620905EB820000F03CF8064670BD10B54D
:10D4A00004460021204600F01EF810BD10B50446C9
:10D4B0000121204600F02DF810BDF8B504460D46B8
:10D4C0006A4629462046F9F73EFF06460098F8BD11
:10D4D000F8B504460D466A4629462046F9F719FF75
:10D4E00006460098F8BDF8B504460D466A4629463A
:10D4F0002046F9F70EFF06463046F8BDF8B504465B
:10D500000D466A4629462046F9F7EAFE06463046A9
:10D51000F8BDF8B504460D466A4629462046F9F797
:10D52000EBFE06460098F8BDF8B504460D466A467F
:10D5300029462046F9F714FF06460098F8BDF8B5CD
:10D5400004460026002000906846FCF765F9206834
:10D5500000686168884215D920680068401E22680A
:10D5600010600178204600F033F80646207A2168E2
:10D570000978401AC5B220680079A84201DA20680B
:10D58000057100BF9DF80000FCF74CF93046F8BD6E
:10D590000246D068081A138AB0FBF3F0C0B2704795
:10D5A000F8B504460D462E46002000906846FCF76C
:10D5B00033F931462046FFF7EBFF21680A68511C1A
:10D5C0002368196010709DF80000FCF72BF9F8BD76
:10D5D0000246138AD06801FB0300704710B501466C
:10D5E00000BF09B90E2010BD00BF087A0B79C01A20
:10D5F000C2B2D1E90030186005E008680368581C21
:10D600000C6820601A70101EA2F10103DAB2F4D186
:10D610000B68187100BFE6E730B502460B46D40828
:10D6200002F00702012090401D5D284030BD0246F7
:10D6300000BF0AB90E20704700BF172901DBF72988
:10D6400001DD0720F7E711800020F4E770B50446FC
:10D650000E4600BF0CB90E2070BD00BF2661F7203A
:10D66000208060801B202071002505E0A11D01EBBA
:10D67000C500FFF7D5FB6D1C002DF7D00020EBE7B0
:10D680002DE9F047064688464546B488012C01DB63
:10D69000BDE8F0873088242820D006DC102809D087
:10D6A00011280CD0232823D11DE03A280CD055286E
:10D6B0001ED10EE03146284602F056FB19E03146F5
:10D6C000284602F05EFD14E03146284602F022FEB4
:10D6D0000FE03146284602F05FFD0AE03146284659
:10D6E00002F01EFC05E03146284602F0C1FC00E0D5
:10D6F00000BF00BFA81D00EBC400007970B3A81DD7
:10D7000030F834102046A5DF0746C7B90021A81D10
:10D7100000EBC40001710121A81D00EBC4004171A0
:10D72000A91D31F834201149114BC91AC908042325
:10D7300043EA014023460F4900F06EFF12E0112F2B
:10D7400010D0384601F02AFD81460849084A891A56
:10D75000C908012242EA01404A4600E003E006A16E
:10D7600000F04EFF00BF00BF92E70000CC4E030068
:10D77000CC4E03009845030073645F626C655F677D
:10D78000617474635F65786368616E67655F6D740B
:10D79000755F72657175657374282920726574757B
:10D7A000726E65642025732E0000000010B50446DB
:10D7B000206841692046884710BD70B504460D4673
:10D7C000164620683246294603692046984770BDB0
:10D7D00001464FF08040405808B1012070470020BA
:10D7E000FCE708B500224FF080410A50095800912B
:10D7F00000BF08BD014908607047000008030040F1
:10D80000012291070A5070472DE9F04104460CB9F6
:10D81000BDE8F08100BF4FF47A7505B904E0054F0B
:10D82000AE013046B84700BF601E041EF3D100BFF2
:10D83000EEE70000A13F030070B540F6F870006805
:10D84000401C18B94FF01020406902E040F6F87013
:10D8500000680546681C00281CD01449144A891A1F
:10D86000C908032242EA01402A4612A100F0C8FE7C
:10D87000284613DF04465CB10C490D4A891AC908D1
:10D88000012242EA014016A100F0B0FE204670BD20
:10D890000020FCE70549064A891AC908012242EA24
:10D8A00001401CA100F0A2FE0420F0E7644F030039
:10D8B000CC4E030053657474696E6720766563749B
:10D8C0006F72207461626C6520746F20626F6F7478
:10D8D0006C6F616465723A203078253038780000CA
:10D8E0004661696C65642072756E6E696E6720733F
:10D8F000645F736F66746465766963655F7665639C
:10D90000746F725F7461626C655F626173655F738F
:10D91000657400004E6F20626F6F746C6F61646598
:10D92000722077617320666F756E640010B50E49C2
:10D930000E4A891AC908032242EA01400C4A0DA185
:10D9400000F05EFE0A4813DF04465CB10649074A50
:10D95000891AC908012242EA014011A100F046FEDD
:10D96000204610BD0020FCE7644F0300CC4E0300AE
:10D970000070020053657474696E67207665637485
:10D980006F72207461626C6520746F206D61696EC6
:10D99000206170703A20307825303878000000001F
:10D9A0004661696C65642072756E6E696E6720737E
:10D9B000645F736F66746465766963655F766563DB
:10D9C000746F725F7461626C655F626173655F73CF
:10D9D0006574000010B500240F48007808B1852454
:10D9E00011E000200C49886048600861C8600B485D
:10D9F00001F02EFC044601F0FBFA08B901F01EFC10
:10DA000001200549087001F00FFC10B10120024906
:10DA10008870204610BD00007458002019AD020027
:10DA200008B5002000906846FBF7F6FE0748C0687E
:10DA3000401E0649C8600846C06808B9FFF7E4F907
:10DA40009DF80000FBF7EEFE08BD000074580020B2
:10DA50002DE9FF4705460C46164698462F781A488A
:10DA600040F82760194840F827804FF00009184B0C
:10DA70000FCB8DE80F0020788DF8000060788DF8CE
:10DA80000100A0788DF80200E0788DF8030020797D
:10DA90008DF8050060798DF80600A0680290207B63
:10DAA0008DF80C00607B8DF80D000EB1094800E088
:10DAB000002002463B466946281D01F067FE81466C
:10DAC000484604B0BDE8F087685900207859002026
:10DAD00038400300292803002DE9FF4704460D467E
:10DAE00016461F46DDF830804FF00009009501967C
:10DAF0000297CDF80C8000226946201D01F094FFAA
:10DB00008146484604B0BDE8F0872DE9FF4704464A
:10DB10000D4616461F46DDF830804FF0000900958F
:10DB200001960297CDF80C8000226946201D01F075
:10DB30007BFF8146484604B0BDE8F0870FB438B596
:10DB40000446059810B938BC5DF814FB002000901D
:10DB500006A800906A462046059900F012F80020B9
:10DB6000009000BFEFE770B50446A06800B970BD33
:10DB7000D4E90403A268216898470020A06000BF90
:10DB8000F5E72DE9FC5F82460D4614460DB9BDE868
:10DB9000FC9F00BF2E786D1C06B9E1E0252E70D1E8
:10DBA00000274FF0010900BF2E782B2E0CD02D2E10
:10DBB00002D0302E0CD103E047F001076D1C0AE0C3
:10DBC00047F002076D1C06E047F004076D1C02E0F9
:10DBD0004FF0000900BF00BFB9F1000FE4D14FF0D2
:10DBE000000800BF2A2E06D12168081D20600868A1
:10DBF00080446D1C0DE02E78302E01DB392E00DDC7
:10DC000007E06D1CA6F1300008EB880100EB41082D
:10DC1000E8E700BF4FF0000B2E782E2E10D16D1CC0
:10DC200000BF2E78302E01DB392E00DD07E06D1CA1
:10DC3000A6F130000BEB8B0100EB410BF1E700BFCD
:10DC40002E7800BF6C2E01D0682E02D16D1C2E786C
:10DC500000E000E0F6E700BF692E21D008DC252EA9
:10DC60006DD0582E39D0632E0CD0642E6CD116E0B6
:10DC7000702E4CD0732E3ED0752E1FD0782E63D1CF
:10DC80002AE065E02168081D2060D1F8009009F0C5
:10DC9000FF00019050460199FCF75AFE55E000BF85
:10DCA0002168081D2060D1F800905B460A22494691
:10DCB0005046CDE90087FEF7BFFE46E02168081D0B
:10DCC0002060D1F800905B460A2249465046CDE9D3
:10DCD000008705F0C1FB38E000BF2168081D206007
:10DCE000D1F800905B46102249465046CDE90087A6
:10DCF00005F0B2FB29E02168081D2060086801904A
:10DD00003B4642465046019904F0D0FE1DE0216892
:10DD1000081D2060D1F8009030215046FCF718FE15
:10DD200078215046FCF714FE002008210B461022F3
:10DD3000CDE900104946504605F08EFB05E025214F
:10DD40005046FCF705FE00E000BF00BF6D1C03E07D
:10DD500031465046FCF7FCFD287800287FF41AAFC6
:10DD600000BF9AF80C0010B15046FFF7FCFE00BF50
:10DD70000DE72DE9FF470C4615461E46DDE90C78F8
:10DD8000684600F0FBF8814644EA450040EA860018
:10DD900040EA072040EA084109F5E060009A40F8AF
:10DDA0002210BDE8FF872DE9FF470C4615461E46A9
:10DDB000DDE90C78684600F0F1F8814644EA450058
:10DDC00040EA860040EA072040EA084109F5E060A1
:10DDD000009A40F82210BDE8FF872DE9FF470C4666
:10DDE00015461E46DDE90C78684600F0E7F88146E6
:10DDF00044EA450040EA860040EA072040EA08413C
:10DE000009F5E060009A40F82210BDE8FF872DE98F
:10DE1000F84F05460C4600263746B046B1460095F9
:10DE2000684600F08BF8824646EA470040EA8400E4
:10DE300040EA082040EA09410AF5E060009A40F80B
:10DE4000221000BFBDE8F88F1CB5044600200090EA
:10DE500003460122114601902046FFF7A4FF1CBD96
:10DE60002DE9F84F06460D4614460027B846B94638
:10DE70000096684600F072F8824647EA480040EA99
:10DE8000850040EA092040EA04410AF5E060009A72
:10DE900040F8221000BFBDE8F88F73B50D46684604
:10DEA00000F06CF8044604F5E060009950F8210099
:10DEB00020F4403104F5E060009A40F82210009907
:10DEC00050F8210040EA054104F5E060009A40F86E
:10DED00022107CBD3CB503460A4D30CDCDE900454E
:10DEE00018460BE05DF82040D4F8204514605DF83A
:10DEF00020501468C5F82045121D401C5C1884424F
:10DF0000F0D83CBDC03F030031B5684600F016F8BC
:10DF100004460121009A01FA02F0C4F80C0500BF82
:10DF200038BD31B5684600F039F804460121009A41
:10DF300001FA02F0C4F80C0500BF38BD01460868BC
:10DF4000202802D24FF0A0407047087800F01F0050
:10DF500008600148F8E70000000300500146086827
:10DF6000202802D24FF0A0407047087800F01F0030
:10DF700008600148F8E70000000300500146086807
:10DF8000202802D24FF0A0407047087800F01F0010
:10DF900008600148F8E700000003005001460868E7
:10DFA000202802D24FF0A0407047087800F01F00F0
:10DFB00008600148F8E700000003005001460868C7
:10DFC000202802D24FF0A0407047087800F01F00D0
:10DFD00008600148F8E700000003005001464A09C4
:10DFE000002312B1012A06D102E04FF0FF3302E014
:10DFF00040F2FF3300BF00BF01F01F010120884045
:10E00000184008B1012070470020FCE731B5684690
:10E01000FFF7B4FF044600BFD4F810050099C840CC
:10E0200000F0010038BD31B56846FFF787FF0446B0
:10E030000121009A01FA02F0C4F8080500BF38BDBA
:10E0400031B56846FFF7AAFF04460121009A01FA9C
:10E0500002F0C4F8080500BF38BD31B56846FFF7C7
:10E06000ADFF04460121009A01FA02F0C4F8080548
:10E0700000BF38BDF8B504460D466DB9009468463A
:10E08000FFF76CFF06460121009A01FA02F0C6F87C
:10E090000C0500BF00BF0DE000946846FFF75EFF6F
:10E0A00006460121009A01FA02F0C6F8080500BFF1
:10E0B00000BF00BFF8BD000001460148084470479A
:10E0C0000060004038B504462046FFF7F5FF002108
:10E0D00001602046FFF7F0FF0068009000BF38BDE8
:10E0E00010B504462046FFF7E7FF0068012800D17D
:10E0F00010BD0020FCE700000149086070470000E7
:10E100000463004070B504460E46FBF7D9FB054694
:10E11000681C08B9284670BDE8B2E168087100BF04
:10E120000A48006928B9094804610020E1680860CC
:10E1300009E006480069C0680068E16808600348B3
:10E140000069C06804602846E5E7000028780020E0
:10E15000704710B5FAF7A4F910BD704738B50446FA
:10E160000D4605484FF48063044A29460090204636
:10E1700000F006F838BD0000891F0300085B00208E
:10E180002DE9F04F93B082460E4617469846DDF8CB
:10E190007090304600F0F5FB18210DA8F9F74AF908
:10E1A0000D97CDF83880CDF8489000252B460822F1
:10E1B00007A9304600F002FC082509980A90BDF82E
:10E1C0002000ADF82C00BDF82200ADF82E00002094
:10E1D0008DF83100079800F0030001281BD1079843
:10E1E0004FEA902B0798C0F3C2008DF830000798D3
:10E1F000C0F38314A2002B4601A9304600F0DEFBD9
:10E2000005EB84050DA80AAB224601A900905846EB
:10E2100000F0F6FA27E0079800F00300022822D168
:10E2200007984FEA905B0798C0F3C2008DF8300062
:10E2300000BFBBF1080F01D2584600E00820044699
:10E240002B46224605A9304600F0B8FB2544ABEB2F
:10E25000040B0DAB0AAA214605A800F017FABBF182
:10E26000000FE6D100BF304600F099FB13B0BDE8C7
:10E27000F08F000010B502460B4C04EBC2030129DD
:10E2800006D0022906D0032906D0042908D105E0CA
:10E29000022007E0042005E0187903E0587901E046
:10E2A000002000BF00BF10BDCC4E030010B54FF0E2
:10E2B000FF34FFF74EFF04210548FFF723FF044614
:10E2C00000BF01200249C968487100BF10BD0000AD
:10E2D000BC4E03002DE9F04F8BB0FCF74FFB18B19B
:10E2E00000200BB0BDE8F08F0021B548816100BF70
:10E2F00000BF00BFBFF34F8F00BF00BF00BFA0F53E
:10E30000805080680A90AF4804680A982040AE495F
:10E3100001EB800A002500260020069000BF0AA914
:10E320005046FEF7E8FBB0B1A548806998B9A64809
:10E330000C3840680A99884207D8A3480C384068CE
:10E34000A1490C3988600020CBE70A9820409E49FB
:10E3500001EB800A00E000E0E1E700BF00270AE0EF
:10E360000A98411C20400A91974951F8200007A9BA
:10E3700041F827007F1C022FF2D3079800F003001A
:10E3800002287AD10798800D05904FF448710798BC
:10E39000B1EB905F02DD0798800D01E04FF448700B
:10E3A0008146079869F39F50079009F1080004908F
:10E3B0000798C0F3C20006908448049900F084FADC
:10E3C0000546002D57D0284600F0DBFA33460822D8
:10E3D00007A9284600F003FB08360A982040611C74
:10E3E000081A4FEA8008C14532D9B8F1000F05D0AC
:10E3F0000A982040744901EB800000E072480390C5
:10E40000B8F1000F01D0404600E0484600F0FF0B95
:10E41000B8F1000F01D06C4800E000200290B8F184
:10E42000000F02D0A9EB080000E00020C0B201906C
:10E4300033465A462846039900F0D1FA5E440298C2
:10E4400028B133462846DDE9012100F0C8FA0BE087
:10E450000A9820405C4901EB800B33464A465946F6
:10E46000284600F0BCFA00BF0598C01C0A9901EBD1
:10E4700090000A9000BF43E0FFE7079800F0030018
:10E4800001283DD10798C0F38310062803DA0798C6
:10E49000C0F3831000E00620079960F3891107910B
:10E4A0000798C0F3831000F102080798C0F3C20078
:10E4B00006904FEA8801454800F006FA0546F5B196
:10E4C000284600F05EFA3346082207A9284600F0E5
:10E4D00086FA083600270DE00A98421C20400A926E
:10E4E000394A02EB800133460422284600F077FACD
:10E4F000361D7F1C0798C0F38310B842ECD800BFCC
:10E50000DDB32F48D0F81080806918B1284600F09C
:10E5100046FA31E019E04FF0000900BFD8F80C00CE
:10E520004079012800D18146B9F1000F08D000BF21
:10E53000D8F80000294602684046904700BF00BF57
:10E54000D8F80C00D0F8008000BFB8F1000FE2D17D
:10E55000284600F024FA0020059005A8FBF75CF996
:10E560001748806918B918490C390A9888609DF8CD
:10E570001400FBF757F900BF1DE0FFE71048D0F883
:10E5800010800AE0C146D9F80000816848468847F3
:10E5900000BFD8F80C00D0F80080B8F1000FF1D11E
:10E5A0000B490C4A891AC908022242EA01400AA111
:10E5B00000F01CF800BFFCF7E1F980F0010090E6E4
:10E5C00028780020F82D002034680020844F0300B4
:10E5D000644F0300CC4E03004261636B656E64734D
:10E5E00020666C75736865640000000070B50446B1
:10E5F0000D4600231A462946204604F013FA70BD42
:10E60000F8B505460E461446009401236A46314685
:10E61000284604F007FAF8BD2DE9FC4106460F46EE
:10E6200014461D460094019502236A463946304639
:10E6300004F0F8F9BDE8FC812DE9FE4306460F46DB
:10E6400014461D46DDF8288000940195CDF8088019
:10E6500003236A463946304604F0E4F9BDE8FE83F8
:10E660002DE9FF4706460F4614461D46DDE90C8995
:10E6700000940195CDF80880CDF80C9004236A46EB
:10E680003946304604F0CEF9BDE8FF872DE9F05F4A
:10E6900007460E4690461D46082E01D9BDE8F09F5C
:10E6A00095F80C90002028732946404602F04CF85B
:10E6B00000240CE0B44205D23A5D1DA12846FFF7C4
:10E6C0003DFA03E01CA12846FFF738FA641C082C29
:10E6D000F0D31AA12846FFF731FA00241DE0B44216
:10E6E00016D217F804A0BAF17E0F09DCF8F77CFE09
:10E6F000006810F80A0000F03E0008B1504600E043
:10E700002E2083465A460EA12846FFF717FA03E04B
:10E710000CA12846FFF712FA641C082CDFD3012253
:10E720002946404601F0ECFF85F80C9000BFB5E7A4
:10E730002025303278000000202020007C000000DE
:10E7400025630000200000002DE9F04106460F4639
:10E7500000BF002009490870094800F01AF9044672
:10E7600014B12046BDE8F081064800F0B5F906482E
:10E770000649401AC5080020F4E700002868002078
:10E78000844F030078420300844F0300CC4E030003
:10E7900002480349401AC00870470000844F030034
:10E7A000CC4E030013B50C4621466846FEF7D4FC58
:10E7B00028B90448009A00EBC20108681CBD00207B
:10E7C000FCE70000CC4E030070B50B480469012043
:10E7D0000A4908700CE000BF0120E168487100BFE1
:10E7E0002546286841682846884700BFE0680468D5
:10E7F000002CF0D170BD000028780020286800208F
:10E800002DE9FF4707460C46164698460C9D95F89D
:10E810000C90002028732946404601F095FF072EF2
:10E8200047D2DFE806F004090F161F2A37003946E1
:10E830002846FFF783F93DE0394628462268FFF76E
:10E840007DF937E039462846D4E90023FFF776F909
:10E8500030E0A068009039462846D4E90023FFF74D
:10E860006DF927E0D4E90201CDE9000139462846D7
:10E87000D4E90023FFF762F91CE0D4E90212206911
:10E88000CDE90012029039462846D4E90023FFF76B
:10E8900055F90FE0D4E90223D4E90410CDE90023AF
:10E8A000CDE9021039462846D4E90023FFF746F99E
:10E8B00000E000BF00BF00222946404601F020FFD3
:10E8C00085F80C90BDE8FF872DE9F84F07468A468A
:10E8D000388AA0F104080AF104004044401EB0FB4D
:10E8E000F8F0C0B200903846FEF729FE044614B98D
:10E8F0000020BDE8F88F0020207101216171A4F88B
:10E90000068025460098A0F1010B2C462F604FF0A1
:10E91000000912E03846FEF712FE064636B160796D
:10E92000401C60712E603760354604E0204600F0E0
:10E9300008F80020DDE709F10109D945EAD32046AE
:10E94000D7E72DE9F05F0446274697F8058026466D
:10E95000A8F1010B002501E036686D1C5D45FBD375
:10E96000D6F800A02646002507E0D6F800903146EC
:10E970005046FEF715FE4E466D1C4545F5D3BDE8E5
:10E98000F09F70B5044625460121281DFEF795FD30
:10E9900070BD10B504462046FEF720FE10BDF8B548
:10E9A000044626460121301DFEF7BEFD00906D464F
:10E9B000287810B92046FFF7C4FFF8BD2DE9FC41C7
:10E9C00005460E4614461F46019401203B4601AA07
:10E9D000314600902846FEF75AFBBDE8FC812DE940
:10E9E000FC4105460E4614461F46019400203B4656
:10E9F00001AA314600902846FEF749FBBDE8FC819C
:10EA000000BF00BF00BFBFF35F8F00BF00BF00BFEC
:10EA10000021016070470246505808B1012070473C
:10EA20000020FCE708B5002242504258009200BF87
:10EA300008BD000010B500200A49087000BF0A494F
:10EA4000086000BF00BF00BF00BFBFF35F8F00BF03
:10EA500000BF00BF00BF0549054800F0FCFA0020D8
:10EA600010BD0000D82D0020D42D002090400300C0
:10EA7000A05A002070B50446144D01212846FEF727
:10EA80003DFD064600BF00BF00BF00BFBFF35F8F64
:10EA900000BF00BF00BF0EB9012000E0002000B998
:10EAA00070BD042C0BD00A48007818B10748FFF756
:10EAB000A7FFF5E70748047001200549087003F037
:10EAC000DFFC0248FFF79CFF00BFE9E7D42D0020E0
:10EAD000D82D0020D02D002000218268916082680E
:10EAE0001161826851618268D16082685160826878
:10EAF00011607047024602F5A86050F82100704787
:10EB000000F5A86343F8212070470146D1F80405B9
:10EB1000704708B5002242504258009200BF08BD1D
:10EB200008B5002242504258009200BF08BDC0F80C
:10EB300048137047C0F848137047C0F84413704733
:10EB4000C0F844137047024650587047C0F8081385
:10EB50007047C0F808137047C0F804137047C0F836
:10EB6000041370470246D2F804030840704701229C
:10EB7000425070470122425070470000024A106024
:10EB8000121D1160704700002C76004001460348BA
:10EB9000085808B1012070470020FCE700700040D1
:10EBA00008B50021034A815011464158009100BF29
:10EBB00008BD0000007000400121014A81507047EB
:10EBC00000700040014609B90E20704702480068F5
:10EBD00008600020F9E7000008430300FEB5064680
:10EBE0000C462046FFF7EEFF05460DB12846FEBD58
:10EBF00000200090019002908DF8006001208DF8B7
:10EC000002000621ADF8041069462020226869DF61
:10EC1000054675B1284600F0C1FA07464F49504AEB
:10EC2000891AC908012242EA01403A464D49FFF7D4
:10EC3000E7FC002000900190029001208DF8010077
:10EC400000208DF802008DF80300694640202268FC
:10EC500069DF054675B1284600F0A0FA07463F492E
:10EC60003F4A891AC908012242EA01403A463E4910
:10EC7000FFF7C6FC00200090019002908DF8006024
:10EC8000F720ADF8020069462320226869DF0546B7
:10EC900075B1284600F082FA07463049304A891A91
:10ECA000C908012242EA01403A463049FFF7A8FC70
:10ECB000002000900190029002208DF8000069462B
:10ECC0000120226869DF054675B1284600F066FA22
:10ECD00007462249224A891AC908012242EA01400C
:10ECE0003A462349FFF78CFC0020009001900290E7
:10ECF0004FF4C86000906946A120226869DF05468C
:10ED000075B1284600F04AFA07461449144A891A90
:10ED1000C908012242EA01403A461649FFF770FC51
:10ED200000200090019002908DF800006946A0201C
:10ED3000226869DF054675B1284600F02FFA0746BC
:10ED40000649074A891AC908012242EA01403A469F
:10ED50000949FFF755FC002049E70000744F030004
:10ED6000CC4E0300204C0300684C0300B44C03005D
:10ED7000804B0300CC4B03002C4B03002DE9F041EA
:10ED800004462568204660DF06462068A84225D94B
:10ED90001E491F4A891AC908022242EA01401DA1E0
:10EDA000FFF724FC19491A4A891AC908022242EAC3
:10EDB00001402A4623A12368FFF72EFC01F066FEDE
:10EDC0002168471A1149124A891AC908022242EADF
:10EDD00001403A4628A1FFF713FC00E000BF1EB92E
:10EDE0000120304908700EE0304600F0D7F90746A0
:10EDF0000649074A891AC908012242EA01403A46EF
:10EE000029A1FFF7FDFB3046BDE8F081744F0300F8
:10EE1000CC4E0300496E73756666696369656E74EE
:10EE20002052414D20616C6C6F6361746564206693
:10EE30006F722074686520536F66744465766963E9
:10EE4000652E00004368616E676520746865205216
:10EE5000414D207374617274206C6F636174696FCB
:10EE60006E2066726F6D203078257820746F2030A8
:10EE70007825782E000000004D6178696D756D2051
:10EE800052414D2073697A6520666F7220617070FF
:10EE90006C69636174696F6E2069732030782578BE
:10EEA0002E0000003F2E002073645F626C655F657A
:10EEB0006E61626C6528292072657475726E656476
:10EEC0002025732E000000002DE9F041ADF5027DF4
:10EED00080461848007818B90DF5027DBDE8F0812C
:10EEE0001DE04FF4FA70049004A905A861DF044600
:10EEF00004B115E005AD104901A800F0ACF809E037
:10EF000000BF03980646376828467168B84701A8CD
:10EF100000F0C2F800BF03980028F1D100BFE0E77D
:10EF200000BF052C04D000BF2046FAF70BF900BF44
:10EF300000BFD1E73F2E0020FC4203001CB51B4858
:10EF4000007808B108201CBD012019490870002074
:10EF500002F0A6FF112801D10020F4E7002002F002
:10EF6000BDFF144800680190002000906846FAF741
:10EF700053FC114901A810DF04460CB9012000E040
:10EF800000200A4908709DF80000FAF74BFC0CB10C
:10EF90002046D8E70020064908700849087003F0A9
:10EFA000E3FA012002F09AFF0020CCE73C2E00207B
:10EFB0003E2E0020D8420300859002003D2E002006
:10EFC0003EB50A49684600F046F809E0684600F098
:10EFD0003FF8044625686068A847684600F05CF87A
:10EFE000684600F035F80028F0D13EBDCC42030061
:10EFF00001480078704700003C2E00202DE9FF41B9
:10F00000074618E003A84BDF044604B114E00F499B
:10F01000684600F020F809E000BF029805462E6817
:10F0200069680398B047684600F036F800BF029858
:10F030000028F1D100BFE5E700BF052C04D000BFD8
:10F040002046FAF77FF800BFBDE8FF811C430300AC
:10F0500001468868704770B504460D4625602868EB
:10F060006060204600F001F870BD14E0D0E9002196
:10F070005268914202D1002181607047416809685D
:10F0800042685268914203D0416809688160F4E7A0
:10F09000416808314160E9E710B50446A06800B94D
:10F0A00010BD2168A06889680844A060D4E90110F7
:10F0B0004968884205D16068083060602046FFF7E3
:10F0C000D4FF00BFECE770B505460E466C6806E05D
:10F0D00020683146AA68904700B903E02468206898
:10F0E0000028F5D100BF20683060266070BD014661
:10F0F00048680068704701464A6810684A681268A4
:10F1000022B14A68126812684B681A60704710B5DD
:10F1100003460A460020596807E00C68944203D170
:10F1200014680C60012003E009680C68002CF4D11D
:10F1300000BF10BD0246505808B1012070470020A2
:10F14000FCE708B5002242504258009200BF08BDBB
:10F15000C0F80813704701224250704770B502464C
:10F160000D4B03F5947413E0E61AF01000EBD07623
:10F17000761003EBC6010D68954201D90C4606E0F6
:10F18000954202D201F1080301E0486870BD00BF5A
:10F19000A342E9D30020F9E7B040030030B50446AC
:10F1A0002046FFF7DBFF05460DB9024830BD284673
:10F1B000FCE700009C40030001464FF4A07000EB08
:10F1C000810080B2704701464FF48030884070471C
:10F1D00008B5002242504258009200BF08BD0021ED
:10F1E000C0F8001570470521C0F8001570470146AA
:10F1F000D1F8C404C1F8C40470470246505808B19D
:10F20000012070470020FCE708B500224250425818
:10F21000009200BF08BDC0F804137047C0F8001288
:10F2200070470122425070470348006808B101202E
:10F2300070470020FCE700000004014010B500F01A
:10F240008DF901200149086000BF10BD180500407C
:10F2500001460020054A12790AB1852004E0034ADC
:10F2600011600122014B1A7170470000642D0020CB
:10F2700010B50220FEF7BEFA4FF48270FEF7B1FA25
:10F280000C20FEF7BDFA00BF00BF03480068C0F3C2
:10F2900000400028F8D110BD1804004070B50446A5
:10F2A00004B970BD024EA5012846B04700BFF8E77B
:10F2B000614003000146080B40B270470146080B4D
:10F2C00040B270470146080B40B270472DE9F04745
:10F2D00006460D46304601F07FF9F0B13046FBF7A7
:10F2E000D1FBA0F10808404601F002FA0446032CC5
:10F2F00008D13046FEF78AFE08B1032000E0022064
:10F30000074605E0012C01D1022000E0032007465A
:10F3100039463046FEF7C1FD2AE0304601F068F973
:10F3200030B33046FBF7AEFB0446A00000F580701A
:10F3300087B220460F4951F8201041F001020D49D3
:10F3400041F8202000BF3846FEF7BCFE7DB13046B4
:10F35000FBF798FB8146FBF74DFB8046B8F1000FA9
:10F3600004D0012101FA04F0FEF7C6FE00BF00BF81
:10F37000BDE8F087106500402DE9FC4706460D46C4
:10F3800017464FF00008304601F018F910B14FF061
:10F39000080864E0A878C0F3400239463046FBF71D
:10F3A00031FB0446601C002856D0A878C0F38000CA
:10F3B00030BBA87800F0010090B1019601A8FEF7DB
:10F3C000DDFD814609F5E060019950F8210020F04B
:10F3D000020A09F5E060019940F821A000BF0CE0A5
:10F3E00095F80190002000904B460246014601909E
:10F3F0003046FEF7BEFC00BF00BF304601F0CEF83D
:10F40000A878C0F34000D0B12878164951F82410EC
:10F41000154A1140134A42F82410114651F824109D
:10F420004FF47C5202EA06224FF4403303EA0043D1
:10F430001A4311430B4A42F8241000BF0EE0A4F116
:10F4400008000A49085C297840EA811042B2A4F118
:10F45000080006490A5401E04FF0040800BF404686
:10F46000BDE8FC8710650040FFC0FCFFE2580020AB
:10F470002DE9F041304890F8640018B10826304674
:10F48000BDE8F081002408E02046FEF7A7FD10B19A
:10F49000204601F0BDF8601CC4B22A2CF4DB002425
:10F4A00004E02046FBF796FA601CC4B20C2CF8DB93
:10F4B00021485E300021016081802048FFF7FEFE78
:10F4C0000546062728463946002804DB4A07130E5E
:10F4D0001B4A135408E04A074FEA126C194A00F01D
:10F4E0000F031B1F02F803C000BF00BF1348FFF744
:10F4F000E5FE0546284600280DDB00BF00BF00F0F2
:10F500001F02012191404209920002F1E022C2F85B
:10F51000001100BF00BF00BF00BF4FF4BE70FEF778
:10F52000D1FD4FF00040FEF7E7FD0120024981F8D0
:10F53000640000263046A3E78858002000600040A1
:10F5400000E400E018ED00E0014601F06040B0F199
:10F55000005F01D1012070470020FCE72DE9F04158
:10F5600006254FF08040FFF7A5FE04462046E2172F
:10F5700004EBD2625211920002F1E022D2F8002193
:10F580002146E31704EBD3635B11A4EB431601237D
:10F59000B3401A400AB1012200E0002282BB4FF0C2
:10F5A0008040FFF787FE04462E462046314600285D
:10F5B00004DB4A07130E134A135406E04A07170EDA
:10F5C000114A00F00F031B1FD75400BF00BF4FF0BC
:10F5D0008040FFF76FFE0446204600280DDB00BF89
:10F5E00000BF00F01F02012191404209920002F188
:10F5F000E022C2F8001100BF00BF00BF00BF00BF83
:10F60000BDE8F08100E400E018ED00E02DE9F843EA
:10F6100007460E46384601F0E9F80446D4B14FF0EB
:10F620000008002000906846FAF7F6F8207910B13B
:10F630004FF0010802E02660012020719DF80000D3
:10F64000FAF7F0F8B8F1000F03D011252846BDE80D
:10F65000F88300BF00252846F9E770B5054628461F
:10F6600001F0C4F8044614B100202060207170BD80
:10F6700010B5044600212068FFF779FA022061796D
:10F6800001EB4101014A505410BD0000882D0020BB
:10F690002DE9F0430346164658792D4A42F820607A
:10F6A000587900EB40002B4A105C18B10824204622
:10F6B000BDE8F08393F904508F7828463A46002835
:10F6C00008DB4FEA427C4FEA1C68DFF88CC00CF87C
:10F6D00000800BE04FEA427C4FEA1C69DFF87CC0F7
:10F6E00000F00F08A8F104080CF8089000BF00BF54
:10F6F00093F90420104600280DDB00BF00BF00F086
:10F700001F070125BD404709BF0007F1E027C7F8E3
:10F71000005100BF00BF00BF00BF0A881868C0F8D2
:10F72000082500BF08795A7902EB4202094D2A44A4
:10F730005070C8785A7902EB42022A449070012036
:10F740005A7902EB4202A85400242046B0E7000098
:10F75000842D0020882D002000E400E018ED00E05A
:10F760002DE9F04104460D464FF4807601273146DD
:10F770002068FFF7CEF939462068FFF7DEF91DB1A2
:10F7800039462068FFF7E8F9BDE8F0812DE9FF4F21
:10F7900083B007460C46387900EBC0006A4901EB9C
:10F7A0008006307F28B14FF0080A504607B0BDE808
:10F7B000F08F3D683A79654B53F822103868FFF7AF
:10F7C00025FF18B14FF0110A5046EFE70598306059
:10F7D00006987060207B012803DC2078FEF7A1FBEF
:10F7E00002E02078FEF72CFC0020009001902078A9
:10F7F00000231A460121FEF7D6FA6078FF2808D0C8
:10F8000094F801904846FEF78CFB4846FEF71CFB37
:10F8100001E04FF0FF39A078FF280ED094F8028065
:10F820004FF0010B002000905B460246014601901C
:10F830004046FEF7B8FA00BF01E04FF0FF38A0786D
:10F8400086F82000E078F077E078FF280DD0207966
:10F8500018B1E078FEF765FB02E0E078FEF7F0FB18
:10F86000E078FEF7F1FA2079B0772078C5F808053E
:10F87000C5F80C95C5F8108500BFA068C5F824052B
:10F8800000BF217B627B0AB1012300E00023184600
:10F8900031B1012906D0022907D0032908D000BFC1
:10F8A00000BF08E040F0020005E040F0040002E084
:10F8B00040F0060000BF00BFC5F8540500BFA079A6
:10F8C000C5F8C00500BF00BF0720C5F8000500BF90
:10F8D000306888B33868FFF7F5FC83466179029198
:10F8E00058460299002804DB4A07130E184A13549D
:10F8F00008E04A074FEA126C164A00F00F031B1F7C
:10F9000002F803C000BF00BF3868FFF7DBFC834686
:10F91000584600280DDB00BF00BF00F01F02012188
:10F9200091404209920002F1E022C2F8001100BFAA
:10F9300000BF00BF00BF00BF0020707701203077FC
:10F940004FF0000A504631E72059002014400300D0
:10F9500000E400E018ED00E02DE9FC4105462879BF
:10F9600000EBC0002D4901EB8004206808B3286833
:10F97000FFF7A8FC06463046002817DB00F01F0200
:10F9800001219140264A430942F8231000BF00BFDD
:10F9900000BFBFF34F8F00BF00BF00BF00BF00BF5D
:10F9A00000BFBFF36F8F00BF00BF00BF00BF00BF2D
:10F9B00000BF2F68206898B11A493846FFF7C8FB86
:10F9C000607F68B114213846FFF7C5FB00BF4FF4D4
:10F9D00082713846FFF7AEFB0028F8D00020607730
:10F9E00094F82000FF280CD094F8206000200090AC
:10F9F00003460122014601903046FEF7D4F900BFCC
:10FA000000BF00BF0020C7F8000500BF2868FFF74F
:10FA100024FE00202077BDE8FC8100002059002052
:10FA200080E100E0520108002DE9F04105460E4654
:10FA30001746287900EBC000154901EB80044FF010
:10FA40000008607F20B14FF011084046BDE8F0810A
:10FA5000206820B107F0140008B90120607796E80B
:10FA60000E10C4E9053CC4E90312E07FFF2808D06A
:10FA7000A07F18B1E07FFEF7E3FA02E0E07FFEF737
:10FA800050FA3B4632462146286802F0EDFEDDE79B
:10FA90002059002000B501460248016000F004F83A
:10FAA00000BD000004E5014000BF024800680028D6
:10FAB000FBD0704700E401402CB51949194A891A56
:10FAC000C908032242EA014017A1FEF78FFD1D4835
:10FAD000002101601C481B49086000BF1B4804F05E
:10FAE00051F80546002D19D019A00D490D4A891A63
:10FAF000C9080322CDE9000542EA0140C82320A23B
:10FB000026A1FEF7ADFDFEF7E5FB00BF00BF24B167
:10FB100000BF2046F9F716FB00BF00BF00BF2CBD99
:10FB2000644F0300CC4E0300696E6974207A6461EF
:10FB300074616368616E6E656C207365727669636B
:10FB4000650000006C2C0020153B03007430002081
:10FB50007A646174616368616E6E656C5F696E6919
:10FB60007428266D5F7A6872732C20267A6461741B
:10FB7000616368616E6E6C655F696E69742900000F
:10FB80007372635C616473313239335F73696D70B2
:10FB90006C655F7465737465722E630025733A2516
:10FBA00064205A4552524F525F434845434B2825E3
:10FBB0007329206661696C3A2564000010B103283E
:10FBC00001D101E000E000BF00BF704710B504465E
:10FBD000FCF7EEFE014A03C210BD0000B82D002064
:10FBE00010B504460548006830B10448006803F0C9
:10FBF0000DF800200149086010BD0000A82D00206C
:10FC0000DCB506463078002823D13B211148008816
:10FC100076DF044600BF2746002F19D00EA01149F9
:10FC2000114A891AC9080322CDE9000742EA0140B6
:10FC300073230EA215A1FEF713FDFEF74BFB00BFC9
:10FC400000BF25B100BF2846F9F77CFA00BF00BF0E
:10FC500000BFDCBD4C2E00206572725F636F64656F
:10FC600000000000644F0300CC4E03002E2E5C6C9D
:10FC700069627A6E6F726469635C7372635C7A62E4
:10FC80006C655F6D6F64756C652E630025733A2536
:10FC900064205A4552524F525F434845434B2825F2
:10FCA0007329206661696C3A2564000070B50546C9
:10FCB000AE883046FCF7AAFE044674B14FF6FF73D7
:10FCC00040F2F31205F1080104F10A00FDF724F8EF
:10FCD000607221463046FBF7E7F870BD2DE9F04130
:10FCE0000546EF7BAE88012F01D0BDE8F0814FF6CD
:10FCF000FF70FCF78BFE04461CB9042002F026F9C5
:10FD0000F3E700BF2680002020720E480168C4F887
:10FD10000A104068C4F80E0000BF4FF6FF7340F2AF
:10FD2000F31205F1100104F10A00FCF7F5FF60720F
:10FD30000548C08918B921463046FBF7B5F800BF21
:10FD4000D3E700005C2D0020DC5700208188014AA9
:10FD500091807047187F0020CA7B012A02D18A88CF
:10FD6000A0F82424704700002DE9F04705460F460F
:10FD7000BE88A81D00EBC6042879A071F87B012875
:10FD800002D0022806D102E02888208003E068889B
:10FD9000208000E000BF00BF20886188884236DDF7
:10FDA00022882049204BC91AC908042343EA01408C
:10FDB00033461EA1FEF730FC21883046A5DF804681
:10FDC000B8F1000F02D1012060711FE0B8F1110FEE
:10FDD0000DD1012020711349134A891AC908042240
:10FDE00042EA014032462149FEF70AFC0EE0404655
:10FDF000FFF7D4F981460B490B4A891AC908012239
:10FE000042EA01404A461AA1FEF7FAFB00BFA07978
:10FE1000E179884203DDA1793046FBF799F9BDE825
:10FE2000F0870000CC4E0300CC4E03005265717584
:10FE3000657374696E6720746F2075706461746592
:10FE400020415454204D545520746F202575206254
:10FE500079746573206F6E20636F6E6E656374696D
:10FE60006F6E20307825782E000000008446030055
:10FE700073645F626C655F67617474635F65786308
:10FE800068616E67655F6D74755F726571756573C6
:10FE90007428292072657475726E65642025732E2E
:10FEA0000000000030B587B00546002003900490A4
:10FEB0000590069002208DF80C00174903C9CDE982
:10FEC000000102A80190154A518990886A46ADDF69
:10FED000044654B902A8FAF743FB30B101218DF86A
:10FEE00012100020ADF8100003E040F2FD10ADF854
:10FEF000100000BF0949888803A9B0DF0446112C0F
:10FF0000F8D0BDF8100008B107B030BD2846FAF7A8
:10FF100071F800BFF8E7000048430300187F002095
:10FF200070B58EB004460E462C22311D03A8F7F79B
:10FF300068FABDF80C50BDF81000C1B2A01D00EB6E
:10FF4000C500C171A11D01EBC501CA792749284B24
:10FF5000C91AC908042343EA01402B4625A1FEF72C
:10FF60005BFBBDF812202149214BC91AC9080423A3
:10FF700043EA01402BA1FEF743FBBDF810201B49CB
:10FF80001B4BC91AC908042343EA01402AA1FEF702
:10FF900037FBBDF816201549154BC91AC9080423AB
:10FFA00043EA014029A1FEF72BFBBDF814200F49BD
:10FFB0000F4BC91AC908042343EA014027A1FEF7E1
:10FFC0001FFB206980B1294903C9CDE90101ADF8C2
:10FFD0000650A01D00EBC500C0798DF8080001A9EE
:10FFE00020462269904700BF0EB070BDCC4E030082
:10FFF000CC4E030044617461206C656E67746820A8
:020000040003F7
:100000007570646174656420746F202575206F6E4F
:1000100020636F6E6E656374696F6E203078253073
:10002000782E00006D61785F72785F6F637465741D
:10003000733A2025750000006D61785F74785F6FFA
:1000400063746574733A2025750000006D61785FF4
:1000500072785F74696D653A202575006D61785F0F
:1000600074785F74696D653A20257500B83F0300A8
:100070002DE9F04705460E46341D2188A81D00EBEA
:10008000C10794F8048022880B490C4BC91AC9088F
:10009000042343EA0140434609A1FEF7BDFAB879BB
:1000A000404501DAB87900E040468146208849465B
:1000B000FBF74EF8BDE8F087CC4E0300CC4E0300B2
:1000C00050656572206F6E20636F6E6E6563746934
:1000D0006F6E203078257820726571756573746550
:1000E0006420612064617461206C656E67746820AF
:1000F0006F662025752062797465732E00000000FC
:100100002DE9F0410646B7883846FCF77FFC0546E6
:100110006DB16868F9F75DFB044614B1204601F043
:1001200015FF00BF4FF6FF70288000BF00BFBDE87D
:10013000F0810000054989888288914200D070478B
:100140004FF6FF71014A918000BFF8E7187F002049
:1001500070B504460E46002084F82E04B088B4F82A
:10016000241488420CD1207950B901212046F9F796
:1001700062FD054625B1A06B10B12846A16B8847EA
:1001800070BD70B504460D46AA88A11D01EBC200E2
:10019000FCF746FE70BD00002DE9FC4706460F4601
:1001A000BD88B7F80690B01D00EBC5042B492C4A5A
:1001B000891AC908042242EA01404B462A4629A16D
:1001C000FEF72AFAB9F1170F01DA172000E04846C6
:1001D00081462088484501DD484600E0208860804F
:1001E000002020710095238862881C49DFF870C0C8
:1001F000A1EB0C01C9084FF0040C4CEA014028A106
:10020000FEF71AFA21882846B5DF8046B8F1000FBC
:100210000ED04046FEF7C2FF82461049104A891AA6
:10022000C908012242EA014052462DA1FEF7E8F931
:10023000607908B1BDE8FC87306968B1344903C909
:10024000CDE90001ADF802506088ADF804006946C0
:1002500030463269904700BF00BFEBE7CC4E030049
:10026000CC4E030050656572206F6E20636F6E6E1A
:10027000656374696F6E20307825782072657175BA
:10028000657374656420616E20415454204D54554B
:10029000206F662025752062797465732E0000003A
:1002A0005570646174696E6720415454204D5455F3
:1002B00020746F2025752062797465732028646529
:1002C00073697265643A20257529206F6E20636F0B
:1002D0006E6E656374696F6E20307825782E00002D
:1002E00073645F626C655F67617474735F65786384
:1002F00068616E67655F6D74755F7265706C792893
:10030000292072657475726E65642025732E000055
:10031000B03F03002DE9FC4105460E46B788B6F80C
:100320000A80A81D00EBC7042088404501DD404637
:1003300000E0208860806088172801DA172000E03C
:100340006088608062881149114BC91AC90804236A
:1003500043EA01403B460FA1FEF75EF9286978B1F8
:10036000607968B11A4903C9CDE90001ADF802709E
:100370006088ADF80400694628462A69904700BFA6
:10038000002060712071BDE8FC810000CC4E0300AC
:10039000CC4E0300415454204D5455207570646177
:1003A00074656420746F20257520627974657320EC
:1003B0006F6E20636F6E6E656374696F6E20307848
:1003C00025782028726573706F6E7365292E000082
:1003D000A83F030070B50546AE1D30880749C9889F
:1003E00088420AD10548007E38B1F9F7CFFD0446AE
:1003F0001CB1024841690220884770BD187F002067
:100400000548D0E900304FF080729A1840F10000A2
:100410000149C1E900207047B02D002070B50546A4
:10042000A8880E498988884200D070BDAC1D20780C
:10043000022810D160880949C98888420BD1207AE6
:10044000042808D0207A062805D0207A052802D072
:10045000A01CFFF727FD00BFE7E70000187F002082
:100460002DE9F04104460D462888262801D0BDE834
:10047000F081287A012802D0287A02280ED1A078AB
:10048000F8F7C4FD074639462046F9F7D4FB06467F
:1004900026B1A06B10B13046A16B884700BFE6E7DC
:1004A0002DE9F0410446A51D28881249C9898842D2
:1004B0001DD1688902281AD1B4F804804046FCF79F
:1004C000A5FA064696B105F10C00FAF752F820B1EC
:1004D00031464046FAF7E8FC08E07068F9F779F928
:1004E000074617B1384601F031FD00BF00BFBDE837
:1004F000F0810000DC570020FEB504460E46B51D15
:1005000000200090019002902988208981420FD11B
:10051000688902280CD105F10C00FAF72AF818B105
:10052000012084F8220029E0002084F8220025E040
:100530002988208B81420FD1688902280CD105F1CE
:100540000C00FAF716F818B1012084F8230015E022
:10055000002084F8230011E02888A18988420DD169
:10056000E06958B100208DF8000005F10C00019001
:100570006989ADF808106846E1698847FEBD014603
:100580000868012805D00868022802D008680428F5
:1005900001D1012070470020FCE7000070B5024641
:1005A00005490B46D40802F007021D5D012696405E
:1005B00035431D5500BF70BDE65800200146054873
:1005C0004056012202EBE07008B101207047002084
:1005D000FCE70000B85800200146044840560828AF
:1005E00001DB012070470020FCE70000B858002024
:1005F000014606484056002805DB044840560828B6
:1006000001DA012070470020FCE70000B858002004
:10061000FF2201490A547047B85800202DE9F84FCD
:10062000814600BF00244FE02C480057401C00B911
:1006300049E0204600F054F8054649462846FCF7B4
:10064000EBFF00283ED0204600F052F80646009509
:100650006846FDF793FC83460BF5E060009950F87F
:100660002100C0F301408046B8F1020F01D1032000
:1006700000E00220824651462846FDF70EFC009518
:100680006846FDF77BFC8346012000998840CBF843
:10069000200500BF2846FAF7F5F98346FAF7AAF9CC
:1006A000074677B1032E09D0B8F1020F01D1012E10
:1006B00004D0B8F1030F04D1022E02D131462846EE
:1006C000B84700BF00BF641C042CADD34846FCF7FC
:1006D00062FB0028A6D1BDE8F88F0000E258002098
:1006E00001460248425C22F0C0007047E2580020F8
:1006F00001460248425C900970470000E258002021
:1007000070B504460D461646207A05280CD0607A4E
:1007100028B10A480AA102682846FDF70FFA09A184
:100720002846FDF70BFA04E01EB106A12846FDF7A6
:1007300005FA2846FDF717FA70BD0000102E0020BC
:10074000257300000D0A0000F8B504460D46E08848
:1007500038B116A00090E38816A218A12846FDF72C
:10076000EDF9207A05281FD0607A58B1217AA08847
:10077000FDF780FD174951F82060324616A1284642
:10078000FDF7DCF92846216802F01EFBA088002155
:10079000FEF708F80646207A104951F82020334623
:1007A0000FA12846FDF7CAF9F8BD00001B5B306DAC
:1007B000000000001B5B313B33316D0025734C6F33
:1007C00067732064726F7070656420282564292522
:1007D000730D0A00102E002025730000FC2D002050
:1007E0003C25733E2025733A200000000146034853
:1007F000814201D1024870470020FCE70020004000
:100800006C2D00202DE9F04107460D4616463C4868
:10081000007808B9BDE8F0813A4C6520A07000204E
:10082000607003202070C4F8037000205AE000EBD1
:10083000400115F8213000EBC001E21D535400EBDC
:10084000400135F82110C1F3072300EBC001491C1A
:10085000535400EB400155F82110C1F3074300EB5E
:10086000C001891C535400EB400105EB81010B7959
:1008700000EBC001C91C535400EB400105EB8101A2
:100880008988C1F3072300EBC001091D535400EB15
:10089000400105EB81014968C1F3074300EBC0014A
:1008A000491D535400EB400105EB81010B7A00EB2D
:1008B000C001891D535400EB400105EB81010989FA
:1008C000C1F3072300EBC001C91D535400EB4001E5
:1008D00005EB81018968C1F3074300EBC0010831D2
:1008E0005354401CB042A2DB06EBC600C01D1FFAE9
:1008F00080F84146034803F03EF900BF8AE7000054
:10090000812C00201C50002070B5064C6820A0707F
:10091000002060700320207003252946204603F044
:100920002AF970BD1C5000202DE9F04105460E4605
:10093000074C6920A0700020607003202070E570D3
:10094000267105273946204603F015F9BDE8F081E8
:100950001C5000202DE9F04704460D4616464FF086
:100960000209022D74D36069A84271D92078012848
:1009700004D0022849D003280DD15EE02F4607EBB2
:100980005707206A00EB57212046FCF701FC8146FF
:10099000B9F1000F00D075E038467F1CC0F30801A4
:1009A00004F1300001EB000805F0010028B1F1B2BC
:1009B00098F8000061F31F1000E0304688F800004E
:1009C0000120E070206A00EB57212046FCF7E0FB95
:1009D0008146B9F1000F00D054E0C7F3080104F1DB
:1009E000300001EB000805F0010010B1C6F307105C
:1009F00006E098F8000000F0F000C6F30321084379
:100A000088F800000120E0703CE0206A00EB15212E
:100A10002046FCF7BDFB8146B9F1000F00D031E064
:100A2000B1B240F2FF1202EA450304F13002981815
:100A300001F0C0FF0120E07024E0206A00EBD51136
:100A40002046FCF7A5FB8146B9F1000F01D019E063
:100A500019E040F2FF1101EA850204F1300150185B
:100A6000FCF7BFF966F31B00064640F2FF1101EAEE
:100A7000850204F130015018314601F08FFF01204A
:100A8000E07000BF00BF4846BDE8F087024800683C
:100A9000810201F1005070470C01001010B586B0C2
:100AA000694630A0FBF7B3FB044630483049086084
:100AB000002C4ED1BDF80400BC2101EB6020A0F554
:100AC000FA602C490870BDF80400C0F34310487068
:100AD000BDF8040000F01F008870BDF80600C012C9
:100AE000C870BDF80600C0F345100871BDF80600D7
:100AF000C006800E48711E4800680A680260496896
:100B000041601B4900980968C86001201849486085
:100B100019491A4A891AC908032242EA014018A150
:100B2000FDF764FD1449154A891AC908032242EAEF
:100B300001400CA215A1FDF763FD0F490F4BC91A27
:100B4000C908032343EA014013A1009AFDF758FDA9
:100B500005E0002006490968C8600549486006B0FC
:100B600010BD0000302E62696E0000001455002098
:100B7000F02C0020F92C0020644F0300CC4E030021
:100B800066696C656C6973743A000000206E616D73
:100B9000653A2573000000002073697A653A256480
:100BA0000000000010B50446142C01DB002010BD2D
:100BB00021460548FCF764FC21460348001FFCF76A
:100BC0005FFC0120F3E700000058002070B50546E7
:100BD000002406E0044901EB84002946FCF732FCBE
:100BE000641C1E2CF6D370BDFC57002010B598B0C5
:100BF0000F488068C04317900D48416817A8FCF75C
:100C000067FC179901A8FAF7C7F82C2201A90CA8CC
:100C1000F6F7F7FB002405E00DA931F81400FFF703
:100C2000D5FF641C0C98A042F6D818B010BD000087
:100C3000F857002010B5044621460248FCF702FC94
:100C400010BD0000005800202DE9F04781460E46F7
:100C500017464FF00008D9F80040022E02D3606911
:100C6000B04202D80220BDE8F08767B100BF4FF064
:100C7000FF3239462046FFF76DFE8046B8F1000F7F
:100C800001D04046EFE700BF31464846FBF794FDF0
:100C9000054605B922E0012D01D10220E3E7681CD9
:100CA00008B90120DFE7002231462046FFF752FE57
:100CB0008046B8F1000F01D04046D4E7D4E90410D3
:100CC000801E814206D22069401C2061207940F0BC
:100CD000010020712E466069B042D5D800BF0020C7
:100CE000C1E70000042804D102490968491C014AEF
:100CF00011607047402E002010B504462046FAF7D8
:100D000078FF08B1FFF77CFB00212046FAF781FE4F
:100D100010B12046FEF764FF01212046FAF779FE64
:100D200010B12046FEF752FF204601F0E1FF2046B9
:100D300000F044F810BD00002DE9F05F83468846BE
:100D40004FF00D09002088F80000DBE90267FBF78F
:100D50002FFE341A67EB010500210846091BA84144
:100D60001ADAB4F5350F05D3F8F7B2FC1149084487
:100D7000002101E03046394682464FF49603524640
:100D800000210D48FAF74BFF8146B9F1000F02D15F
:100D90000120BDE8F09F03E000210748FAF72EFE8E
:100DA000B9F10D0F04D1584601F030FF88F800006A
:100DB0000020EEE7FFFFB400A02D0020F8B50746A5
:100DC00055E000BF2B48FEF792F906460EB13046BB
:100DD00000E0002004460025002C40D06B1ED4E922
:100DE000021059405840014302D101F0D9FB3EE0C6
:100DF0002148006808B9012517E01F49D4E90230ED
:100E00000A68D2E90212591A90410ED201251A48F5
:100E10000068D0E90210AA1E51405040014304D09E
:100E2000154801681348FEF74EF9BDB101F0B8FB53
:100E3000044669462046FFF77FFF58B10E48006818
:100E400010B93846FAF7DDFE0B4804609DF8000043
:100E500018B90DE000200849086007E008E00648DE
:100E6000006810B93846FAF7D3FE01E000BFA8E7E2
:100E700000BFF8BD4C400300A82D002070B504460B
:100E80000E462546D5E90010884770BD10B50446CA
:100E90002046F7F711FE10B942F2010010BD2046BE
:100EA000002803DB1F4A125C520905E01E4A00F0CD
:100EB0000F031B1FD25C52091146082904D20120DE
:100EC000884000F0EC0008B9002000E0012010B9D3
:100ED00042F20200E2E71548806868B160091349F0
:100EE00051F8200004F01F020121914008436109DC
:100EF0000E4A42F8210012E0204600280DDB00BF18
:100F000000BF00F01F02012191404209920002F14E
:100F1000E022C2F8001100BF00BF00BF00BF0020E8
:100F2000BCE7000000E400E018ED00E0945A002067
:100F300070B50446F7F7DCFD054614488068D8B95B
:100F400001201249886012480068124908400F4980
:100F5000086010484FF0E021C1F880010C4880384B
:100F6000D0F88400094948604FF0FF310848001D5F
:100F700001600020207001E0012020701DB900BF39
:100F800062B600BF00BF002070BD0000945A002070
:100F900080E100E0FC06FFBD38B504460D4624B1F3
:100FA000012C1FD0032C38D132E00020002817DBA1
:100FB00000F01F0201219140194A430942F8231011
:100FC00000BF00BF00BFBFF34F8F00BF00BF00BF17
:100FD00000BF00BF00BFBFF36F8F00BF00BF00BFE7
:100FE00000BF1BE0002000906846F8F715FC0D4894
:100FF000007808B9FCF7EEFC0A48C068401C0949B3
:10100000C860012088709DF80000F8F70BFC05E02F
:10101000FEF714F9FCF704FD00E000BF00BF38BD87
:1010200080E100E07458002070B501460878821114
:1010300022B1012A1CD0022A26D100E000BF087A82
:101040008009CE7900EB86008E7906F0030600EB6E
:101050008623487900F00F04887AC0094E7A06F09A
:10106000030600EB46056019C61F581CB04070BD52
:10107000487A0C7A00EB0420CC7904F03F0400EBB2
:101080000443581C8002F2E700BF00BF0020EEE7D7
:101090002DE9F04705460E4690463A4890F8230061
:1010A00010B11120BDE8F08700240121354880F8F7
:1010B000231005F08000A8B106240221314880F8F1
:1010C000231077202F4981F8280000212D4880F82F
:1010D000291080F82A1080F82B1080F82C10FF219E
:1010E00080F82D1005F07F01264828300155320E7A
:1010F000601C244928310A54C6F30742A01C0A5434
:10110000C6F30722E01C0A54201D0E54402D02D0C5
:10111000482D04D101E0952703E0872701E0FF2750
:1011200000BF00BF601D174928310F54B8F1020FEE
:1011300003D0B8F1030F0AD104E00521114880F86B
:10114000241009E005210F4880F8241004E0012153
:101150000C4880F8241000BF00BF05F0800008B1E3
:10116000012002E0074890F82400814609F10E00B2
:10117000C3B2044A38320621A2F1100000F054FE36
:1011800000208FE7AC5A00202DE9FE430546687821
:101190004249087042480668B469287820B101289D
:1011A00034D002286CD14CE0687880B1B146484612
:1011B000F9F7B6FA074600BFB846B8F1000F04D0F9
:1011C00000BF4046F7F7BEFF00BF00BF00BFF8F703
:1011D00071F9006820604FF400706060304800686A
:1011E0008069806888B10020009001900290687842
:1011F00008B1012000E000208DF80100A0690290F4
:1012000069463046A268904700BF43E02448006822
:1012100080698068A0B1234A07CA8DE80700687812
:1012200008B1012000E000208DF8010004F10C005D
:101230000190A069029069463046A268904700BFBD
:1012400028E01748006880698068C0B1154A0C32F0
:10125000D2E900109268CDE901020091687808B1E6
:10126000012000E000208DF8010004F10C00019045
:10127000A069029069463046A268904700BF09E025
:1012800000BF032700BF0320F7F75CFF00BF00BFCC
:10129000BDE8FE8300BF00BFFAE70000DC2D0020A0
:1012A000E02D0020F04103002DE9FC5F80468946D7
:1012B000154698F8006098F80100000698F80210AA
:1012C00040EA014098F8031040EA012098F8041021
:1012D00040EA010B0127FE48808BB0F50E7F7DD0E0
:1012E00010DC40F21322A0EB0201904252D004DC49
:1012F000D0B1B0F5047F72D12FE006297AD013293E
:10130000F9D1BAE040F26122811A904269D006DC3C
:10131000A0F24D20002870D00628ECD174E10A29F3
:101320006CD00F29E7D1FEE12BE201220021402001
:10133000FFF7AEFE044600BFA246BAF1000F04D08C
:1013400000BF5046F7F7FEFE00BF00BF00BF0027FA
:101350004FF40471DE48818300BF17B90120BDE856
:10136000FC9F00BF012200214020FFF791FE0446B0
:1013700000BFA246BAF1000F04D000BF5046F7F7F5
:10138000E1FE00BF00BF00BF002740F21321D0489C
:10139000818300BF0FB90120E1E700BF00BF26F045
:1013A000030040B100BF0420287000BF0021C848DE
:1013B00081830220D3E700BF03224FF4D571482078
:1013C000FFF766FE044600BFA246BAF1000F04D044
:1013D00000BF5046F7F7B6FE00BF03E089E0D1E159
:1013E00008E04BE100BF00BF002740F21921B848D8
:1013F000818300BF1FB90120B1E7D7E072E100BFD0
:1014000006F00400A0B9B248807A20F00700C01CA2
:10141000AF49887200BF26F0030040B100BF04202E
:10142000287000BF0021AA488183022097E700BFEF
:101430000021A7480184807A00F00700032802D128
:101440004FF0804000E0002001900222E920019945
:10145000FFF71EFE044600BFA246BAF1000F04D0FB
:1014600000BF5046F7F76EFE00BF00BF00BF002769
:1014700040F226219648818300BF0FB901206EE714
:1014800000BF06F00400B8B39148807A20F007004E
:10149000401C8F49887226F0040600BF8C48008CDF
:1014A000401C81B28A480184008CB0F5FA6F08DDD7
:1014B00000BF0220287000BF0021854881830220E0
:1014C0004DE7022200214120FFF7E2FD044600BF64
:1014D000A246BAF1000F04D000BF5046F7F732FE23
:1014E00000BF00BF00BF00274FF40E717848818312
:1014F00000BF17B9012032E713E000BF00BF26F09C
:10150000030040B100BF0420287000BF00217048D4
:101510008183022023E700BF06F001000028BDD12F
:101520008EE000BF26F0030040B100BF0420287009
:1015300000BF002166488183022010E700BF47E01A
:101540006348008C401C81B261480184008CB0F576
:10155000FA6F08DD00BF0220287000BF00215C4840
:1015600081830220FBE65A48807A00F007000328B6
:1015700002D14FF0804000E0002001900222E920DB
:101580000199FFF785FD044600BFA246BAF1000F9E
:1015900004D000BF5046F7F7D5FD00BF00BF00BF25
:1015A000002740F24D214A48818300BF0FB9012036
:1015B000D5E600BF00BF26F0030040B100BF042005
:1015C000287000BF0021424881830220C7E600BF87
:1015D00006F001000028B3D1022200217A20FFF793
:1015E00057FD044600BFA246BAF1000F04D000BF69
:1015F0005046F7F7A7FD00BF00BF00BF002740F22D
:1016000053213348818300BF0FB90120A7E600BFF3
:1016100000BF26F0030040B100BF0420287000BFC7
:1016200000212B488183022099E600BF0BF0804007
:1016300030B12748807A20F00800083024498872A9
:101640002348807A00F00700032829D001225102A4
:101650005020FFF71DFD044600BFA246BAF1000F5F
:1016600004D000BF5046F7F76DFD00BF00BF00BFBC
:10167000002740F261211648818300BF0FB9012085
:101680006DE600BF00BF26F0030040B100BF04209C
:10169000287000BF00210E48818302205FE600BF52
:1016A0000B4848300A49C86001214838818201222C
:1016B00000214920FFF7ECFC044600BFA246BAF126
:1016C000000F04D000BF5046F7F73CFD00BF01E01B
:1016D000AC5A002000BF00BF002740F26B212C480D
:1016E000818300BF0FB9012039E600BF00BF26F09B
:1016F000030040B100BF0420287000BF002124482F
:10170000818302202BE600BF08F10108A9F1010046
:1017100000F0FF0900BF00211D48C18300BF4FF446
:101720001C71818300BF6B4610224946404600F081
:10173000B3F8022801DA002011E600BF00BF00BFA5
:101740009DF8000048B100BF9DF80000287000BF60
:1017500000210F488183022001E600BF0C48483079
:10176000FFF762FC0A4948604FF4007108480181A4
:1017700000BF0020287000BF00210548818302209F
:10178000EDE5D2E500270021014881830320E6E54D
:10179000AC5A00202DE9F84F06460F4614464FF08C
:1017A000010A3C48808B38B1B0F5267F22D0A0F2E8
:1017B000A220002867D156E064E096F8008000BFC0
:1017C00028F0030048B100BF0420207000BF0021B2
:1017D000304881830220BDE8F88F00BF761C781E58
:1017E000C7B200BF00212B48C18300BF4FF4267150
:1017F000818300BF6B464FF400723946304600F0DB
:101800004BF8022801DA0020E5E700BF00BF00BF67
:101810009DF8000048B100BF9DF80000207000BF97
:1018200000211C4881830220D5E700BF1948808A27
:1018300001281EDD012200214C20FFF729FC05466E
:1018400000BFA946B9F1000F04D000BF4846F7F722
:1018500079FC00BF00BF00BF4FF0000A40F2A22198
:101860000C48818300BFBAF1000F01D10120B2E71B
:1018700000BF00BF0020207000BF00210548818309
:101880000220A8E799E74FF0000A00210148818370
:101890000320A0E7AC5A00202DE9F04704460D468E
:1018A00016461F464FF001088448C08B40F2D912FB
:1018B000811A90427AD005DC48B1A0F2C710002806
:1018C00075D16EE0072973D01329F9D1DBE0ECE084
:1018D0007A48818AC182BDE0002178480184FF20D6
:1018E000764981F82800002174480183032180F89B
:1018F00023105FE07148008C401C81B26F48018466
:10190000008C44F62061884209DD00BF0220387057
:1019100000BF00216948C1830220BDE8F08702E0D2
:10192000641C681EC5B215B12078FF28F8D045B3F5
:101930002078FE281CD1641C681EC5B204225F48B2
:1019400080F82320B54201DD304600E028460146FC
:10195000002004E0225C594BDB681A54401C88428A
:10196000F8D356480183C0680844544AD06021E047
:1019700000BF0520387000BF00215048C1830220FD
:10198000CBE710234D4A38320121A2F1100000F0BC
:101990004BFA00BF4FF0000840F2C7114748C1831F
:1019A00000BFB8F1000F04D10120B6E72CE07DE0C4
:1019B00049E000BF414890F8230003289AD029E06D
:1019C0003E48008B301A1FFA80F9B9F1F00F01DDA3
:1019D0004FF0F00909F0FF0338480121C2682830B0
:1019E00000F022FA3548C06848443449C8600846C7
:1019F000008B484481B23148018300BF4FF000089A
:101A000040F2D911C18300BFB8F1000F01D101200C
:101A100083E700BF2948008BB042D1DB2748C08A4A
:101A2000401E81B22548C182022300F13802012103
:101A3000283000F0F9F900BF4FF000084FF4F071C2
:101A40001E48C18300BFB8F1000F01D1012064E737
:101A500000BF00251948C08A00287FF43DAFFF2051
:101A6000164981F82800022301F138020121A2F170
:101A7000100000F0D9F900BF4FF000084FF4F671E4
:101A80000E48C18300BFB8F1000F01D1012044E727
:101A900000BF0021094880F8231000BF00203870E3
:101AA00000BF0648C183022037E711E74FF0000866
:101AB00000210248C18303202FE70000AC5A002018
:101AC0002DE9F0470646884614460125D548808B07
:101AD000B0F53B7F70D009DC88B1A0F2C3200028AC
:101AE00042D010287DD0212868D1A3E0A0F20A308E
:101AF000002879D0162878D02628F5D16CE18AE123
:101B000096F800A000BF2AF0030048B100BF0420EF
:101B1000207000BF0021C34881830220BDE8F08708
:101B200000BFC048807A00F00700012830D0BD48CF
:101B3000808A01282CDDBB48012201695920FFF76A
:101B4000A7FA074600BFB946B9F1000F04D000BF9D
:101B50004846F7F7F7FA00BF00BF00BF002540F284
:101B6000C321B048818300BF0DB90120D6E700BF73
:101B700096F800A000BF2AF0030040B100BF042087
:101B8000207000BF0021A74881830220C6E700BF64
:101B9000A448818AC182D2E00021A24801830421A5
:101BA00080F82310FF209F4981F828000846808A8A
:101BB000012804DDFC2103E05DE012E02CE1FE21C0
:101BC000984880F82910022300F13802194628307D
:101BD00000F02AF900BF002540F2D321914881830B
:101BE00000BF1DB9012099E78DE0C7E000BF25E0E7
:101BF0008C48008BC0F500701FFA80F9B9F1F00F26
:101C000001DD4FF0F009874AD368128B981809F06C
:101C1000FF010123834A383200F006F98148008B26
:101C2000484481B27F48018300BF00254FF43971D9
:101C3000818300BF0DB9012070E700BF7948008B98
:101C4000B0F5007FD4DB7748C06800F500707549B7
:101C5000C8600321734880F82310032300F1380281
:101C60000121283000F0E0F800BF00254FF43B715F
:101C70006C48818300BF0DB901204FE700BF694860
:101C800090F83A0000F01F01052915D00B2901D06A
:101C90000D2908D100BF0520207000BF0022614837
:101CA000828302203AE700BF0420207000BF002298
:101CB0005C488283022031E700215A48018433E0E6
:101CC0005848008C401C81B256480184008C44F670
:101CD0002061884208DD00BF0220207000BF002183
:101CE00050488183022019E710234E4A38320121DF
:101CF000A2F1100000F098F800BF002540F20A3170
:101D00004848818300BF0DB9012007E700BF0020CC
:101D100007E0315C21B10022424981F8232002E032
:101D2000401C4045F5D300BF3E4890F823000328EF
:101D3000C6D03C48C08A401E81B23A48C182394868
:101D4000C08A00287FF428AF3648808A012859DDF0
:101D5000FF20344981F82800FD21324880F82910FD
:101D6000032300F138020221283000F05DF800BFA3
:101D700000254FF448712B48818300BF0DB9012025
:101D8000CCE600BF002127480184032180F82310FE
:101D900033E02448008C401C81B222480184008C2E
:101DA00044F62061884208DD00BF0220207000BF99
:101DB00000211C4881830220B0E61023194A3832E2
:101DC0000121A2F1100000F02FF800BF00254FF410
:101DD0004C711448818300BF0DB901209EE600BFFD
:101DE000002007E0315C21B100220E4981F8232058
:101DF00002E0401C4045F5D300BF0A4890F823009C
:101E00000328C6D000BF0020207000BF0021054875
:101E10008183022082E673E6002500210148818348
:101E200003207BE6AC5A00202DE9F84305460E4618
:101E30001746984600BF134890F85800009068462F
:101E4000FCF7BCF881460121009A01FA02F0C9F8BA
:101E50000C0500BF00BF00BF3B46324629460A487A
:101E6000CDF80080FBF751FE044600BFA146B9F152
:101E7000000F04D000BF4846F7F764F900BF00BF69
:101E8000BDE8F883AC5A00203842030010B501E0E9
:101E900001F037FCF7F7FEFA0028F9D110BD000079
:101EA000FEB505460C496846FDF7D5F80DE06846D5
:101EB000FDF7CEF80446266828466168B04708B9A1
:101EC0001120FEBD6846FDF7E7F86846FDF7C0F84B
:101ED0000028ECD100BFF4E794420300FEB50546AC
:101EE0000A496846FDF7B7F80AE06846FDF7B0F81A
:101EF0000446266828466168B0476846FDF7CCF876
:101F00006846FDF7A5F80028EFD1FEBDB0420300FA
:101F100070B504460D46A1200B4908700120487099
:101F200008462168C0F80210A188C180A179017219
:101F3000093029680160A9888180A97981711021FF
:101F4000093801F011FE70BD9C31002010B5044627
:101F50000348806918B1024881692046884710BD4E
:101F6000DC57002070B505460E463146284675DF21
:101F7000044624B1112C02D02046FFF7E7FF0CB92C
:101F8000012070BD0020FCE72DE9F84F884615467A
:101F9000002D35D04FF000090A20009000BF08EB5B
:101FA00009012A460020F6F77FFA0446A1442D1BBA
:101FB000FCB91448007800B920E0012606B90FE00A
:101FC00000BF4FF47A7707B906E0DFF83CA04FEA8C
:101FD000871B5846D04700BF701E061EF1D100BFB8
:101FE0000098401E0090009818B90020054908701C
:101FF00004E0012003490870002DD0D100BF00BFCC
:10200000BDE8F88FE42D0020714203002DE9F04770
:1020100007460E4614469A46B86A10B90720BDE82E
:10202000F0874FF0000836E008EB4801B86A00EB93
:102030008105A88800F10209B9F1FE0F01D90C2031
:10204000EDE709F10100218870542088401C2080B0
:102050001620218870542088401C208022889119E5
:10206000288801F0F2F9218808442080A8880028F7
:102070000DDDA86808B90720D1E7AA882388981938
:10208000A968F5F7BEF92088A9880844208008F1DE
:10209000010000F0FF0897F82C004045C4DC002048
:1020A000BDE70246022082F8310092F8240010B108
:1020B0000720087001E003200870108A8881002042
:1020C000C2F8200402F226404860D06888600020F0
:1020D00070470246012082F831000020C2F8200437
:1020E00002F22640486000208860022008708020AC
:1020F00088810020704770B504460D466069A8606D
:10210000208BA88194F8240018B1062084F83C00A4
:1021100002E0012084F83C00204601F033FA78B157
:102120000220287504212046FAF79DFA064600BFD2
:10213000304600B170BD00BF052084F8310002E0D8
:10214000032084F8310004F58260C4F820040020E4
:10215000F0E770B504460D46E069A860208CA881C0
:1021600094F8240018B1062084F83C0002E0012015
:1021700084F83C00204601F005FA78B10220287569
:1021800004212046FAF76FFA064600BF304600B138
:1021900070BD00BF062084F8310002E0042084F8FE
:1021A000310004F58260C4F820040020F0E700004C
:1021B00070B5054611480068407E08B1062070BD24
:1021C00000BF0F4800F10801026828469047044606
:1021D00000BF24B901200949096848760BE00F2C9B
:1021E00009D10849084A891AC908012242EA01406E
:1021F0000649FCF7FBF92046E1E700006C2E0020C1
:10220000347F0020644F0300CC4E0300FC4C0300DD
:1022100000BF0A7822F00F020A700A7822F0F0025A
:102220000A7000BF062850D2DFE800F0030E1B281A
:10223000354200BF0A7822F00F020A700A7822F0B5
:10224000F0020A7000BF40E000BF0A7822F00F02DF
:10225000521C0A700A7822F0F00210320A7000BF95
:1022600033E000BF0A7822F00F02521C0A700A788D
:1022700022F0F00220320A7000BF26E000BF0A7888
:1022800022F00F02521C0A700A7822F0F00230325B
:102290000A7000BF19E000BF0A7822F00F02921CFA
:1022A0000A700A7822F0F00210320A7000BF0CE0C7
:1022B00000BF0A7822F00F02921C0A700A7822F0FE
:1022C000F00220320A7000BF00BF00BF704700005C
:1022D0000EB501F0A5FBF6F78DF9F6F76BF9F6F7F9
:1022E00019FCF6F745F94548F6F75AFE03211F2079
:1022F000FBF78DFD03211F20FBF789FD00BFFDF7D4
:10230000B7F80546002D1AD03DA04249424A891A25
:10231000C9080322CDE9000542EA01404FF4A87341
:102320003EA245A1FCF79CF9FBF7D4FF00BF00BF1C
:1023300024B100BF2046F6F705FF00BF00BF00BF75
:1023400045480068029003208DF8090002208DF8AE
:10235000080000BF414A02A91F20FDF70DF80546FD
:10236000D5B13F482B492C4A891AC9080322CDE927
:10237000000542EA01404FF4AA7328A22EA1FCF7FF
:102380006FF9FBF7A7FF00BF00BF24B100BF2046D5
:10239000F6F7D8FE00BF00BF00BF01211F20FCF7E9
:1023A00095FF29E0F6F766FFFBF794FFFAF71EFBAF
:1023B00008B1012000E00020054601F01DFD0446A3
:1023C00028480068A04216D02648046001F008FDA5
:1023D00006461049104A891AC908032242EA0140F8
:1023E000214932460B6821A1FCF716F9F8F7E2FA09
:1023F00000201D49086000BFD4E70000B82B002072
:102400006E7266785F6770696F74655F696E697414
:1024100028290000644F0300CC4E03007372635CF4
:10242000616473313239335F73696D706C655F74E9
:1024300065737465722E630025733A2564205A45CE
:1024400052524F525F434845434B2825732920661B
:1024500061696C3A25640000743F0300098E020034
:10246000E84303007C2C0020542C002025642063CA
:1024700068616E6765636F756E743A25640A000063
:1024800010B50CE000BF2C48806804462B4800784B
:102490002168884700B910BD2748FCF7FDFD00BF43
:1024A000254880680028EDD100BFFCF78DF900BFFA
:1024B00000BFFBF70FFF0028FBD100BF00BF1F4884
:1024C0000078032803D01D48007802281DD100BFE2
:1024D00000BF00BF00BF00BFBFF34F8F00BF00BFF2
:1024E00000BF1748006800F4E06016490843001D6B
:1024F0001349086000BF00BF00BFBFF34F8F00BF8C
:1025000000BF00BF00BF00BFFDE7FCF771FD10B1C9
:1025100033DF044600BF00BF01200B49086000BF45
:1025200000BF00BF00BFBFF34F8F00BF00BF00BFA1
:1025300000E020BFFDE70000A05A0020D02D0020C1
:102540000CED00E00000FA050005004070B50446FF
:102550000D462CB90120034948700020F8F7C4FB50
:1025600070BD00007458002070B51620FEF78EFC78
:10257000044600BF254625B100BF2846F6F7E2FD18
:1025800000BF00BF70BD10B500BF00F009F818B162
:102590004FF0FF328260C2600028F6D110BD00000B
:1025A00010B50448FCF7A7FD04460CB1204610BD49
:1025B0000020FCE74C4003002DE9FE430646884618
:1025C000F468357C9648C08A30B900BF944991F8C8
:1025D0005800FBF742FD00BF914890F82300022805
:1025E00004D08F4890F8230001287DD1A81FC5B2E0
:1025F000A41D706800784C2803D115B1681EC5B2BF
:10260000641C02E0681EC5B2641C15B12078FF2866
:10261000F8D045B9706800784C2803D1681CC5B261
:10262000641E00E00024002C49D17D4890F822006F
:10263000012844D001208DF80100794890F822004B
:10264000012806D0022805D0042816D005281CD160
:1026500017E000BF00208DF800000321704880F8CB
:10266000221000BFF6F7B4FF074627B100BF384677
:10267000F6F768FD00BF00BF10E001208DF80000F4
:102680000CE002208DF8000008E000BF032700BF27
:102690000320F6F757FD00BF00BF00BF00BF00BF1B
:1026A0005F4991F85800FBF7D8FC00BF03215C4854
:1026B00080F82210016868468847BDE8FE835848C4
:1026C00090F82300022817D10121554880F82310E3
:1026D000277827F0010070B9514890F824000E3097
:1026E000C3B24F4A383200E00AE00621A2F10A00E4
:1026F000FFF79AFBE1E700BF0021494880F823106B
:1027000006200290464890F82200012806D00228B0
:102710000BD0042830D0052875D150E00221404864
:1027200080F822100021818300BF02AA294620469A
:10273000FEF7BAFD02281EDB00208DF804009DF88C
:1027400008008DF805000321354880F8221000BFED
:10275000014691F85800FBF780FC00BF00BF314AEA
:102760004FF080415068C0F8241500BF00BF2C48CE
:10277000016801A888474FE002AA29462046FFF7D2
:1027800009F802281ADB01208DF804009DF80800E2
:102790008DF805000321224880F822100021818253
:1027A000C18280F8231000BF014691F85800FBF762
:1027B00054FC00BF1A48016801A888472CE002AA0F
:1027C00029462046FFF77CF902281ADB02208DF803
:1027D00004009DF808008DF805000321104880F8DA
:1027E0002210002180F823108182C18200BF01469F
:1027F00091F85800FBF731FC00BF0948016801A8B7
:10280000884709E0FFE700BF032700BF0320F6F772
:1028100099FC00BF00BF00BF00BF00BF4DE7000034
:10282000AC5A00203842030070B586B004460D460D
:102830002E4620788DF8040060680290217A8DF889
:102840000C10E1680491217C8DF81410044850F8B4
:102850002610044850F8262001A8904706B070BD05
:1028600078590020685900202DE9F04704460E46AB
:1028700015461F46286818B12868FCF765FE28B180
:10288000A86850B1A868FCF75FFE30B900207077E7
:102890004FF010084046BDE8F087D5E90001C4F8C4
:1028A00044054FF4A962115100BFD5E90201C4F8F3
:1028B00034054FF4A762115100BF4FF48C712046CC
:1028C000FCF73FFC2046394601F0010232B100BF5F
:1028D00001234FF4AA62135000BF06E000BF00239B
:1028E0004FF4AA62135000BF00BF01F0020232B1E0
:1028F00000BF01234FF4A862135000BF06E000BFE1
:1029000000234FF4A862135000BF00BF00BF07F0C0
:10291000080018B910212046FCF71DFC3068A0B94A
:1029200000BF4FF48C712046FCF704FC0028F8D05F
:10293000F07FFF281CD0B07F18B1F07FFBF7F1FAD1
:1029400016E0F07FFBF77CFB12E0A146012020EAB5
:10295000970ABAF1000F04D140214846FCF7F8FB72
:1029600004E04020C9F8040300BF00BF00BF00BF5F
:102970004FF0000840468EE770B506460C461546F7
:10298000A9B204F11A0000F015F83078032804D138
:10299000290C04F1140000F00DF870BD00F8011BC3
:1029A000090A00F8011B090A00F8011B090A00F8CE
:1029B000011B704700F8011B091200F8011B70474A
:1029C0002DE9F05F05460E4690461F46DDF828903B
:1029D0004FEA154AF9F706F883464AEA0B42781C93
:1029E00000EA09000E4941F8202007EA090001EB3E
:1029F0008004206865F3C5002060206868F38910B2
:102A00002060206866F39F202060206820F003008B
:102A1000401C2060206820F004002060BDE8F09F8A
:102A2000346800202DE9FC478046894616461C463E
:102A30001C480768012201A92046F7F715FFC0B11D
:102A4000019800F1020A002509E056F825205046B9
:102A50000AF1010A3840144941F820206D1CA542B2
:102A6000F3D30097224649464046019BFFF7A8FF53
:102A700000BF0D480C38007880B1002000906846F7
:102A8000F6F7CAFE00BF00BFFBF724FC0028FBD10D
:102A900000BF9DF80000F6F7C5FE00BFFAF7CBF9BE
:102AA000BDE8FC87F82D0020346800202DE9F047B0
:102AB00081460C4615469846002608F00100A0B154
:102AC00005E0641C761C39464846F7F741FF277835
:102AD000002FF6D104E06D1E20214846F7F738FF9D
:102AE000B5421BD9002DF6D118E01CB12046F4F7F1
:102AF000ACFC064604E06D1E20214846F7F728FF8F
:102B0000B54201D9002DF6D105E0641C761C39468A
:102B10004846F7F71DFF2778002FF6D1BDE8F0876C
:102B200070B50446204600F043F80546002D38D124
:102B3000207803282ED1207901282BD142020021B0
:102B400004F13000FAF79AFA4AF6552104F22E20E1
:102B5000FFF730FF144904F13000FFF71FFF13495E
:102B600004F50570FFF71AFF04F506702169FFF7F9
:102B700015FF04F50770E168FFF710FFE069401CDE
:102B8000E0626078012304F13001E26AF8F7AAFEFE
:102B900000202071607800221146F8F753FD00B143
:102BA0000125284670BD0000525261417272416198
:102BB0002DE9F04104460027E078F8B1E56A607835
:102BC00001232A4604F13001F8F78CFE08B10127F1
:102BD00014E00020E070206A281AA16988420DD212
:102BE000A67809E0A0690544607801232A4604F12B
:102BF0003001F8F777FE761E022EF3D23846BDE894
:102C0000F0810246501A20F07F4070472DE9FE43C4
:102C100004464FF000083348007801285ED1002CAC
:102C20005CD0F9F7C5FED4E90232C01A914147D30E
:102C3000002000906846F6F7EFFD206918B94FF0C4
:102C4000FF31A160E1609DF80000F6F7EBFD6069DF
:102C50000190A0690290244A082101A8F6F7AEFA73
:102C6000054600BF2F4627B100BF3846F6F76AFA7F
:102C700000BF00BF002000906846F6F7CDFD206938
:102C800088B14FF0FF33D4E9021059405840014356
:102C900009D0D4E902302169591840F10000C4E993
:102CA0000210012600E000269DF80000F6F7BAFDAC
:102CB0002EB121460D48FCF706FA4FF001080DE051
:102CC0004FF0FF33D4E9021059405840014305D07A
:102CD00021460648FCF7F7F94FF001084046BDE8E9
:102CE000FE830000AC2D00207D0E03004C4003004D
:102CF000F8B50646694620480068FAF787FB04469F
:102D000037E0207820B1012810D0022824D11DE01E
:102D10006068D0E902104FF0FF335940584001433A
:102D200003D016486168FCF7CEF916E014496068D4
:102D30000968884203D100201149086005E00F4866
:102D40006168FCF7E4F9054600BF06E0FFF71BFCED
:102D500001200C49087000E000BF00BF694606482A
:102D60000068FAF745FB694603480068FAF74EFB2E
:102D70000446002CC5D1F8BD484003004C40030078
:102D8000A82D0020AC2D0020F8B505460E4669465A
:102D90000B480068FAF71EFB04467CB1257066609C
:102DA000694607480068FAF73FFB28B100BF0548AD
:102DB000F8F704FF00BF00BF0020F8BD0420FCE7C7
:102DC00048400300A02D00207047000010B52649A0
:102DD0002648F5F7D5FFA2202549264A126801EBBF
:102DE0000211087002202249224A126801EB0211E6
:102DF00048701D4800681E491E4A126801EB021106
:102E0000C1F802001848416819481A4A126800EBD4
:102E10000210C0F80610144881681548154A126857
:102E200000EB0210C0F80A1002211148114A126882
:102E300000EB02108173A2200D490E4A126801EBCB
:102E40000211C8730B480068401C0A490860084614
:102E50000068082806D18021054800F085FE002082
:102E60000449086010BD0000044E0020B82B00206B
:102E70001C320020502C00202DE9F043A3B0054661
:102E80000E4690461F4600203880012229462448DD
:102E9000F8F7F8FF8146B9F1000F0DD02149224A19
:102EA000891AC908012242EA01402A461FA1FBF7FC
:102EB000A7FB23B0BDE8F0830024194A802103A8B2
:102EC000F8F789FF11E001AB02AA1CA103A8F4F7EF
:102ED000D9FA029806F8140006EB440101984870EC
:102EE000641C444500DB07E000BF0D4A802103A8B5
:102EF000F8F771FF0028E6D100BF3C8009490A4A73
:102F0000891AC908032242EA014023462A460DA134
:102F1000FBF782FB0248F8F74DFF00BFC9E700004E
:102F20009C320020644F0300CC4E03006F70656E2E
:102F3000202573206661696C65640A0025782C255C
:102F4000780000006C6F6164202573206366672041
:102F500073697A653A25640A0000000070B586B08E
:102F600006460C462146304600F051F908B106B03D
:102F700070BD94F82F0018BB207B022802D0207B64
:102F800003281DD1616AA069814219D1E06960629C
:102F90006069A06294F82000C0F3401084F82C000F
:102FA000002084F82D00207B032804D121463046E0
:102FB00000F0C4F93DE02146304600F08DF838E0DD
:102FC000142204F10C0101A8F4F71BFA94F82F0065
:102FD000E0B13046FCF70BF9054605F0020018B1E8
:102FE00001208DF8000010E005F0040018B1022067
:102FF0008DF8000009E005F0010018B103208DF8FC
:10300000000002E004208DF8000002E000208DF8AE
:103010000000002084F8300094F8200000F0040044
:1030200010B194F82F0018B16846D4E900219047F8
:1030300000BF00BF9BE70146032001F001020AB177
:103040004FF4024001F002020AB148F2012001F0FF
:1030500004020AB148F20220704770B505460C46DA
:10306000A16A606B884235D200BFD5F81805C0B29E
:10307000626B616A8854606B401C6063A06A401E8A
:10308000616B814209D194F8200000F0400020B922
:1030900002212846FCF7C2F818E0A16A606B88425A
:1030A00006D194F8200000F0400008B9012070BD5E
:1030B000A16A606B884209D194F8200000F04000BA
:1030C00020B1022084F82D000020F0E720212846BE
:1030D000FCF7A7F80120EAE7F8B506460C460027FA
:1030E000344800904FF482713046FCF78DF84FF46D
:1030F00092713046FCF788F84FF48E713046FCF739
:1031000083F84FF484713046FCF77EF8002060634A
:1031100084F82F00A06A012809D194F8200000F05B
:10312000400020B902213046FCF778F803E0012185
:103130003046FCF773F820213046FCF772F894F81B
:103140002D00022803D000213046FCF76AF82068E1
:1031500038B140F28620A060A1683046FCF75BF8E9
:1031600025E002E00098401E00900098002805DD50
:103170002146304600F04BF80028F3D194F82F0098
:1031800058B13046FCF733F8054625B12846FFF71D
:1031900052FF074600E0032700BF0098002806DC26
:1031A0003046FCF71CF83046FCF71DF8032738467C
:1031B000F8BD0000A086010070B505460C46A16A66
:1031C000606B884206D2626B616A885CC5F81C0538
:1031D00000BF1AE094F82C0028B11C212846FCF707
:1031E00020F8002070BD94F8200000F0400040B1AD
:1031F0001C212846FCF715F8012084F82D0000203A
:10320000F0E714212846FCF70CF80120EAE770B536
:1032100005460C4600264FF482712846FBF7EDFF69
:1032200028B14FF482712846FBF7EEFF012694F88F
:103230002F0078B14FF492712846FBF7E5FF4FF469
:103240008E712846FBF7E0FF4FF484712846FBF7A8
:10325000DBFF5FE04FF492712846FBF7CEFF60B1D1
:103260004FF492712846FBF7CFFF14212846FBF755
:10327000D8FF012084F82F004CE04FF48E712846CF
:10328000FBF7BBFF08B34FF48E712846FBF7BCFF7A
:10329000606B401C60634FF492712846FBF7ADFFF2
:1032A00060B14FF492712846FBF7AEFF1421284617
:1032B000FBF7B7FF012084F82F002BE021462846BA
:1032C000FFF77AFF30BB002070BD4FF484712846B1
:1032D000FBF793FFF0B14FF484712846FBF794FF9E
:1032E0004FF492712846FBF788FF60B14FF492715A
:1032F0002846FBF789FF14212846FBF792FF01209F
:1033000084F82F0006E021462846FFF7A6FE08B9FC
:103310000020D9E77EB1002084F82D0094F82F001A
:1033200038B92146284600F0F1F980F0010084F810
:103330002F000020C8E70120C6E70000F8B50646C8
:103340000C4600272F4800904FF482713046FBF75F
:103350005BFF4FF492713046FBF756FF4FF48E71CE
:103360003046FBF751FF4FF484713046FBF74CFFBA
:1033700000213046FBF752FF0020606384F82F00E5
:1033800020213046FBF74DFF94F82D00012803D093
:1033900008213046FBF745FF21463046FFF70CFF7A
:1033A000206838B140F28620A060A1683046FBF763
:1033B00032FF25E002E00098401E009000980028AF
:1033C00005DD21463046FFF722FF0028F3D194F8AF
:1033D0002F0058B13046FBF70AFF054625B12846B5
:1033E000FFF729FE074600E0032700BF00980028EA
:1033F00006DC3046FBF7F3FE3046FBF7F4FE03270E
:103400003846F8BDA086010030B504461088C01CBF
:10341000984201D90C2030BD0220158848551088EB
:10342000401C10800A20158848551088401C1080C8
:1034300015884C551088401C10800020EBE7014691
:1034400008784A7840EA0220704702460A70100A5B
:1034500048700220704700002DE9FF4F81B0884678
:1034600016461F46DDE90E4B45464FF0010A03E0C4
:10347000B5FBF6F50AF1010AB542F9D2574500D974
:10348000BA460BF0010098B994B10BF00200022883
:1034900003D117B93020009001E02020009004E013
:1034A000641EDDE90010F7F753FA0CB1A245F7D31B
:1034B000012509E0012F01D97F1E04E0B8FBF5F9D1
:1034C000B14500D201E07543F4E700BF00BFB8FB8F
:1034D000F5F909FB15880D4810F809100198F7F760
:1034E00037FAB5FBF6F5002DF1D10BF0010048B12C
:1034F00044B104E0641E20210198F7F729FA0CB1C9
:10350000A245F7D305B0BDE8F08F00006640030088
:10351000F8B506463546A8B2F9F778FA04466CB312
:10352000207A1749097B88420ADAA8B204F10A0115
:10353000FEF718FD074617B1207A401C20721DE0E7
:10354000002020720E48007C50B1A8B23B2176DFEB
:10355000074627B1082F02D03846FEF7F7FC00BF18
:103560000748406950B100208DF80000A8B2ADF8BE
:103570000200034841696846884700BFF8BD000063
:10358000DC57002010B50446607940B194F82E0451
:1035900028B9204600F0B6F808B1012010BD00207F
:1035A000FCE72DE9FC478046894615469A46DDE949
:1035B0000A675346022249464046CDE9006700F0BB
:1035C00017F8044600BF204608B1BDE8FC8700BFDD
:1035D0005346102229464046CDE9006700F008F81E
:1035E000044600BF204600B1EFE700BF0020ECE733
:1035F0002DE9FF5F07468B4696461D460E9C4FF011
:10360000000920880390C84647E0786800EB8800EE
:1036100000680190002202A901A864DF064600BFED
:10362000304610B104B0BDE8F09F00BF9DF808001F
:10363000704530D1B9F1000F01D0002000E0022028
:10364000009020889DF808100144009801440F98CC
:10365000814201DD0C20E5E7B9F1000F0AD1208895
:10366000401C2080208805F800B02088401C208065
:103670004FF001092088421902A901A864DF06461B
:1036800000BF304600B1CDE700BF21889DF808009B
:103690000844208000BF08F1010838884045B4DCA8
:1036A000B9F1000F0DD021880398401C081A1FFAA9
:1036B00080FABAF1FF0F01DD0C20B3E7039805F89B
:1036C00000A00020AEE770B504460D4684B1206826
:1036D00070B12068007858B12068C088A1888842FD
:1036E00006D121684878F8F775F800F0010018B1A4
:1036F00000202860092602E0206828600026304665
:1037000070BD7047014691F83004704770B50546AA
:103710000C46A16A606B884207D02846FBF75FFD24
:103720002846FBF760FD002070BD0120FCE700008B
:1037300001480088704700004E2E0020F0B5ADB063
:10374000054600BF9DF8A80020F00F00401C2A90FD
:103750009DF8A80020F0F00010302A9000BF2868E3
:10376000F3F773FE86B232462AA829687CDF044646
:1037700000BF2746002F1AD08DA09049904A891A81
:10378000C9080322CDE9000742EA014040F23113A3
:103790008CA294A1FAF764FFFAF79CFD00BF00BF6A
:1037A00026B100BF3046F5F7CDFC00BF00BF00BF1B
:1037B00000202B902C901020ADF8AC003C20ADF8F0
:1037C000AE000020ADF8B0004FF4C870ADF8B20004
:1037D0002BA87ADF044600BF2746002F1AD074A01A
:1037E0007649774A891AC9080322CDE9000742EAD7
:1037F000014040F23B1373A27AA1FAF731FFFAF7C6
:1038000069FD00BF00BF26B100BF3046F5F79AFC46
:1038100000BF00BF00BF7B497B48F9F717FF044694
:1038200000BF2746002F1AD061A06449644A891A54
:10383000C9080322CDE9000742EA014040F24513DE
:1038400060A268A1FAF70CFFFAF744FD00BF00BFC1
:1038500026B100BF3046F5F775FC00BF00BF00BFC2
:10386000F7216948F9F7E3FE044600BF2746D7B1C0
:103870004FA05249524A891AC9080322CDE90007CC
:1038800042EA01404FF4A4734EA256A1FAF7E8FEB3
:10389000FAF720FD00BF00BF26B100BF3046F5F7A4
:1038A00051FC00BF00BF00BF686808B1686880476E
:1038B000AC2102A8F3F7BEFD02208DF8080000201D
:1038C0008DF80A0006208DF80B000121ADF8541088
:1038D0004E49169101218DF8841040212491002138
:1038E00025914B482B9002A94A48F6F702F9064663
:1038F00000BF3746D7B12EA03049314A891AC908CE
:103900000322CDE9000742EA01404FF4B8732DA22B
:1039100034A1FAF7A5FEFAF7DDFC00BF00BF24B121
:1039200000BF2046F5F70EFC00BF00BF00BF01211D
:103930003848F6F7DBF81C2126A8F3F77BFD0020BA
:1039400026904FF4A03027904FF4F02028900320C9
:103950008DF8A4000020ADF8A6008DF8A8002E4830
:103960002B902E482C9026A8F6F720FA064600BF8A
:103970003746D7B10EA01149114A891AC908032246
:10398000CDE9000742EA014040F287130DA215A1DC
:10399000FAF766FEFAF79EFC00BF00BF24B100BF35
:1039A0002046F5F7CFFB00BF00BF00BF2DB0F0BD34
:1039B0006572725F636F646500000000644F03000E
:1039C000CC4E03002E2E5C6C69627A6E6F72646955
:1039D000635C7372635C7A626C655F6D6F64756C57
:1039E000652E630025733A2564205A4552524F5282
:1039F0005F434845434B28257329206661696C3A2B
:103A00002564000035C70200047F0020482E0020F6
:103A1000BDFB0200D07A002001FC020097AE02003C
:103A20007CB503211148F6F706F9054600BF2E467E
:103A3000002E19D00EA01149114A891AC908032273
:103A4000CDE9000642EA014087230EA215A1FAF74C
:103A500007FEFAF73FFC00BF00BF24B100BF2046BD
:103A6000F5F770FB00BF00BF00BF7CBDD07A00201F
:103A70006572725F636F646500000000644F03004D
:103A8000CC4E03002E2E5C6C69627A6E6F72646994
:103A9000635C7372635C7A626C655F6D6F64756C96
:103AA000652E630025733A2564205A4552524F52C1
:103AB0005F434845434B28257329206661696C3A6A
:103AC000256400007FB505460C461148006890F853
:103AD000230010B9082004B070BD2088F42801DD4F
:103AE0000720F8E70020009001900290039008481A
:103AF0000068808AADF800000395029401208DF8DB
:103B0000020003490968098C88B26946AEDFE2E722
:103B1000582E0020704700007FB505460C4611481E
:103B2000006890F8220010B9082004B070BD208809
:103B3000F42801DD0720F8E70020009001900290B2
:103B40000390084800688088ADF80000039502944F
:103B500001208DF8020003490968098C88B2694682
:103B6000AEDFE2E7582E002013B5044601A9204637
:103B7000FFF7D2FF1CBD13B5044601A92046FFF78D
:103B8000CBFF1CBDF0B58DB004460E465D48046009
:103B90004FF0FF305B49096808845B4B0FCB08ADE1
:103BA0000FC500BF14B90E200DB0F0BD00BF00BF9F
:103BB0000EB90E20F8E700BF3068E061214608A882
:103BC00062DF054600BF284600B1EDE700BF207860
:103BD0008DF832000120ADF83000A21C0CA9A8DF3E
:103BE000054600BF284600B1DEE700BF2021684639
:103BF000F3F720FC0220ADF8000020788DF80200D9
:103C0000F420ADF804000120ADF806008DF80C009A
:103C10009DF80D0020F0080008308DF80D009DF88B
:103C20000D0020F00400001D8DF80D0000208DF81F
:103C3000110001208DF8120000BF608804F10C0211
:103C40006946F6F725FF07460FB13846ACE700BFD7
:103C500020216846F3F7EEFB0320ADF80000207842
:103C60008DF80200F420ADF804000120ADF8060044
:103C70008DF80C009DF80D0020F0100010308DF82C
:103C80000D0001208DF811008DF812008DF8130041
:103C900000BF6088221D6946F6F7FAFE07460FB19D
:103CA000384681E700BF20216846F3F7C3FB0420B4
:103CB000ADF8000020788DF80200F420ADF8040083
:103CC0000120ADF806008DF80C009DF80D0020F0E5
:103CD000100010308DF80D0001208DF811008DF8C6
:103CE00012008DF8130000BF608804F114026946C9
:103CF000F6F7CEFE07460FB1384655E700BF002065
:103D000052E70000582E00203843030004480068A2
:103D1000B0F92000401C08B1012070470020FCE7EA
:103D2000582E002070B505460E4606B105B970BD87
:103D300034462888102804D011281CD050282DD1B2
:103D400027E01849184A891AC908032242EA0140A3
:103D500016A1FAF74BFCA88800B220842189A88814
:103D6000F9F7A0FA84F822002189A888F9F79AFACD
:103D700084F8230013E00B490B4A891AC90803226F
:103D800042EA01400FA1FAF731FC4FF0FF302084E6
:103D900005E029462046FCF7AFFB00E000BF00BF6E
:103DA00000BFC4E7644F0300CC4E0300424C455FA4
:103DB0004741505F4556545F434F4E4E454354452F
:103DC00044000000424C455F4741505F4556545FF8
:103DD000444953434F4E4E45435445440000000070
:103DE00072B60449096801EB4102C2EBC11062B628
:103DF00070470000402E002000B572B6FFF7F0FFBC
:103E00004FF47A71B0FBF1F362B6184600BD0000C2
:103E10007CB54FF480410020FAF796FC044600BFC1
:103E2000254625B100BF2846F5F78CF900BF00BF35
:103E3000FAF73CFAF6F744F8044600BF254625B1E8
:103E400000BF2846F5F77EF900BF00BFF5F75CFC20
:103E5000044600BF254625B100BF2846F5F772F994
:103E600000BF00BFFAF7E6FD044600BF254625B1B6
:103E700000BF2846F5F766F900BF00BFFBF75EF804
:103E8000044600BF254625B100BF2846F5F75AF97C
:103E900000BF00BF0020019001A90120FAF79EFE9B
:103EA000044600BF254625B100BF2846F5F74AF96C
:103EB00000BF00BF01A8FAF761FF044600BF254616
:103EC00025B100BF2846F5F73DF900BF00BF0F49F7
:103ED00003C9CDE9000140F6FF70ADF800000C4ABF
:103EE00069460C48FBF7D4FB044600BF254625B1C4
:103EF00000BF2846F5F726F900BF00BF012105489D
:103F0000FBF72EFC0348FBF7B3FB7CBD30430300FB
:103F1000E50C0300284303002DE9F0430246104658
:103F200001231C460D460026374600BF202802D23A
:103F30004FF0A04803E000F01F00DFF82480C446E3
:103F400043EA440848EA850848EA062848EA074957
:103F50000CF5E06848F8209000BFBDE8F083000051
:103F60000003005002000000003002400100000089
:103F70000100000003000000882C0020A82C002075
:103F8000D8410300904503008C450300844503009D
:103F900000020000110B04057C5700200000000007
:103FA0000338FDD870470000770A000000000000C9
:103FB000770A0000000000007ADA0000000000002C
:103FC00000000050000300506E7266785F677069F1
:103FD0006F74655F696E6974006E7266785F677092
:103FE000696F74655F6F75745F696E6974006E7276
:103FF00066785F6770696F74655F696E5F696E6927
:10400000740000006E7266785F7370696D5F696E30
:10401000697400002D850200558502007370696D7A
:104020005F78666572006E7266785F7370696D5F47
:104030007866657200000000FFFFFFFF0006FF00CA
:104040000000004000000000845A00200000000032
:10405000C02D00205BAD0200010006000000000042
:104060000338FDD87047303132333435363738397C
:104070004142434445460000984F03009C4F0300D3
:104080000000000000000000000000000000000030
:10409000784003009040030004000000556E6B6EF2
:1040A0006F776E206572726F7220636F64650000B7
:1040B00000000000504A030001000000FC4803001B
:1040C00002000000F04603000300000070490300F6
:1040D00004000000C449030005000000A4480300D8
:1040E000060000004048030007000000AC49030040
:1040F00008000000B8480300090000001C49030044
:104100000A000000384A03000B000000D8460300F4
:104110000C000000D04803000D000000A04A03007E
:104120000E0000009C4903000F000000D849030066
:10413000100000000C4A030011000000B44A030004
:1041400012000000884A030013000000244A030004
:1041500080000000584803008100000094470300DD
:10416000820000005447030083000000344703002E
:104170008400000070470300850000007C480300B5
:1041800086000000844903009000000020480300DE
:10419000910000001447030092000000E44803006F
:1041A00000820000EC49030001820000384903004E
:1041B000028200005449030000840000B04703005D
:1041C000018400005C4A030002840000F8470300F9
:1041D00003840000D4470300D9A5020021A70200F0
:1041E00095A6020081A7020061A60200D1A50200E7
:1041F00002000000000000000000000003000000BA
:1042000000000000000000000001000000000000AD
:10421000000000000100000000000000000000009D
:104220000201000000000000000000000201000088
:10423000000000000000000000000000003000400E
:104240000000000001000000000000FF06FF000069
:10425000000000040000000000000000000000005A
:104260005DE102005BE1020051E10200000000009C
:104270000338FDD87047000010660020FF010000E1
:104280001068002000000000000000000000000096
:104290000000000084420300944203000800000074
:1042A0000450030014500300000000000000000050
:1042B000A0420300B042030008000000F44F0300D6
:1042C000045003000000000000000000BC42030096
:1042D000CC42030008000000001002019C4F0300C4
:1042E000A44F0300A44F0300C44F0300C44F0300B6
:1042F000DC4F0300DC4F0300E44F0300DC4203000B
:10430000FC42030008000000B82B0020E44F03002B
:10431000EC4F0300EC4F0300F44F03000C43030089
:104320001C43030008000000004002402400040079
:1043300000000641000000009ECADC240EE5A9E052
:1043400093F3A3B50000406E0200000000000000DF
:1043500050EADA308883B89F604F15F30000C98EA9
:104360000040404040404040404041414141414088
:10437000404040404040404040404040404040403D
:1043800040050202020202020202020202020202CC
:1043900002202020202020202020200202020202D1
:1043A0000202909090909090101010101010101029
:1043B0001010101010101010101010100202020235
:1043C0000202888888888888080808080808080879
:1043D0000808080808080808080808080202020275
:1043E00040000000614303006E7266785F67706989
:1043F0006F74655F696E5F696E69742841445331FB
:104400003239335F52454144595F50494E2C202682
:10441000696E436F6E6669672C206164733132394F
:10442000335F72656164795F70696E5F697271296B
:10443000000000006170705F74696D65725F637287
:104440006561746528266D5F7265636F72645F7560
:10445000706C6F61645F746D722C204150505F54BA
:10446000494D45525F4D4F44455F5245504541547B
:1044700045442C205265636F726455706C6F6164A3
:104480005F746D725F636229000000006170705F8D
:1044900074696D65725F63726561746528266D5F0E
:1044A0007265636F72645F75706C6F61645F66697B
:1044B0006E6973685F7061636B65745F7265706F5E
:1044C00072745F746D722C204150505F54494D4599
:1044D000525F4D4F44455F53494E474C455F5348EB
:1044E0004F542C205265636F726455706C6F616419
:1044F0005F66696E6973685F7061636B65745F7234
:1045000065706F72745F746D725F63622900000082
:104510006170705F74696D65725F73746172742825
:104520006D5F7265636F72645F75706C6F61645FFD
:1045300066696E6973685F7061636B65745F7265ED
:10454000706F72745F746D722C204150505F5449CB
:104550004D45525F5449434B53283330292C202872
:10456000766F69642A296D5F7265706F72745F641B
:104570006174615F73756D636865636B636F6465B8
:1045800029000000312E3030000000005344430069
:1045900049464C59544F50005265717565737469A2
:1045A0006E6720746F207570646174652041545487
:1045B000204D545520746F202575206279746573E1
:1045C000206F6E20636F6E6E656374696F6E20304E
:1045D00078257820287265747279292E00000000F1
:1045E00073645F626C655F6761705F646174615F73
:1045F0006C656E6774685F757064617465282920E6
:10460000287265717565737429206F6E20636F6EF3
:104610006E656374696F6E203078257820726574DA
:1046200075726E65642025732E0000005468652045
:1046300072657175657374656420636F6D62696E10
:104640006174696F6E206F6620545820616E64201B
:104650005258207061636B6574206C656E67746876
:104660007320697320746F6F206C6F6E672062799E
:10467000202575206D6963726F7365636F6E647357
:104680002E00000073645F626C655F676174746321
:104690005F65786368616E67655F6D74755F72658D
:1046A00071756573742829206F6E20636F6E6E6557
:1046B0006374696F6E203078257820726574757226
:1046C0006E656420627573792C2077696C6C20723A
:1046D000657472792E0000004E52465F4552524F6B
:1046E000525F494E56414C49445F44415441000099
:1046F0004E52465F4552524F525F534F46544445C7
:10470000564943455F4E4F545F454E41424C4544E8
:10471000000000004E52465F4552524F525F4645E0
:1047200041545552455F4E4F545F454E41424C45B2
:10473000440000004E52465F4552524F525F4D5565
:104740005445585F554E4C4F434B5F4641494C458D
:10475000440000004E52465F4552524F525F4D5545
:104760005445585F4C4F434B5F4641494C454400CC
:104770004E52465F4552524F525F4D555445585F19
:10478000434F4E445F494E49545F4641494C45446E
:10479000000000004E52465F4552524F525F4D5549
:1047A0005445585F494E49545F4641494C45440081
:1047B0004E52465F4552524F525F424C455F495000
:1047C00053505F52585F504B545F5452554E4341C3
:1047D000544544004E52465F4552524F525F424C40
:1047E000455F495053505F504545525F52454A45D9
:1047F00043544544000000004E52465F4552524F1C
:10480000525F424C455F495053505F4C494E4B5F9D
:10481000444953434F4E4E45435445440000000025
:104820004E52465F4552524F525F4150495F4E4F84
:10483000545F494D504C454D454E54454400000091
:104840004E52465F4552524F525F4E4F545F535542
:1048500050504F52544544004E52465F4552524FBD
:10486000525F4D4F44554C455F4E4F545F494E4942
:104870005449414C495A4544000000004E52465F9D
:104880004552524F525F4D4F44554C455F414C523B
:10489000454144595F494E495449414C495A454460
:1048A000000000004E52465F4552524F525F4E4F3D
:1048B000545F464F554E44004E52465F4552524F4C
:1048C000525F494E56414C49445F53544154450050
:1048D0004E52465F4552524F525F444154415F53DE
:1048E000495A45004E52465F4552524F525F494F1A
:1048F0005F50454E44494E47000000004E52465F0F
:104900004552524F525F5356435F48414E444C45C7
:10491000525F4D495353494E470000004E52465F87
:104920004552524F525F494E56414C49445F4C45A7
:104930004E475448000000004E52465F4552524FC9
:10494000525F4452565F5457495F4552525F414E41
:1049500041434B004E52465F4552524F525F4452C4
:10496000565F5457495F4552525F444E41434B0096
:104970004E52465F4552524F525F494E5445524E39
:10498000414C00004E52465F4552524F525F5354C5
:104990004F524147455F46554C4C00004E52465FD2
:1049A0004552524F525F4E554C4C00004E52465F9E
:1049B0004552524F525F494E56414C49445F504117
:1049C00052414D004E52465F4552524F525F4E4F3C
:1049D0005F4D454D000000004E52465F4552524F1C
:1049E000525F464F5242494444454E004E52465F44
:1049F0004552524F525F4452565F5457495F455299
:104A0000525F4F56455252554E0000004E52465F7F
:104A10004552524F525F494E56414C49445F4144C2
:104A2000445200004E52465F4552524F525F52452B
:104A3000534F5552434553004E52465F4552524FD5
:104A4000525F494E56414C49445F464C41475300E2
:104A50004E52465F53554343455353004E52465FB3
:104A60004552524F525F424C455F495053505F434D
:104A700048414E4E454C5F414C52454144595F457B
:104A800058495354530000004E52465F4552524F0E
:104A9000525F434F4E4E5F434F554E54000000004F
:104AA0004E52465F4552524F525F54494D454F5505
:104AB000540000004E52465F4552524F525F4255DD
:104AC000535900007761726E696E670064656275A4
:104AD000670000001B5B313B33306D001B5B306DAA
:104AE000000000001B5B313B33316D001B5B313B31
:104AF00033326D001B5B313B33336D001B5B313B4D
:104B000033346D001B5B313B33356D001B5B313B38
:104B100033366D001B5B313B33376D00696E666F5A
:104B2000000000006572726F7200000073645F62C3
:104B30006C655F6366675F736574282920726574AE
:104B400075726E6564202573207768656E206174C8
:104B500074656D7074696E6720746F20736574205E
:104B6000424C455F47415454535F4346475F53456A
:104B700052564943455F4348414E4745442E000045
:104B800073645F626C655F6366675F736574282931
:104B90002072657475726E65642025732077686570
:104BA0006E20617474656D7074696E6720746F2017
:104BB00073657420424C455F434F4D4D4F4E5F43EC
:104BC00046475F56535F555549442E0073645F62F4
:104BD0006C655F6366675F7365742829207265740E
:104BE00075726E6564202573207768656E20617428
:104BF00074656D7074696E6720746F2073657420BE
:104C0000424C455F47415454535F4346475F4154CC
:104C100054525F5441425F53495A452E00000000F0
:104C200073645F626C655F6366675F736574282990
:104C30002072657475726E656420257320776865CF
:104C40006E20617474656D7074696E6720746F2076
:104C500073657420424C455F434F4E4E5F43464759
:104C60005F4741502E00000073645F626C655F63B4
:104C700066675F73657428292072657475726E6546
:104C800064202573207768656E20617474656D708B
:104C900074696E6720746F2073657420424C455FA1
:104CA0004741505F4346475F524F4C455F434F5526
:104CB0004E542E0073645F626C655F6366675F735A
:104CC000657428292072657475726E656420257379
:104CD000207768656E20617474656D7074696E67A5
:104CE00020746F2073657420424C455F434F4E4ED5
:104CF0005F4346475F474154542E00005468652087
:104D0000626F6F746C6F6164657220686173207785
:104D1000726974652070726F74656374656420696C
:104D200074732073657474696E677320706167654E
:104D30002E20546869732070726F68696269747399
:104D40002073657474696E67207468652061647689
:104D50006572746973696E67206E616D652E20548B
:104D6000686520626F6F746C6F61646572206D7529
:104D7000737420626520636F6D70696C6564207761
:104D8000697468204E52465F424C5F534554544903
:104D90004E47535F504147455F50524F544543542F
:104DA0003D3020746F20616C6C6F77207365747474
:104DB000696E6720746865206164766572746973D2
:104DC000696E67206E616D652E0000006E72665F11
:104DD000626C655F6761747400000000626C655FFF
:104DE0006E757300636C6F636B000000434C4F4340
:104DF0004B0000004750494F5445000050525300AB
:104E000055415254000000005541525445000000E5
:104E100053414144430000005350494D00000000FD
:104E20005457490050574D005744540052544300C2
:104E300054494D45520000006170705F6275747492
:104E40006F6E00006170705F74696D6572000000C4
:104E50007077725F6D676D7400000000736F72741D
:104E60006C697374000000007274745F6C6F675F2C
:104E70006261636B656E6400617070006E72665F84
:104E8000736468006E72665F7364685F626C65006D
:104E90006E72665F7364685F736F63001450030023
:104EA000B82B0020BC020000E07902000051030092
:104EB000742E0020EC600000AA8A02006042030009
:104EC00000000000684E0300E82D0020CC4D0300D8
:104ED00000000404DC4D030000000000E44D03006A
:104EE00000000000EC4D030000000000F44D030042
:104EF00000000000FC4D030000000000004E030015
:104F000000000000084E030000000000104E0300E7
:104F100000000000184E030000000000204E0300B7
:104F200000000000244E030000000000284E030093
:104F3000000000002C4E030000000000304E030073
:104F400000000000384E030000000000444E030043
:104F500000000000504E0300000000005C4E030003
:104F600000000000784E0300000004047C4E0300A3
:104F700000000303844E030000000303904E03006F
:104F800000000303F02D0020085F0020305F0020A8
:104F9000305F00202C0000002D96020029A20200A4
:104FA0000000000071A1020000000000E9A1020061
:104FB00000000000FB9B0200D07A002081D6020096
:104FC000047F0020253D030074300020253D0300B0
:104FD0001C510020A99F0200187F0020E1A20200BE
:104FE000000000004D2503000000000081A0020029
:104FF00000000000C9EE020000000000FDEF02000A
:1050000000000000990F03000000000095A90200B5
:1050100000000000A110080119022E031604120559
:105020001406080712081209100A0A170B070C7455
:105030000D010E160F03100511161205133F141261
:10504000151216141705181219121A121B121C1217
:105050001D100A2101222023202420251226162794
:1050600008280829122A122B122C122D162E332F43
:1050700070301231123212331234123512361237A6
:1050800012381239123A123B123C123D123E123FB4
:105090001440FF501260021B621AFF015306FF0208
:1050A00028402934290109362001400922800114B1
:1050B00064803F03024F0115100140110A4404DCD3
:1050C000A90C59AF14244B0314C44A031A1C081A20
:1050D000CC081ADC041AD4041AE4041AEC041AF4F6
:1050E000041AFC041A04201A0C041A1404F9FC1102
:1050F0001492650112020422FFFF14040090D003F1
:040000050002720182
:00000001FF
